:020000040800F2
:10000000F8B5012099010008915000080D41000841
:10001000714900083B100008D97D0008000000006D
:10002000000000000000000000000000B1710008A6
:10003000D516000800000000070200081D73000824
:10004000B3010008B3010008B3010008B3010008C0
:10005000B3010008B3010008B3010008B3010008B0
:10006000B3010008B3010008B3010008B3010008A0
:10007000B3010008B3010008B3010008B301000890
:10008000B3010008B3010008B3010008B301000880
:10009000B3010008B3010008B3010008B301000870
:1000A000B3010008B3010008B3010008B301000860
:1000B000B3010008B3010008B3010008B301000850
:1000C000B3010008B3010008B3010008B301000840
:1000D000B3010008B3010008B3010008A9730008C8
:1000E000B3010008B3010008B3010008B301000820
:1000F000B3010008B3010008B3010008B301000810
:10010000B3010008B3010008B3010008B3010008FF
:10011000B3010008B3010008B3010008B3010008EF
:10012000B3010008B3010008B3010008B3010008DF
:10013000B3010008051E0008B3010008B301000860
:10014000B3010008B3010008B3010008B3010008BF
:1001500041100008B3010008B3010008B1730008A2
:10016000B3010008B3010008B3010008B30100089F
:10017000B3010008B3010008B3010008B30100088F
:10018000B3010008DFF80CD000F084FD0048004700
:10019000E91D0108F8B501200648804706480047D8
:1001A000FEE7FEE7FEE7FEE7FEE7FEE7FEE7FEE727
:1001B000FEE7FEE74173000885010008EFF31080B9
:1001C00072B6704780F3108870471F484FF0FF01E8
:1001D0000170002080F309881C48016881F30888B9
:1001E0001B48012101701B484FF08051016062B62D
:1001F000FEE718484FF080510160704715484FF0F6
:1002000080510160704772B6EFF3098028B1203841
:1002100080E8F00F10490968086000B50F48804772
:100220005DF804EB0E480F490A7802700A480E493F
:100230000A680260106890E8F00F203080F30988A7
:100240004EF0040E62B6704722ED00E0E0000020A0
:10025000A500002004ED00E0AC00002029600008AB
:100260009E0000209F000020B40000202DE9F05FD8
:100270000546002092469B46884606468146402415
:100280001BE0284641464746224600F0CCFB534639
:100290005A46C01A914110D311461846224600F022
:1002A000B3FB2D1A67EB01084F46224601200021BF
:1002B00000F0AAFB17EB00094E41201EA4F1010437
:1002C000DFDC484631462A464346BDE8F09F40EA17
:1002D00001039B0703D009E008C9121F08C0042AC4
:1002E000FAD203E011F8013B00F8013B521EF9D2AB
:1002F0007047D2B201E000F8012B491EFBD27047D3
:100300000022F6E710B513460A4604461946FFF7E1
:10031000F0FF204610BD421E12F8013F002BFBD11A
:1003200011F8013B02F8013B002BF9D1704730B5C1
:1003300005462A460B4612F8010B13F8014B08B18B
:10034000A042F8D01CB1002802D06D1CF1E728466D
:1003500030BD421C10F8011B0029FBD1801A7047E8
:1003600010B5002200E0521C835C8C5CA34201D1DA
:10037000002BF8D1D8B2E1B2401A10BD30B5044616
:100380000020034600E05B1C934203D2E05CCD5C9E
:10039000401BF8D030BD034611F8012B00F8012BAB
:1003A000002AF9D11846704730B5054600200346AB
:1003B00000E05B1C934205D2EC5CC85C201A01D1C2
:1003C000002CF6D130BD00000FB400B58DB010A9DF
:1003D00009900B9000914FF0FF300A9000200C9094
:1003E00005480690054807906A4609A80F9900F04D
:1003F0005FFB0DB05DF814FBCD0A0008EB0A0008A6
:100400002DE9FF5F1D464FF0FF3BD5E901469146C0
:100410005F464FF00008A9697F1C01988847296A48
:10042000824688470028F6D1BAF1FF3F0CD024F469
:10043000C064002E19DD600614D5BAF12B0F09D067
:10044000BAF12D0F0ED103E0584604B0BDE8F09F7D
:1004500044F48064A9697F1C01988847761E82460F
:10046000002E02DDBAF1300F03D0B9F1000F26D013
:1004700032E0A969761E44F400747F1C0198884715
:100480008246002E05DDBAF1780F06D0BAF1580F7A
:1004900003D0B9F1000F10D01EE0B9F1000F02D067
:1004A000B9F1100F18D1A969761E24F400747F1CCD
:1004B000019888478246102002E0082000E00A20C8
:1004C000814609E008FB0908A969761E44F4007416
:1004D0007F1C019888478246002E05DD494650461C
:1004E00000F0D1FA0028EDDAE96901988847A00503
:1004F00002D46FF00100A8E7E00725D1600613D50C
:10050000600502D5C8F1000000E0404629680A1DD8
:100510002A600968220501D5087015E0220701D577
:10052000088011E008600FE02868011D296000685C
:10053000210502D580F8008006E0210702D5A0F849
:10054000008001E0C0F8008038467EE72DE9FF5FBB
:10055000D2E901A74FF00008916999461446DDF8E9
:1005600038B0464601988847054659EA0B0005D041
:1005700009E0A169761C019888470546216A28464A
:1005800088470028F5D1681C03D05FEACA7005D0FF
:1005900015E04FF0FF3004B0BDE8F09F2068011D6A
:1005A0002160D0F800800AE05FEACA7001D108F843
:1005B000015BA169761C7F1E019888470546002FC4
:1005C0001ADD681C18D0B9F1000F0DD0E81705EB43
:1005D000D060421120F01F0059F822102A1A012081
:1005E00090400142E0D107E0BBF1000FDCD1216A6D
:1005F000284688470028D7D0E16901988847BBF191
:10060000000F07D1002E05DD5FEACA7002D100217C
:1006100088F80010A068B84203DDBBF1000F03D0DA
:1006200017B16FF00100B6E73046B4E72DE9F047A7
:1006300091460F4680460446002614F8015B2DB112
:1006400000F014FA0068405DC007F6D12B2D02D0EF
:100650002D2D18D0641E4A463946204600F056FA21
:1006600027B13968A14201D1C7F8008071054FF068
:1006700002040BD54042002803DD07F0D3FB0460E1
:10068000A007BDE8F08746F48066E4E70028F8DAC2
:1006900007F0C8FB04606FF00040F2E72DE9FE4F61
:1006A000804681EA0300C00F0C46009021F0004113
:1006B00023F00045B8EB0200A94105D2404621468F
:1006C00090461C460B46024623F00040104347D09C
:1006D000270DC7F30A00C3F30A510290401A019094
:1006E00040286BDAC3F3130040F4801B0098924655
:1006F00020B10023D2EB030A63EB0B0B01985946A0
:10070000C0F14002504600F07FF906460D465046C3
:100710005946019A00F097F910EB08006141002456
:1007200087EA115284EAE7731A4340D0009A62B311
:10073000019A012A4FEA075215DC001B61EB020106
:100740004FF0004202EA0752CDE90042001C41F599
:10075000801132462B4600F037FA03B0BDE8F08F27
:1007600040462146F9E7001B61EB0201001C41F500
:10077000801300185B412018A2F5001747EB030116
:1007800040EAD570B6196D4111E06D084FEA3606A2
:1007900045EAC0754FEA0752001B61EB0201001CDD
:1007A00041F5801149084FEA3000001951413246A5
:1007B0002B4603B0BDE8F04F00F0F7B900980122D6
:1007C00040000023D0EB020263EBE0730098214667
:1007D0004FEAE074B8EB000061EB0401E9E783F055
:1007E00000435BE781F0004158E72DE9FE4F81EAC5
:1007F000030404F0004421F0004100944FF0000B8A
:1008000023F0004350EA01045ED052EA03045BD0B7
:10081000C3F30A54C1F30A552C44A4F2F3340194EF
:10082000A0FB0254C1F3130141F48011C3F313037D
:1008300043F4801301FB024400FB034E840A970A31
:1008400044EA815447EA8357A4FB076802958D0A5E
:1008500005FB07854FEA932C04FB0C542705029DEA
:100860004FEA065847EA1637B5EB08056EEB070C5A
:10087000870E920E47EA811742EA8312A7FB020114
:10088000B6EB0B0164EB00042B0D43EA0C335E184E
:1008900044EB1C50DA465146E7FB0201C5F3130452
:1008A0004FEA0B3343EA14534FEA0432019C43EA04
:1008B0000603A4F10C040294009CCDE900B400F0FE
:1008C00083F903B0BDE8F08F00200146F9E72DE978
:1008D000F04D81EA030404F0004B21F0004514467A
:1008E0004FF0000A23F0004150EA050220D054EAFC
:1008F00001021DD0C5F30A570246C5F31303C1F325
:100900001300C1F30A5640F4801543F48013A7EB9B
:100910000608101BD64608F2FD3873EB050002D31B
:1009200008F1010801E092185B41B8F1000F03DA09
:1009300000200146BDE8F08D00204FF480110646EE
:1009400084460EE0171B73EB050705D3121B63EB00
:10095000050306434CEA010C49084FEA300092189F
:100960005B4150EA0107EDD152EA030012D082EA5E
:10097000040083EA0501084305D0101BAB4106D2F1
:100980000122002306E000224FF0004302E06FF056
:10099000010253101AEB06004CEB085110EB0A0051
:1009A00041EB0B01BDE8F04D00F0FFB830B5041E7F
:1009B00071F1000404DB4FF00044404264EB01019C
:1009C000141E73F1000405DB1C464FF00043524235
:1009D00063EB0403994208BF904230BD30B50B462B
:1009E000014600202022012409E021FA02F59D425F
:1009F00005D303FA02F5491B04FA02F52844151E33
:100A0000A2F10102F1DC30BD202A04DB203A00FA19
:100A100002F1002070479140C2F1200320FA03F355
:100A2000194390407047202A04DB203A21FA02F053
:100A30000021704721FA02F3D040C2F12002914018
:100A4000084319467047202A06DBCB17203A41FAA3
:100A500002F043EAE07306E041FA02F3D040C2F14B
:100A60002002914008431946704700000048704733
:100A7000CC56040810B50446FFF7F8FF0068005D87
:100A800000F0010010BD3A2800D2303820F02002DA
:100A9000412A01D3A2F13700884201D34FF0FF3041
:100AA00070470000026811441378016018467047CF
:100AB000D16004495161044911620021116111465C
:100AC00000F0FAB8A50A0008750A0008426842B1A9
:100AD000016811F8013B23B1521EC0E9001218460B
:100AE00070470121C160881E704742685AB1C368CF
:100AF000016843B983688B4205D0491E521CC0E986
:100B00000012002070474FF0FF3070472DE9F05F72
:100B100082460078002715468B460AF10104B94643
:100B2000302801D09DB113E014F8010B012778287B
:100B300003D0582801D045B10AE00DB1102D07D1DE
:100B40000027102514F8010B02E0082500E00A2513
:100B50000026B0460EE005FB080005FB06F1012764
:100B600001EB10461FFA80F8B6F5803F00D3B94676
:100B700014F8010B2946FFF786FF0028EBDABBF1DA
:100B8000000F05D00FB1641E00E05446CBF80040C2
:100B9000B9F1000F06D007F045F902210160C81E27
:100BA000BDE8F09F48EA0640FAE710B5141E73F15D
:100BB000000408DA401C41F1000192185B411A431D
:100BC00001D120F0010010BD2DE9F04D92469B4669
:100BD00011B1B1FA81F202E0B0FA80F2203290460F
:100BE000FFF712FF04460F4640EA0A0041EA0B01F4
:100BF00053465A46084313D0114653EA010019D010
:100C0000C8F140025046FFF70EFF05460E4650461B
:100C100059464246FFF7F8FE084305D0012004E09C
:100C200020463946BDE8F08D0020054346EAE076CF
:100C30002C4337430A986305E40AA0EB080000221E
:100C4000FD0A44EA47540A3002D500200146E9E78C
:100C5000010510196941DDE9084500196941BDE840
:100C6000F04DA2E7C1F30A52C1F3130140F2FF3382
:100C700041F480119A4202DA00200146704740F2A6
:100C800033439A42A2F2334202DC5242FFF7CBBE18
:100C9000FFF7BABE064C074D06E0E06840F00103DE
:100CA00094E8070098471034AC42F6D3FFF76EFA89
:100CB000A8590408C85904082DE9F34F8BB04FF028
:100CC000000801F10C000C464FF0010B46460DF1F7
:100CD000080A01906269012101989047051E2DD0F4
:100CE000252D2CD0216A8847C0B162690121019865
:100CF0009047216A88470028F7D1411E6269019810
:100D0000904700E0761CA1690B988847216A8847C4
:100D10000028F7D1E1690B988847DBE7A1690B98B8
:100D200088470746A84201D1761CD3E7E1690B98B2
:100D300088477F1C02D1B8F1000F6FD046E1002731
:100D400062693D463946019890472A2804D1626974
:100D50000121019890470125DFF884926269012101
:100D600001989047A0F130010A290AD24F45E5DCED
:100D700007EB870100EB4107303FDFD445F010055A
:100D8000ECE7E90601D46FF000476C280AD04C2844
:100D900014D0682815D06A280DD074281CD07A2861
:100DA0001AD01DE062690121019890476C2802D099
:100DB00045F0040514E045F002050DE045F020057E
:100DC0000AE06269012101989047682802D045F045
:100DD000080505E045F40065626901210198904726
:100DE000C4E9015765283DD019DC58287AD00CDCBD
:100DF000452837D004DC252826D0412831D131E0E0
:100E000046282FD047282CD12CE05B2877D06128AA
:100E100028D063287CD0642823D15AE0D0E06F2802
:100E200048D008DC66281DD067281BD0692821D04F
:100E30006E2816D127E0702845D0732868D0752811
:100E400047D078280DD14DE0A1690B988847054619
:100E500025283FF469AFE1690B9888476D1C3FF482
:100E60006AAFB3E023466A466FF001000B99AFF317
:100E700000809EE045F040006060A80723464FF0E8
:100E8000000236D43EE0E8077FF447AF2068011D3A
:100E900021600068290501D506701BE7290701D5E7
:100EA000068017E7A90703D5F117C0E9006111E72C
:100EB00006600FE745F040006060A80723464FF04A
:100EC000080216D41EE040F60E0125EA010060601B
:100ED00016E045F040006060A80723464FF00A0284
:100EE00007D40FE045F040006060A80708D523460E
:100EF00010226FF001000B99AFF3008059E007E07A
:100F0000234610226FF001000B99FFF779FA50E0A9
:100F10004FF000094F464B46632802D05B2806D0AD
:100F200040E0E80601D40120A06001273AE06269B0
:100F30000121019890475E2805D14FF001096269AF
:100F4000494601989047216939B900210A4653461C
:100F500043F82120491C0829FADBB0B3216969B99B
:100F6000C11700EBD16253110AEB830122F01F027B
:100F7000821A01200B68904003430B6062690121D3
:100F8000019890475D28E8D1B9F1000F09D0002001
:100F9000514651F82020D24341F82020401C082817
:100FA000F7DB02AB224600976FF001000B99FFF7C9
:100FB000CDFA00280CDA401C08D1BBF1000F05D097
:100FC0004FF0FF300DB0BDE8F08FFFE74046F9E786
:100FD000E90701D108F1010806444FF0000B79E65A
:100FE000CCCCCC0C70B58C1810F8015B15F0070355
:100FF00001D110F8013B2A1106D110F8012B03E0B2
:1010000010F8016B01F8016B5B1EF9D12B0705D4B9
:101010000023521E0DD401F8013BFAE710F8013B02
:10102000CB1A921C03E013F8015B01F8015B521E1E
:10103000F9D5A142D8D3002070BD00BFFEE7000063
:1010400010B50549054800F0E9F918B1024903480F
:1010500000F08CF810BD00000088001028640240E9
:1010600070B504460D46344884423AD032481830B0
:10107000844236D030483030844232D02E48483016
:1010800084422ED02C48603084422AD02A487830BE
:10109000844226D028489030844222D02648A83066
:1010A00084421ED0254884421BD0244818308442F4
:1010B00017D022483030844213D020484830844230
:1010C0000FD01E48603084420BD01C4878308442D8
:1010D00007D01A489030844203D01848A830844280
:1010E00000D104E040F2214115A007F033FE05F0E5
:1010F0004050B0F1405F07D005F0405020B1194892
:10110000284008B905B104E040F222410CA007F0E4
:1011100021FE0A48844202D2074E103E01E0074EEB
:10112000103E05F0005018B10F482840F06002E072
:101130000D482840B06070BD10600240106402404D
:101140002E2E5C4C69627261726965735C737263A6
:101150005C73746D3332663278785F646D612E63D0
:101160000000000082F082C07D0F7D0F70B5044644
:101170000D46344884423AD032481830844236D042
:1011800030483030844232D02E48483084422ED00D
:101190002C48603084422AD02A487830844226D0B5
:1011A00028489030844222D02648A83084421ED05D
:1011B000254884421BD024481830844217D0224846
:1011C0003030844213D02048483084420FD01E482B
:1011D000603084420BD01C487830844207D01A48D3
:1011E0009030844203D01848A830844200D104E0F3
:1011F00040F2D64115A007F0ADFD05F04050B0F12A
:10120000405F07D005F0405020B11DB1184828407C
:1012100000B904E040F2D7410CA007F09BFD0A485A
:10122000844202D2074E103E01E0074E103E05F008
:10123000005018B10F482840F06002E00D482840E7
:10124000B06070BD10600240106402402E2E5C4CF5
:1012500069627261726965735C7372635C73746DE9
:101260003332663278785F646D612E63000000006F
:10127000820082407D0F7D0F70B504460D462C48DC
:1012800084423AD02A481830844236D02848303038
:10129000844232D02648483084422ED024486030E0
:1012A00084422AD022487830844226D02048903088
:1012B000844222D01E48A83084421ED01D48844259
:1012C0001BD01C481830844217D01A483030844252
:1012D00013D01848483084420FD0164860308442FA
:1012E0000BD014487830844207D0124890308442A2
:1012F00003D01048A830844200D104E04FF4EC71D0
:101300000DA007F027FD0DB1012D00D104E040F242
:10131000D91109A007F01EFD25B1206840F0010099
:10132000206003E0206820F00100206070BD000014
:1013300010600240106402402E2E5C4C69627261A3
:10134000726965735C7372635C73746D3332663299
:1013500078785F646D612E630000000010B504466C
:10136000234884423AD022481830844236D020485C
:101370003030844232D01E48483084422ED01C483F
:10138000603084422AD01A487830844226D01848E7
:101390009030844222D01648A83084421ED015488E
:1013A00084421BD013481830844217D01148303083
:1013B000844213D00F48483084420FD00D4860302B
:1013C00084420BD00B487830844207D009489030D3
:1013D000844203D00748A830844200D104E040F2A0
:1013E000832105A007F0B6FC606880B210BD000044
:1013F00010600240106402402E2E5C4C69627261E3
:10140000726965735C7372635C73746D33326632D8
:1014100078785F646D612E63000000002DE9F0476D
:1014200005460C464FF000080027B946784885422B
:101430003AD077481830854236D0754830308542EA
:1014400032D07348483085422ED071486030854292
:101450002AD06F487830854226D06D48903085423A
:1014600022D06B48A83085421ED06A4885421BD0E6
:1014700068481830854217D066483030854213D00E
:101480006448483085420FD06248603085420BD0B6
:1014900060487830854207D05E489030854203D05E
:1014A0005C48A830854200D104E040F286415AA051
:1014B00007F050FC6148844278D06148844275D07E
:1014C0006048844272D0604884426FD05F48844252
:1014D0006CD05F48844269D05E48844266D05E48E2
:1014E000844263D05848FC3084425FD057483F3034
:1014F00084425BD05948844258D05948844255D0E0
:101500005848844252D0584884424FD05748844269
:101510004CD05748844249D05648844246D0564819
:10152000844243D05548844240D0554884423DD0FF
:10153000544884423AD05448844237D05348844275
:1015400034D05348844231D0524884422ED052483D
:1015500084422BD05148844228D05148844225D01F
:101560004B48FC30844221D04A483F3084421DD051
:101570004C4884421AD04C48844217D04B4884428D
:1015800014D04B48844211D04A4884420ED04A4875
:1015900084420BD04948844208D04948844205D04F
:1015A0004848844202D04848844200D104E040F2D6
:1015B000874119A007F0CEFB1648854202D2144E8F
:1015C000103E01E0134E103E4048204030B11E2036
:1015D00000EAD427286800EA070902E0686900F0F9
:1015E000800904F0005008B1776800E03768384897
:1015F000074007EA040028B1B9F1000F02D04FF00C
:10160000010801E04FF000084046BDE8F087000007
:1016100010600240106402402E2E5C4C69627261C0
:10162000726965735C7372635C73746D33326632B6
:1016300078785F646D612E630000000020800010E8
:10164000104000100820001004100010010000904D
:1016500000880010004400100022001000802010BC
:10166000004010100020081000100410000001902D
:10167000008000180040001400200012001000112B
:101680000000409020800020104000200820002012
:1016900004100020010000A0008800200044002069
:1016A0000022002000802020004010200020082080
:1016B00000100420000001A0008000280040002449
:1016C0000020002200100021000040A03C0F3C0F31
:1016D0007D0F7D0F7047000030B5ADF5197D0546D3
:1016E0002A4616A1684606F089FB002215A10DA81E
:1016F0000CF0EAFA04461CB1214613A006F06EFB7A
:1017000068460CF055FD044624B9294614A006F09D
:1017100065FB0BE0042C04D1294616A006F05EFB05
:1017200004E0224629461AA006F058FB002205A133
:1017300010460CF0C9FA0DF5197D30BD303A2F2551
:1017400073000000303A0000B9D2D4D8CEC4BCFE39
:10175000CFB5CDB3CAA7B0DC20282564290D0A0077
:10176000C9BEB3FDCEC4BCFE20257320B3C9B9A643
:101770000D0A0000C3BBD3D0B7A2CFD6CEC4BCFEE7
:10178000BBF2C4BFC2BC203A25730D0A00000000A2
:10179000C9BEB3FD2573CAA7B0DC28B4EDCEF3B43F
:1017A000FAC2EB203D2025642920CEC4BCFED6BB66
:1017B000B6C1BBF2C4BFC2BCB7C7BFD50D0A0000DB
:1017C00010B500F0A5F901F07DF800F0B7FF08486A
:1017D000007800F0010008B101F056F80DF05CFA55
:1017E00028B10348006840F010000149086010BDAE
:1017F0006C00002010B504460648204008B904B12A
:1018000004E040F2927104A007F0A4FA0B4844618E
:1018100010BD00000018FEFF2E2E5C4C6962726144
:10182000726965735C7372635C73746D33326632B4
:1018300078375F6574682E630000000000900240F6
:1018400070B504460D461048204008B904B104E0C4
:1018500040F243710DA007F07DFA0DB1012D00D1CA
:1018600004E040F2447109A007F074FA2DB1104869
:10187000C06920430E49C86104E00D48C069A04317
:101880000B49C86170BD00000018FEFF2E2E5C4C95
:1018900069627261726965735C7372635C73746DA3
:1018A0003332663278375F6574682E63000000005B
:1018B0000090024010B504460CB1012C00D104E0A8
:1018C0004FF4FF6108A007F045FA34B10F48806972
:1018D00040F002000D49886105E00C48806920F065
:1018E00002000A49886110BD2E2E5C4C696272614B
:1018F000726965735C7372635C73746D33326632E4
:1019000078375F6574682E63000000000090024025
:1019100070B50C4613460021124D286000BF18E038
:1019200000EB01124FF00045156044F2F45555608C
:10193000C1EBC11505EB450504EB850595605D1E02
:101940008D4204D900EB01151035D56000E0D06060
:10195000491C9942E4D3044DE860044D044E3560BF
:1019600070BD0000500000200090024030C90020EF
:101970005400002070B504460D460DB1012D00D174
:1019800004E040F2666107A007F0E4F925B1606861
:1019900020F00040606003E0606840F0004060605C
:1019A00070BD00002E2E5C4C6962726172696573B5
:1019B0005C7372635C73746D3332663278375F6563
:1019C00074682E630000000010B504460CB1012CB1
:1019D00000D104E040F2E17108A007F0BBF934B196
:1019E0000F48806940F400500D49886105E00C48BB
:1019F000806920F400500A49886110BD2E2E5C4C8D
:101A000069627261726965735C7372635C73746D31
:101A10003332663278375F6574682E6300000000E9
:101A20000090024030B50C46134600210F4D28604F
:101A300000BF15E000EB01124FF480151560C1EBFB
:101A4000C11505EB450504EB850595605D1E8D42CE
:101A500004D900EB01151035D56000E0D060491CB9
:101A60009942E7D3024D286130BD00004C000020B0
:101A70000090024070B505460C4644B1B4F5800FA5
:101A800005D0B4F5000F02D0B4F5400F00D104E04A
:101A900040F2975103A007F05DF9286820432860C1
:101AA00070BD00002E2E5C4C6962726172696573B4
:101AB0005C7372635C73746D3332663278375F6562
:101AC00074682E630000000010B50121480605F07F
:101AD0002FF800214FF0007005F02AF810BD01B575
:101AE00081B0002000900198009002E00098401E14
:101AF000009000980028F9D10CBD000003488069CF
:101B000040F4801001498861704700000090024055
:101B10001CB50121572004F0D1FF0121880305F0F5
:101B2000B3F8002005F046FB03208DF805000220E5
:101B30008DF8040000208DF806008DF807008F2036
:101B400000906946364801F095FF0B220021344889
:101B500002F060F80B220121314802F05BF80B2201
:101B600002212F4802F056F80B2203212C4802F0E4
:101B700051F80B2207212A4802F04CF840F203509A
:101B800000906946274801F075FF0B220021254887
:101B900002F040F80B220121224802F03BF80B2210
:101BA0000821204802F036F80B220A211D4802F0D5
:101BB00031F83E20009069461B4801F05BFF0B2284
:101BC0000121194802F026F80B220221164802F0E2
:101BD00021F80B220321144802F01CF80B220421E7
:101BE000114802F017F80B2205210F4802F012F8F5
:101BF0004FF4D040009069460C4801F03BFF0B22A7
:101C000011460A4802F006F80B220D21074802F09F
:101C100001F80B220E21054801F0FCFF1CBD00005D
:101C20000000024000040240000802400018024088
:101C300070B504460025B4F1005F2AD0B4F1805F8E
:101C400027D0B4F1006F24D0B4F5803F21D0B4F593
:101C5000004F1ED0B4F5804F1BD0B4F5005F18D0F4
:101C6000B4F5806F15D0B4F5007F12D0B4F5807F45
:101C70000FD0802C0DD0402C0BD0202C09D0102C54
:101C800007D0082C05D0042C03D0022C01D0012C45
:101C900000D104E040F2FE6105A007F05BF80D48BA
:101CA0004069204008B1012500E00025284670BDAC
:101CB0002E2E5C4C69627261726965735C7372632B
:101CC0005C73746D3332663278375F6574682E6387
:101CD000000000000090024000200449096801F063
:101CE000010109B1012000E000207047009002408E
:101CF0000FB5002101910291039100916FE00099CD
:101D0000491C00913D490968096801F40071A1B1BD
:101D10003A490968096801F4807171B9374909685D
:101D2000374A126811600121354A126891603349BF
:101D30000968C968314A116051E030490968096889
:101D400001F4807191B92D490968096801F40071A5
:101D500061B92B4909688968491C294A1268916050
:101D600026490968C968254A116038E0234909688D
:101D7000234A12685160224909688968491C204A2F
:101D8000126891601E4909688968012904D11B49BC
:101D900009681B4A12681160184909680968C1F38B
:101DA0000D41091F0191164909688968012905D962
:101DB0001349096809688968029103E00F490968B5
:101DC000896802910D49096803910C490968C9683D
:101DD0000A4A116001A90EC980E80E000FBD07492B
:101DE0000968096801F0004111B90099082986D3F2
:101DF00001A90EC980E80E0000BFEFE750000020E7
:101E00005400002010B54020FFF712FF012803D135
:101E10000548006803F080FE4020FFF7EBFC4FF41C
:101E20008030FFF7E7FC10BDA00100202DE9F04154
:101E300086B004460F464FF00008002500200590AC
:101E4000F84E00902068012801D0206800B904E015
:101E50004FF48C71F4A006F07DFF606818B16068E3
:101E6000B0F5000F00D104E040F21911EEA006F029
:101E700071FFA06818B1A068B0F5800F00D104E030
:101E80004FF48D71E8A006F065FFE068D8B1E06816
:101E9000B0F5003F17D0E068B0F5802F13D0E068B0
:101EA000B0F5C02F0FD0E068B0F5002F0BD0E06880
:101EB000B0F5202F07D0E068B0F5402F03D0E068E0
:101EC000B0F5602F00D104E040F21B11D6A006F05F
:101ED00041FF206918B12069B0F5803F00D104E0CE
:101EE0004FF48E71D0A006F035FF606918B16069BB
:101EF000B0F5804F00D104E040F21D11CAA006F0F9
:101F000029FFA06918B1A069B0F5005F00D104E015
:101F10004FF48F71C4A006F01DFFE069B0F5805F3B
:101F200001D0E06900B904E040F21F11BEA006F044
:101F300011FF206AB0F5006F01D0206A00B904E0FB
:101F40004FF49071B8A006F005FF606AB0F5806F9D
:101F500001D0606A00B904E040F22111B2A006F09D
:101F6000F9FEA06A18B1A06AB0F5007F00D104E0C4
:101F70004FF49171ACA006F0EDFEE06A802801D02C
:101F8000E06A00B904E040F22311A7A006F0E2FEE7
:101F9000206B40B1206B202805D0206B402802D058
:101FA000206B602800D104E04FF492719EA006F0EF
:101FB000D1FE606B102801D0606B00B904E040F2E4
:101FC000251199A006F0C6FEA06BB0F1004F01D01C
:101FD000A06B00B904E04FF4937193A006F0BAFE31
:101FE000E06BB0F5007F05D0E06BB0F5407F01D02D
:101FF000E06B00B904E040F227118BA006F0AAFEC6
:10200000206C402805D0206C802802D0206CC0288D
:1020100000D104E04FF4947183A006F09BFE606C45
:1020200010B1606C202800D104E040F229117EA09C
:1020300006F090FEA06C10B1A06C082800D104E05E
:102040004FF4957178A006F085FE40F20441206DB2
:10205000884207D0206D042804D0206D10B1206D77
:10206000102800D104E04FF496716FA006F072FEC4
:1020700040F20241606D884204D0606D022801D0B8
:10208000606D00B904E040F22D1167A006F062FE19
:10209000206EB0F5803F00D204E04FF4977162A04B
:1020A00006F058FE606E10B1606E802800D104E02A
:1020B00040F22F115CA006F04DFEA06E40B1A06E64
:1020C000102805D0A06E202802D0A06E302800D1A4
:1020D00004E04FF4987154A006F03CFEE06E08282E
:1020E00001D0E06E00B904E040F231114EA006F0DC
:1020F00031FE206F042801D0206F00B904E04FF4B6
:10210000997149A006F026FE606F022801D0606F29
:1021100000B904E040F2331143A006F01BFEA06FAB
:10212000B0F5803F01D0A06F00B904E04FF49A7180
:102130003DA006F00FFEE06FB0F5803F00D204E056
:1021400040F2351138A006F005FED4F8800020B129
:10215000D4F88000B0F1806F00D104E040F2371174
:1021600031A006F0F7FDD4F88400B0F1007F02D072
:10217000D4F8840000B904E04FF49C712AA006F062
:10218000E9FDD4F8880020B1D4F88800B0F1807F50
:1021900000D104E040F2391123A006F0DBFDD4F8B1
:1021A0008C00B0F5001F02D0D4F88C0000B904E018
:1021B0004FF49D711CA006F0CDFDD4F8900010B333
:1021C000D4F89000B0F5804F1DD0D4F89000B0F551
:1021D000004F18D0D4F89000B0F5404F13D0D4F889
:1021E0009000B0F5803F0ED0D4F89000B0F5A03F3D
:1021F00009D0D4F89000B0F5C03F04D0D4F89000D6
:10220000B0F5E03F00D104E040F23B1106A006F03B
:10221000A1FDD4F89400802802D0D4F89400A8B985
:102220001AE00000008793032E2E5C4C69627261F5
:10223000726965735C7372635C73746D333266329A
:1022400078375F6574682E63000000004FF49E715C
:10225000AFF22C0006F07EFDD4F89800402802D0A2
:10226000D4F8980000B905E040F23D11AFF2480003
:1022700006F070FDD4F89C0058B1D4F89C000828F2
:1022800007D0D4F89C00102803D0D4F89C0018285C
:1022900000D105E04FF49F71AFF2740006F05AFDD3
:1022A000D4F8A000042802D0D4F8A00000B905E0BA
:1022B00040F23F11AFF2900006F04CFDD4F8A400BC
:1022C000B0F1007F02D0D4F8A40000B905E04FF4CB
:1022D000A071AFF2AC0006F03DFDD4F8A800B0F557
:1022E000803F02D0D4F8A80000B905E040F24111C7
:1022F000AFF2CC0006F02EFDD4F8AC00B0F5003FF4
:1023000036D0D4F8AC00B0F5802F31D0D4F8AC0082
:10231000B0F5002F2CD0D4F8AC00B0F5801F27D03A
:10232000D4F8AC00B0F5001F22D0D4F8AC00B0F562
:10233000800F1DD0D4F8AC00B0F1817F18D0D4F854
:10234000AC00B0F1827F13D0D4F8AC00B0F1847F40
:102350000ED0D4F8AC00B0F1887F09D0D4F8AC002E
:10236000B0F1907F04D0D4F8AC00B0F1A07F00D1E0
:1023700005E04FF4A171AFF2501006F0EBFCD4F879
:10238000B000B0F5807F36D0D4F8B000B0F5007F53
:1023900031D0D4F8B000B0F5806F2CD0D4F8B000B4
:1023A000B0F5006F27D0D4F8B000B0F5805F22D030
:1023B000D4F8B000B0F5005F1DD0D4F8B000B0F193
:1023C000012F18D0B149D4F8B000884213D0B049D9
:1023D000D4F8B00088420ED0AE49D4F8B00088429C
:1023E00009D0AD49D4F8B000884204D0AB49D4F844
:1023F000B000884200D105E040F24311AFF2D8109E
:1024000006F0A8FCD4F8B4001F2800D805E04FF46B
:10241000A271AFF2EC1006F09DFCD4F8B80090B1B8
:10242000D4F8B800B0F5804F0DD0D4F8B800B0F5AE
:10243000004F08D0D4F8B800B0F5404F03D0D4F81E
:10244000B800022800D105E040F24511AFF2282083
:1024500006F080FC9248056925F01C0501A804F0EF
:102460004DFC029E8F48864205D38F48864202D299
:1024700045F0080511E08C48864205D38B4886421A
:1024800002D245F00C0508E08848864203D388480C
:10249000864200D201E045F00405814805614FF411
:1024A00000420021384600F08DFB18B9002006B02C
:1024B000BDE8F0817F48FFF712FB2068A0B300BFA2
:1024C0000098401C00900121384600F09DFA00F071
:1024D000040018B9784900988842F1D376490098E9
:1024E000884201D10020E2E7002000904FF48052A2
:1024F0000021384600F066FB08B90020D7E700BF8E
:102500000098401C00900121384600F07DFA00F050
:10251000200018B9684900988842F1D366490098AC
:10252000884202D10020C2E719E00020009010216B
:10253000384600F069FA804608F0040018B14FF4FC
:102540000060206201E00020206208F0020010B16B
:102550000020606116E04FF48040606112E0206A64
:10256000C0F3CF006169C1F34F0140EA01020021CD
:10257000384600F027FB08B9002098E76FF07F404D
:10258000FFF7ADFA464805684C480540D4E901011B
:102590000843E16808432169084361690843A16968
:1025A0000843E1690843216A0843616A0843A16A54
:1025B0000843E16A0843216B0843616B0843054304
:1025C00037480560D4E90E010843216C0843616C6B
:1025D0000843A16C0843E16C0843216D0843616D19
:1025E00008432F494860A06D8860E06DC8600846C8
:1025F00085694FF641700540B4F86010606E40EA9E
:102600000140A16E0843E16E0843216F0843616FEA
:102610000843054322488561D4E91E010843204947
:10262000C8612748856927480540D4E92001084347
:10263000D4F888100843D4F88C100843D4F89010CC
:102640000843D4F894100843D4F898100843D4F8F9
:102650009C100843D4F8A01008430543184885612E
:10266000D4E929010843D4F8AC100843D4F8B010D9
:102670000843D4F8B41040EA8100D4F8B8100843F5
:1026800040F400000E490860012010E7000200013C
:1026900000040001000800010010000100200001FA
:1026A00000800240002D3101C00E16020087930306
:1026B00000E1F505FFFF0F00FFFF04000F8120FF81
:1026C00000900240233FDEF870B504460D462CB161
:1026D000082C03D0102C01D0182C00D104E04FF4AA
:1026E0004F710CA006F036FB2879697940EA012683
:1026F000114820440664E8780006A97840EA0140C1
:10270000697840EA0120297840EA01060A48204415
:10271000466470BD2E2E5C4C69627261726965738D
:102720005C7372635C73746D3332663278375F65E5
:1027300074682E63000000000080024000B5AFB056
:1027400001214FF0606004F0B9F9FFF7BDF900F026
:10275000B5F900BFFFF7C0FA0128FBD0684600F0CA
:10276000D7F901200090002007904FF400700A90E4
:1027700000200B900E9011901390149015904FF430
:1027800080600990002020904FF00070219000118F
:10279000239000202590269004202890C0052990A1
:1027A00040122A9080012B9040122C9040002E90D5
:1027B00001216846FFF73AFB18B101200349086080
:1027C00002E00020014908602FB000BD6C0000202D
:1027D00010B504460CB1012C00D104E040F28D216B
:1027E00008A006F0B7FA34B10F48006840F00400C2
:1027F0000D49086005E00C48006820F004000A4913
:10280000086010BD2E2E5C4C69627261726965733E
:102810005C7372635C73746D3332663278375F65F4
:1028200074682E63000000000080024010B504466A
:102830000CB1012C00D104E040F2752108A006F093
:1028400089FA34B10F48006840F008000D4908606B
:1028500005E00C48006820F008000A49086010BD37
:102860002E2E5C4C69627261726965735C7372636F
:102870005C73746D3332663278375F6574682E63CB
:10288000000000000080024008B53D208DF80000E7
:1028900002208DF8010000208DF8020001208DF843
:1028A0000300684602F0FCFB4020FEF7A3FF4FF454
:1028B0008030FEF79FFF01210148FEF7C1FF08BDF0
:1028C000400001001CB50121102004F0F7F804209D
:1028D000009002208DF8050001208DF804000020F2
:1028E0008DF806008DF8070069460C4801F0C2F823
:1028F00004210A4801F030FB0A2013F00FFC0421E8
:10290000064801F0D5FA0A2013F008FC0421034818
:1029100001F022FB0A2013F001FC1CBD0010024054
:1029200070B5024600230025002435480068006881
:1029300000F0004008B1002070BD3148016840F24D
:10294000F450824208DD92FBF0F392FBF0F600FBBC
:10295000162010B15B1C00E00123012B1AD128487E
:102960000068006840F04050254E36683060C2F381
:102970000C00234E3668706021480068006840F003
:1029800000401F4E366830601D480068C0681C4E0D
:10299000306028E0002422E03CB919480068006853
:1029A00040F08050164E3668306040F2F450486077
:1029B000581EA0420DD1086840F000500860581E13
:1029C000C0EBC01000EB4000A2EB8005C5F30C008B
:1029D0004860086840F000400860C968641C9C4278
:1029E000DAD3074801600748406900F0040020B1CD
:1029F0000420044E70610020706001209CE70000FC
:102A00004C00002000900240F8B506460D46002418
:102A100000200090202E00DC04E040F692011CA073
:102A200006F098F91DB1012D01D0102D00D104E060
:102A300040F6930116A006F08DF91E48046904F0D3
:102A40001C044FF4784000EAC62004434FF4F860B9
:102A500000EA8510044324F0020444F00104154800
:102A6000046100BF0098401C00901248046904F003
:102A7000010018B1104900988842F3D30E4900981C
:102A8000884201D10020F8BD0A48406980B2FAE7C7
:102A90002E2E5C4C69627261726965735C7372633D
:102AA0005C73746D3332663278375F6574682E6399
:102AB0000000000000800240FFFF0400034800689F
:102AC00040F001000149086070470000009002409A
:102AD00010B50120FFF7AAFEFFF710F80120FFF75D
:102AE00077FE0120FEF770FF0120FEF7E3FE10BD28
:102AF00010B50020FEF768FF0020FEF7DBFE002087
:102B0000FFF766FEFEF7FAFF0020FFF78FFE10BD0D
:102B100001210160002141608160C16001614FF4C9
:102B20008041416100218161C1614FF40061016216
:102B3000002141628162C162016341638163C163BB
:102B4000402101642021416400218164C164016548
:102B500041658165C165016680214166002181660C
:102B6000C166016741678167C1674FF08061C0F846
:102B700080104910C0F884100021C0F888104FF46C
:102B80000011C0F88C100021C0F89010C0F894100B
:102B9000C0F89810C0F89C10C0F8A0104FF0007159
:102BA000C0F8A4104912C0F8A8108901C0F8AC10F0
:102BB0004912C0F8B0100021C0F8B410C0F8B81025
:102BC00070470000F8B506460D4617460024002061
:102BD0000090202E00DC04E040F6C1011BA006F0AE
:102BE000B9F81DB1012D01D0102D00D104E040F63F
:102BF000C20116A006F0AEF81D48046904F01C04DA
:102C00004FF4784000EAC62004434FF4F86000EA2D
:102C10008510044344F0020444F001041448476161
:102C2000046100BF0098401C00901148046904F042
:102C3000010018B10F4900988842F3D30D4900985C
:102C4000884201D10020F8BD0120FCE72E2E5C4C0B
:102C500069627261726965735C7372635C73746DCF
:102C60003332663278375F6574682E630000000087
:102C700000800240FFFF040070B504460D46102C92
:102C800002D0B4F5807F00D104E04FF4E8711AA0BF
:102C900006F060F80DB1012D00D104E040F2D11131
:102CA00015A006F057F89DB1102C08D14FF0204028
:102CB000006E40F004004FF0204108661BE017480A
:102CC000006840F004004FF02041C1F8800012E09D
:102CD000102C08D14FF02040006E114908404FF0F1
:102CE0002041086607E00D4800680D4908404FF094
:102CF0002041C1F8800070BD2E2E5C4C696272616B
:102D0000726965735C7372635C73746D33326632BF
:102D100078785F66736D632E63000000800000A00A
:102D2000FBFF0F002DE9F041044600250026002797
:102D30002068102803D02068B0F5807F00D104E01F
:102D400040F2751170A006F005F8606810B1606877
:102D5000022800D104E04FF4BB716BA005F0FAFF2C
:102D6000A06810B1A068102800D104E040F27711EB
:102D700065A005F0EFFFE06810B1E068402800D1E1
:102D800004E04FF4BC7160A005F0E4FF206998B145
:102D90002069B0F5003F0FD02069B0F5802F0BD02F
:102DA0002069B0F5C02F07D02069B0F5002F03D0FF
:102DB0002069B0F5202F00D104E040F2791152A033
:102DC00005F0C8FF6069FF2800D804E04FF4BD712A
:102DD0004DA005F0BFFFA069FF2800D804E040F235
:102DE0007B1149A005F0B6FFE0690068FF2800D814
:102DF00004E04FF4BE7144A005F0ACFFE069406808
:102E0000FF2800D804E040F27D113FA005F0A2FFAA
:102E1000E0698068FF2800D804E04FF4BF713AA051
:102E200005F098FFE069C068FF2800D804E040F290
:102E30007F1135A005F08EFF206A0068FF2800D8BA
:102E400004E04FF4C07130A005F084FF206A4068B0
:102E5000FF2800D804E040F281112BA005F07AFF92
:102E6000206A8068FF2800D804E04FF4C17126A0D2
:102E700005F070FF206AC068FF2800D804E040F227
:102E8000831121A005F066FF606840F00800A1688A
:102E90000843E168084321690843616940EA412029
:102EA000A16940EA4135E0690068E169496840EAA2
:102EB0000120E169098940EA0140E169097B40EAB2
:102EC0000166206A0068216A496840EA0120216A97
:102ED000098940EA0140216A097B40EA01672068CC
:102EE000102805D14FF0204005668666C76608E0C9
:102EF0000E4805604FF02040C0F888600B480C3049
:102F00000760BDE8F08100002E2E5C4C69627261A2
:102F1000726965735C7372635C73746D33326632AD
:102F200078785F66736D632E63000000800000A0F8
:102F30002DE9F04107460D461646984600201649F1
:102F4000087016490E70301208700D70280A08704B
:102F5000280C0870302010490870002401E0601C23
:102F600084B2142CFBDB00BF40210D4800F020FF91
:102F70000028F9D000240AE0385D4FF0E0410978DC
:102F8000884202D00120BDE8F081601C84B2444533
:102F9000F2DB0020F7E70000000001700000027083
:102FA000000C024010B50446602007490870A401D7
:102FB00006490C70200A0870200C0870D0200249C5
:102FC000087000F005F810BD0000017000000270EC
:102FD00070B54FF48034402500F010FA054603E048
:102FE00000F00CFA0546641E402D01D0002CF7D1EC
:102FF00004B98025284670BD00B58FB00121084670
:1030000003F0D0FD0121182003F058FD0C2200210F
:103010003F4800F0FFFD0C2201213D4800F0FAFD81
:103020000C2204213A4800F0F5FD0C220521384815
:1030300000F0F0FD0C220621354800F0EBFD0C22DB
:103040000721334800F0E6FD0C220B21304800F048
:10305000E1FD0C2211462E4800F0DCFD0C22072178
:103060002C4800F0D7FD0C2208212A4800F0D2FDA0
:103070000C220921274800F0CDFD0C220A21254809
:1030800000F0C8FD4DF6B3000D9002208DF8390018
:103090008DF8380000208DF83A008DF83B000DA91E
:1030A0001B4800F0E7FC4FF4F0600D900DA91948A3
:1030B00000F0E0FC40200D9002208DF83900002047
:1030C0008DF8380001208DF83B000DA9104800F064
:1030D000D1FC01200090022001900290039010206A
:1030E000049000200590069040200790000308906F
:1030F000002009900A90CDF82CD0CDF830D004A84B
:10310000FFF710FE01211020FFF7B6FD0FB000BD44
:10311000000C02400010024070B504460D4604F059
:10312000400005F04001884206D02A4621461EA0F4
:1031300004F054FE012070BD002028490870284981
:10314000087008700C70200A0870200C0870352078
:1031500022490870002601E0701CC6B2142EFBDB69
:1031600000BF40211F4800F023FE0028F9D0852031
:103170001A49087000201A49087008700D70280A52
:103180000870280C0870102014490870FFF720FF01
:10319000402801D10020CEE72A46214612A004F0A3
:1031A0001DFE0120C7E700004572726F72203A20B1
:1031B00046534D435F4E414E445F50616765436FD8
:1031C00070794261636B4578287372633D25642C86
:1031D000207461723D256429200D0A0000000170F1
:1031E00000000270000C02404572726F723A204675
:1031F000534D435F4E414E445F50616765436F706E
:10320000794261636B2825642C202564290D0A000E
:103210002DE9F84304460D4690461F46DDF8209000
:1032200004F0400005F04001884207D02A462146BC
:10323000284804F0D3FD0120BDE8F883002026498A
:1032400008702649087008700C70200A0870200C5D
:103250000870352020490870002601E0701C86B2F5
:10326000142EFBDB00BF40211D4800F0A1FD00280B
:10327000F9D0852018490870002018490870087096
:103280000D70280A0870280C0870852012490870F3
:1032900012490F7038120870002606E018F8060070
:1032A0004FF0E0410870701C86B24E45F6DB1020EE
:1032B00009490870FFF78CFE402801D10020BBE7C8
:1032C0003B462A4621460748CDF8009004F086FD8B
:1032D0000120B1E7F45604080000017000000270FC
:1032E000000C02407C5704082DE9F04105460E46CB
:1032F00017461C46B4F5006F06DD214606A004F013
:103300006DFD0120BDE8F08123463A46314628464E
:1033100000F014F8F6E700004572726F723A20462A
:10332000534D435F4E414E445F5265616444617446
:103330006128292025640D0A000000002DE9F041D4
:1033400007460D4616469846002014490870144951
:103350000E70301208700D70280A0870280C087062
:1033600030200E490870002401E0601C84B2322C29
:10337000FBDB00BF40210B4800F01AFD0028F9D00C
:10338000002405E04FF0E04000783855601C84B21E
:103390004445F7DB0020BDE8F0810000000001702B
:1033A00000000270000C02402DE9F04106460F4675
:1033B00015461C46402C06DD214607A004F00EFDF4
:1033C0000120BDE8F08105F5006082B22346394650
:1033D0003046FFF7B3FFF4E74572726F723A20464A
:1033E000534D435F4E414E445F526561645370617B
:1033F000726528292025640D0A0000000020702233
:10340000084B1A701206117801F001020AB101206E
:1034100006E001F04002402A01D1402000E00020F7
:10342000704700000000017010B5FF2004490870CB
:10343000FFF7CEFD402801D1002010BD0120FCE7A0
:10344000000001702DE9F04105460E4617461C4666
:10345000B4F5006F06DD214606A004F0BFFC012094
:10346000BDE8F08123463A463146284600F014F87C
:10347000F6E700004572726F723A2046534D435F83
:103480004E414E445F5772697465446174612829E6
:103490002025640D0A0000002DE9F04106460D4686
:1034A0001746984680202749087027490F70381220
:1034B00008700D70280A0870280C0870002401E0BC
:1034C000601C84B2142CFBDB002405E0305D4FF05F
:1034D000E0410870601C84B24445F7DB10201949B4
:1034E0000870002401E0601C84B2142CFBDB00BFD8
:1034F0004021164800F05CFC0028F9D0FFF768FD79
:10350000402816D143463A4629461148FFF716FF90
:10351000424631460E48FCF731FF40B143463A4639
:1035200029460CA004F05AFC0120BDE8F0810020DF
:10353000FBE743463A46294615A004F04FFC01201C
:10354000F3E700000000017000000270000C024070
:103550003CD100204572726F72313A2046534D4380
:103560005F4E414E445F57726974655061676528CC
:10357000706167653D25642C20616464723D25643B
:103580002C20636F756E743D2564290D0A000000C0
:103590004572726F72323A2046534D435F4E414E30
:1035A000445F57726974655061676528706167652B
:1035B0003D25642C20616464723D25642C20636F7A
:1035C000756E743D2564290D0A0000002DE9F04157
:1035D00006460F4615461C46402C06DD214607A030
:1035E00004F0FCFB0120BDE8F08105F5006082B22B
:1035F000234639463046FFF74FFFF4E74572726FB6
:10360000723A2046534D435F4E414E445F577269B4
:103610007465537061726528292025640D0A0000C5
:1036200070B504460D462CB1022C03D0042C01D0F9
:10363000062C00D104E04FF4867111A005F08AFB3E
:103640000DB1012D00D104E040F20D110CA005F0E8
:1036500081FB55B1A000A0F1C040006840F001011D
:10366000A000A0F1C040016009E0A000A0F1C040AE
:1036700000680C490840A100A1F1C041086070BD7C
:103680002E2E5C4C69627261726965735C73726341
:103690005C73746D3332663278785F66736D632E57
:1036A00063000000FEFF0F0010B50446206840B123
:1036B0002068022805D02068042802D02068062847
:1036C00000D103E09021C8A005F044FB606810B170
:1036D0006068022800D103E09121C3A005F03AFB05
:1036E000A06828B1A068042802D0A068082800D1EA
:1036F00003E09221BCA005F02DFBE06810B1E0686A
:10370000102800D103E09321B7A005F023FB206926
:1037100018B12069B0F5807F00D103E09421B2A0F8
:1037200005F018FB606918B16069B0F5004F00D171
:1037300003E09521ACA005F00DFBA06918B1A069CC
:10374000B0F5007F00D103E09621A7A005F002FBB1
:10375000E06918B1E069B0F5806F00D103E097210E
:10376000A1A005F0F7FA206A18B1206AB0F5006F41
:1037700000D103E098219CA005F0ECFA606A18B132
:10378000606AB0F5805F00D103E0992196A005F052
:10379000E1FAA06A18B1A06AB0F5005F00D103E0B9
:1037A0009A2191A005F0D6FAE06A18B1E06AB0F566
:1037B000804F00D103E09B218BA005F0CBFA206B5A
:1037C00018B1206BB0F5002F00D103E09C2186A03A
:1037D00005F0C0FA606B00680F2800D803E09D2157
:1037E00081A005F0B7FA606B40680F2800D803E0AD
:1037F0009E217DA005F0AEFA606B806820B1606B01
:103800008068FF2800D803E09F2177A005F0A2FA86
:10381000606BC0680F2800D803E0A02172A005F0FB
:1038200099FA606B00690F2800D803E0A1216EA00F
:1038300005F090FA606B40690F2800D803E0A221E0
:1038400069A005F087FA606B806970B1606B806970
:10385000B0F1805F09D0606B8069B0F1005F04D087
:10386000606B8069B0F1405F00D103E0A3215EA0EE
:1038700005F070FAD4E901010843E16808432169C1
:10388000084361690843A1690843E1690843216A63
:103890000843616A0843A16A0843E16A0843216B4F
:1038A000084321688900A1F1C0410860A068082888
:1038B0000BD120688000A0F1C040006840F04001BA
:1038C00020688000A0F1C0400160606B0068616BFF
:1038D000496840EA0110616B896840EA0120616B28
:1038E000898940EA0140616B098A40EA0150616BB5
:1038F000097D40EA0160616B896908432168491CC0
:103900008900A1F1C0410860E06AB0F5804F62D142
:10391000A06B00680F2800D803E0C52132A005F095
:1039200019FAA06B40680F2800D803E0C6212EA02A
:1039300005F010FAA06B806820B1A06B8068FF28AA
:1039400000D803E0C72128A005F004FAA06B0069A5
:103950000F2800D803E0C82123A005F0FBF9A06BD5
:1039600040690F2800D803E0C9211FA005F0F2F933
:10397000A06B806970B1A06B8069B0F1805F09D0E5
:10398000A06B8069B0F1005F04D0A06B8069B0F1DA
:10399000405F00D103E0CA2113A005F0DBF9A06B62
:1039A0000068A16B496840EA0110A16B896840EA90
:1039B0000120A16B098A40EA0150A16B097D40EA10
:1039C0000160A16B8969084321688900A1F1C041A8
:1039D000C1F8040107E06FF0704120688000A0F199
:1039E000C040C0F8041110BD2E2E5C4C696272619B
:1039F000726965735C7372635C73746D33326632C3
:103A000078785F66736D632E6300000000B597B031
:103A100003F0E8F90121084603F0C4F80020019002
:103A2000029002200390002004900F200590069041
:103A30000020079004200890002009900A90102090
:103A40000B9000200C900D900E900F9010904FF462
:103A500080501190002012901390149001A815909E
:103A6000169008A8FFF720FE01210420FFF7D8FDDB
:103A700017B000BD2DE9F04104460D460026002791
:103A8000B0465248844217D05148844214D051481D
:103A9000844211D0504884420ED0504884420BD00A
:103AA0004F48844208D04F48844205D04E48844253
:103AB00002D04E48844200D103E0BA214CA005F068
:103AC00049F9002010B9286800B103E0BB2148A0E3
:103AD00005F040F9287940B12879012805D02879E6
:103AE000022802D02879032800D103E0BC2140A09D
:103AF00005F030F9E87928B1E879012802D0E879B1
:103B0000022800D103E0BD2139A005F023F90026E9
:103B100057E0012000FA06F7286800EA0708B845D0
:103B20004ED120687200032191408843206028799B
:103B3000710088402168084320602879012802D05C
:103B40002879022830D1687940B16879012805D0F8
:103B50006879022802D06879032800D103E0CF21D8
:103B600023A005F0F7F8A068720003219140884374
:103B7000A060687971008840A1680843A060A879B6
:103B800010B1A879012800D103E0D62118A005F0D2
:103B9000E1F861680120B040814361606068A97903
:103BA000B14089B208436060E0687200032191402F
:103BB0008843E060E87971008840E1680843E0608C
:103BC000761C102EA5D3BDE8F08100000000024055
:103BD0000004024000080240000C024000100240B5
:103BE0000014024000180240001C02400020024065
:103BF0002E2E5C4C69627261726965735C737263CC
:103C00005C73746D3332663278785F6770696F2EDB
:103C1000630000002DE9F04106460D4614460027DA
:103C2000B8465148864217D05048864214D0504872
:103C3000864211D04F4886420ED04F4886420BD064
:103C40004E48864208D04E48864205D04D488642AE
:103C500002D04D48864200D104E040F215214BA02D
:103C600005F078F8EDB1012D1BD0022D19D0032DF0
:103C700017D0042D15D0052D13D0062D11D0072DEA
:103C80000FD0082D0DD0092D0BD00A2D09D00B2DEA
:103C900007D00C2D05D00D2D03D00E2D01D00F2DEA
:103CA00000D104E040F2162138A005F053F89CB38F
:103CB000092C31D084B37CB374B36CB3012C2BD0FA
:103CC0002AD0022C28D027D026D0032C24D0042C94
:103CD00022D021D020D0052C1ED01DD0092C1BD0E5
:103CE000062C19D0092C17D0072C15D014D013D0BE
:103CF000082C11D010D00FD0092C0DD00CD00A2CCC
:103D00000AD009D00B2C07D00C2C05D004D003D03E
:103D10000D2C01D00F2C00D104E040F217211BA084
:103D200005F018F86807C00E04FA00F7E91006F16C
:103D3000200050F821006907CA0E0F2191408843E6
:103D4000EA1006F1200141F82200E91006F12000F6
:103D500050F8210040EA0708E91006F1200040F879
:103D60002180BDE8F0810000000002400004024014
:103D700000080240000C0240001002400014024003
:103D800000180240001C0240002002402E2E5C4C15
:103D900069627261726965735C7372635C73746D7E
:103DA0003332663278785F6770696F2E6300000087
:103DB00070B505460C4600262B48854217D02B4887
:103DC000854214D02A48854211D02A4885420ED017
:103DD000294885420BD02948854208D02848854289
:103DE00005D02848854202D02748854200D104E00A
:103DF00040F22F1125A004F0ADFF012C25D0022C9C
:103E000023D0042C21D0082C1FD0102C1DD0202C06
:103E10001BD0402C19D0802C17D0B4F5807F14D043
:103E2000B4F5007F11D0B4F5806F0ED0B4F5006FFB
:103E30000BD0B4F5805F08D0B4F5005F05D0B4F5C1
:103E4000804F02D0B4F5004F00D104E04FF49871D8
:103E50000EA004F07FFF2869204008B1012600E091
:103E60000026304670BD0000000002400004024001
:103E700000080240000C0240001002400014024002
:103E800000180240001C0240002002402E2E5C4C14
:103E900069627261726965735C7372635C73746D7D
:103EA0003332663278785F6770696F2E6300000086
:103EB00070B504460D461648844217D01548844212
:103EC00014D01548844211D0144884420ED01448AE
:103ED00084420BD01348844208D01348844205D052
:103EE0001248844202D01248844200D104E040F2D9
:103EF000911110A004F02EFF002008B905B104E0D4
:103F00004FF4C9710BA004F025FF2804A06170BD17
:103F1000000002400004024000080240000C024081
:103F2000001002400014024000180240001C024031
:103F3000002002402E2E5C4C6962726172696573CA
:103F40005C7372635C73746D3332663278785F676A
:103F500070696F2E6300000070B504460D46164868
:103F6000844217D01548844214D01548844211D099
:103F7000144884420ED0144884420BD01348844223
:103F800008D01348844205D01248844202D0124817
:103F9000844200D104E04FF4BF7110A004F0DAFEB7
:103FA000002008B905B104E040F27F110BA004F035
:103FB000D1FEA56170BD0000000002400004024077
:103FC00000080240000C02400010024000140240B1
:103FD00000180240001C0240002002402E2E5C4CC3
:103FE00069627261726965735C7372635C73746D2C
:103FF0003332663278785F6770696F2E6300000035
:1040000070B505460C4616462E48854217D02E48F8
:10401000854214D02D48854211D02D4885420ED0BE
:104020002C4885420BD02C48854208D02B4885422D
:1040300005D02B48854202D02A48854200D104E0B1
:1040400040F2A51128A004F085FE012C25D0022CF9
:1040500023D0042C21D0082C1FD0102C1DD0202CB4
:104060001BD0402C19D0802C17D0B4F5807F14D0F1
:10407000B4F5007F11D0B4F5806F0ED0B4F5006FA9
:104080000BD0B4F5805F08D0B4F5005F05D0B4F56F
:10409000804F02D0B4F5004F00D104E04FF4D3714B
:1040A00011A004F057FE0EB1012E00D104E040F241
:1040B000A7110DA004F04EFE0EB1AC6101E020048A
:1040C000A86170BD000002400004024000080240E8
:1040D000000C024000100240001402400018024090
:1040E000001C0240002002402E2E5C4C696272616E
:1040F000726965735C7372635C73746D33326632BC
:1041000078785F6770696F2E6300000000BFFEE77C
:104110002DE9FE4F04460D4616461F46DDF830A039
:104120000020029001978046814601A811F07AFA9A
:104130008DF808000298C0F3C00028700298C0F300
:10414000031020706946019800F034F98146019906
:1041500008440190DDE9001000EB01080198A8EB8C
:104160000000022800DA06E001A811F062FA3080AF
:104170004FF0010900BF4846BDE8FE8F2DE9FF471B
:1041800004460D46164699460020039002960027E5
:104190008046009002A811F045FA8DF80C000398B3
:1041A000C0F30310022800D01FE001A9029800F01C
:1041B00001F98046029908440290DDE90110471890
:1041C0000298381A022800DA0FE002A811F02AFA41
:1041D0008DF80000009800F00100207002A811F096
:1041E00021FA28704FF0010800BF404604B0BDE836
:1041F000F0872DE9FF5F06460C4617469846DDE935
:104200000FABDDF838900020039011980290002544
:1042100000200190009002A811F004FA8DF80C0023
:104220000398C0F30310032800D032E00398C0F3D2
:10423000C00030700398C0F341002060039800F084
:10424000010038706946029800F0B4F801900299B4
:10425000084402900099029845182A4602A9484647
:1042600011F0F4F910B10298281A00D511E0206875
:10427000002804DD02A811F0DCF9A8F8000002987B
:10428000281ACBF800000298CAF80000012001901B
:1042900000BF019804B0BDE8F09F2DE9FE4F054630
:1042A0000E4614461F46DDE90C9B00200290CDF817
:1042B00004908046824601A811F0B4F98DF80800F8
:1042C0000298C0F30310092800D02CE06946019839
:1042D00000F070F88246019908440190DDE9001071
:1042E00000EB01080198A8EB0000022800DA1AE0B0
:1042F00001A811F09EF92880002020600DE02068C0
:10430000B04202DD4FF0FF3A0DE001A811F08AF94A
:104310002268511C216047F8220001984045EED3E5
:104320004FF0010A00BF5046BDE8FE8FFEB50446BF
:104330000D46164600200290019000272B4622468B
:1043400001A902A80096FFF7E3FE07469DF80800C2
:104350000B2800D101273846FEBD2DE9F84305465C
:104360000C46012600270020206000BF4FF0FF38D8
:10437000781C0746042801DD00BF17E001216846CC
:10438000A8478046B8F1010F00D00FE09DF800105B
:1043900001F07F01206801FB06002060F6019DF816
:1043A000000000F080000028E0D100BF3846BDE8E2
:1043B000F883000070B504460D46034804602946A2
:1043C0000248FFF7CAFF70BDB0010020598D0008F8
:1043D00030B50246002300BF0846CD1701EB5565F6
:1043E000ED11A1EBC515ECB2CD1701EB5565E91147
:1043F000002901DD44F0800418465B1C1454002998
:10440000EADC184630BD0000401C802801DA401C60
:104410000AE0B0F5804F01DA801C05E003498842CC
:1044200001DAC01C00E0001D70470000FFFF1F0004
:104430002DE9FC4104460F4615464FF0FF38002099
:1044400001900026009001212046A847012800D0B5
:104450001EE0012669462846FFF77FFF601C009991
:10446000FFF7B6FF064400983044B84200DD0FE085
:10447000009830B1A0190099A8470099884200D04F
:1044800006E020788DF804000198C0F3031800BFFF
:104490004046BDE8FC812DE9FC4704460E46154622
:1044A0001F46DDF828800020019081460094042EEC
:1044B00002DA6FF0010924E0019865F3071001901A
:1044C000019867F3C3000190062D01D1012100E09E
:1044D0000021019861F3420001909DF804106846A4
:1044E00016F051F802210098FFF772FF0099084476
:1044F00000904146684616F04CF80098A0EB04097D
:1045000000BF4846BDE8FC872DE9FE4305460E4640
:104510001446029500200190009000274FF0FF38CC
:10452000204600F0A5F807468146FFF76DFFB04230
:1045300002DD6FF001088FE000208DF80400019883
:1045400020F0F000103001909DF8041002A816F041
:104550001AF839460298FFF73BFF02990844029087
:10456000207A042808D13EA102A815F0F8FF042102
:1045700002A816F008F807E03BA102A815F0EFFF2B
:10458000032102A815F0FFFF00208DF80000A17E96
:10459000009861F341000090E07E08B1012100E045
:1045A0000021009861F3820000900098C0F3800021
:1045B00058B194F83D10009861F3C400009094F84D
:1045C0003C10009861F345100090206C08B9A06C75
:1045D00020B1009820F0800080300090E06C08B995
:1045E000606D20B1009820F04000403000909DF8B0
:1045F000001002A815F0C7FF218B02A815F0C9FF13
:1046000002A8D4E90423E16815F0DBFFE07E58B18D
:1046100002A8D4E90A23616A15F0D3FF02A8D4E9FD
:104620000D23216B15F0CDFF0098C0F3C01028B109
:1046300002A8D4E91123216C15F0C3FF0098C0F340
:10464000801028B102A8D4E91423E16C15F0B9FF59
:104650000298A0EB050800BF4046BDE8FE830000BD
:104660004D515454000000004D51497364700000D6
:1046700070B504460025207A032801D10C2503E0FB
:10468000207A042800D10A25D4E90412E06800F059
:1046900063F9801C0544E07E68B1D4E90A12606ABF
:1046A00000F05AF9861CD4E90D12206B00F054F981
:1046B0003044801C0544206C08B9A06C30B1D4E9AA
:1046C0001112206C00F048F9801C0544E06C08B918
:1046D000606D30B1D4E91412E06C00F03DF9801C3B
:1046E0000544284670BD70B504460D460C22294687
:1046F000204600F00BF970BDF8B505460E4614468D
:1047000000230422314628460094FFF7C4FEF8BD7A
:10471000F8B505460E4614460023072231462846C2
:104720000094FFF7B8FEF8BD2DE9F04F87B00546BD
:104730000F4690461C46DDE915B6DDE9109A069550
:1047400000200590049003900096204612A90EC9FF
:1047500000F042F804900290FFF756FEB84203DDE5
:104760006FF00100039033E0059820F0F000303046
:104770000590059868F3C3000590059864F342001E
:104780000590059869F3000005909DF8141006A89F
:1047900015F0F9FE04990698FFF71AFE06990844E9
:1047A000069006A812A90EC915F00BFF002C03DD18
:1047B000514606A815F0EDFE324659460698FBF71D
:1047C00086FD0698304406900698401B039000BF73
:1047D000039807B0BDE8F08F7FB50546089E00241A
:1047E00001A807C800F0B8F8801C30440444002D2C
:1047F00000DDA41C204604B070BDF8B506460F4687
:1048000014461D4623460522394630460095FFF7DB
:1048100042FEF8BDF8B506460F4614461D4623462F
:104820000622394630460095FFF735FEF8BD2DE9E2
:10483000FF5F05460E4617469846DDE90E9A03953A
:10484000002002900190009000245146484600F05C
:1048500046F883460190FFF7D7FDB04202DDA01E67
:10486000009038E000208DF80800029820F0F00059
:1048700080300290029867F3C3000290029820F003
:104880000600801C02909DF8081003A815F07BFE1E
:1048900001990398FFF79CFD039908440390414652
:1048A00003A815F076FE00240FE004EB44000AEBA9
:1048B000800C03A89CE80E0015F083FE109810F8F9
:1048C000241003A815F05FFE641C4C45EDDB039833
:1048D000401B009000BF009804B0BDE8F09F2DE998
:1048E000F04105460E46022700240AE004EB44008E
:1048F00006EB800393E8070000F02EF8C01C074485
:10490000641CAC42F2DB3846BDE8F0812DE9FC4185
:1049100004460D46164600200190471E0094022DC5
:1049200001DA871E15E000208DF80400019866F377
:10493000071001909DF80410684615F024FE002130
:104940000098FFF745FD0099084400900098071B68
:1049500000BF3846BDE8FC8137B50024009820B17F
:104960000098FBF7F6FC044600E0019C20463EBDA3
:1049700000BFFEE738B5002406E04FF6FF702C4973
:1049800021F81400601C84B2B4F5806FF5DB0024BC
:1049900021E0A101042300226846FEF705FD9DF8F1
:1049A0000000FF2815D19DF802109DF8030001EBCF
:1049B000002085B2B5F5806F0BDA1D4830F8150080
:1049C0004FF6FF71884201D0012038BD184820F809
:1049D0001540601C84B2B4F5806FDADB00240AE075
:1049E000134830F81400B0F5806F02DB11480480E2
:1049F00004E0601C84B2B4F5806FF1DB00BF0D48A9
:104A00000088642801DA0120DFE70AE0084830F86E
:104A100014004FF6FF71884201D00120D5E7601CD9
:104A200084B2044800888442F0DB0020CDE7000017
:104A30003CC900206400002070B5054640F2FF34F8
:104A400005F0400028B104F0010038B9601E84B2BE
:104A500004E004F0010008B1601E84B20CE02046BE
:104A600000F084F808B1204670BD022C02DA4FF63F
:104A7000FF70F9E7A01E84B2F1E738B500250024E5
:104A80000DE02046FEF78EFA204600F051F820B9DE
:104A90002046FEF787FA681C85B2601C84B2B4F524
:104AA000806FEEDB642D01DA012038BD622068439F
:104AB000642190FBF1F085B200200090002418E002
:104AC000204600F035F890B9A10102231A46684645
:104AD000FEF77CFD08B10120E7E7BDF80000401CAF
:104AE00080B20090BDF80000A84200D104E0601C34
:104AF00084B2B4F5806FE3DB00BFFFF73BFF00201B
:104B0000D3E700000448008862225043642290FBEF
:104B1000F2F14804704700006400002010B5FEF771
:104B20006BFAFEF781FCFFF725FF0446204610BD17
:104B300038B50446A101012300226846FEF734FC83
:104B40009DF80000FF2801D0012038BD012000EBB6
:104B50008411034600226846FEF726FC9DF80000FB
:104B6000FF2801D00120F0E70020EEE738B5044629
:104B70002046FFF7DDFF08B1002038BDA101012369
:104B80001A466846FEF710FC9DF80000FF2801D188
:104B90000120F2E70020F0E7014606480088814244
:104BA00002D34FF6FF707047034830F811201046CB
:104BB000F9E70000640000203CC9002038B5044635
:104BC00021460AA003F00AF9A50100200090012364
:104BD000002229466846FEF7F9FC012805D1012389
:104BE0000022691C6846FEF7F1FC38BD4E414E4478
:104BF0005F4D61726B426164426C6F636B28256428
:104C0000290D0A0038B50446A501F02000900123C3
:104C10001A4629466846FEF7D9FC012800D138BD5E
:104C20000020FCE72DE9FF5F81460F4614469A46B7
:104C300000253BE04FF4006090FBF4F0800179190F
:104C4000B1FBF0FB5846FFF7A7FF0646B6F5806FAD
:104C500007D3314617A003F0C1F8012004B0BDE826
:104C6000F09F7819A0FB04104FF400320023CDE927
:104C7000001008460199FBF7F9FA9046B00100EBE5
:104C8000D8200390C8F30A00029005FB0490234645
:104C9000DDE90221FEF728FB012806D11448DDE9F1
:104CA000022103F09BF80120D8E76D1C5545C1D3C4
:104CB0000020D3E74572726F723A204E414E445F36
:104CC000526561644D756C7469536563746F72737A
:104CD00028292C206E6F7420666F726D61742C20F1
:104CE000757350424E203D2025640D0A00000000DF
:104CF000385704082DE9FF4F83B00646894614460D
:104D000000257DE04FF4006090FBF4F0800109EB9A
:104D10000501B1FBF0FA5046FFF73EFF0746B7F535
:104D2000806F08D33A465146384803F057F80120BF
:104D300007B0BDE8F08F4FF4006090FBF4F0800105
:104D400009EB0501B1FBF0F200FB121000FB04FBC4
:104D5000B80100EBDB28CBF30A000290FF222146CA
:104D60002B48FBF7C6FA234641462948029AFEF72C
:104D7000DFF8002832D105FB046023464146029A41
:104D8000FEF760FB012816D122A003F027F805FBEF
:104D9000046123464046029A00F084F8019001988D
:104DA00020B128A003F01AF80120C1E74FEA9810BB
:104DB000FFF704FF23E04FEA9810FFF723FF0128D5
:104DC0001CD105FB046123464046029A00F06AF8B4
:104DD0000190019808B10120AAE710E005FB0461E9
:104DE00023464046029A00F05DF80190019820B1F8
:104DF00020A002F0F3FF01209AE700E000BF6D1C45
:104E000006988542FFF47EAF002091E7C45704085E
:104E10003CD100204572726F72333A204E414E44AD
:104E20005F57726974654D756C7469536563746F0F
:104E3000727328292C205772697465204661696C49
:104E4000650D0A004572726F72343A204E414E442D
:104E50005F57726974654D756C7469536563746FDF
:104E6000727328292C205772697465204661696C19
:104E7000650D0A004572726F72353A204E414E44FC
:104E80005F57726974654D756C7469536563746FAF
:104E9000727328292C205772697465204661696CE9
:104EA000650D0A002DE9FC5F8046894692469B46C7
:104EB000C8F38F1608F03F000190002761E04046DC
:104EC000FFF7BAFD0546B5F5806F06DB294633A02E
:104ED00002F084FF0120BDE8FC9F00242CE0019833
:104EE000844215D104EB851104EB861053464A46E3
:104EF000CDF800B0FEF78CF901281BD1314630A067
:104F000002F06CFF2846FFF759FEFFF733FD15E06E
:104F100004EB851104EB8610FEF7FEF8012809D199
:104F2000314630A002F05AFF2846FFF747FEFFF750
:104F300021FD03E0601C84B2402CD0DB00BF402C7C
:104F40001CD12846FFF75EFE012805D12846FFF751
:104F500035FEFFF70FFD12E03046FEF723F840283C
:104F600009D0314628A002F039FF3046FFF726FE6F
:104F7000FFF700FD03E0FFF7FDFC04E000BF781C35
:104F800087B20A2F9BDB00BF0A2F05D1394628A024
:104F900002F024FF01209EE700209CE74572726F1B
:104FA00072313A204E414E445F5772697465546FB6
:104FB0004E6577426C6F636B28292025640D0A00CB
:104FC0004572726F72323A204E414E445F57726999
:104FD0007465546F4E6577426C6F636B282920258A
:104FE000640D0A004572726F72333A204E414E448E
:104FF0005F5772697465546F4E6577426C6F636B6F
:1050000028292025640D0A004572726F72343A20F7
:1050100046534D435F4E414E445F45726173654256
:105020006C6F636B28292C2025640D0A000000009A
:105030004572726F72353A2046534D435F4E414E72
:10504000445F4572617365426C6F636B2829206E03
:105050003D25640D0A0000001CB50121202001F04F
:105060002DFD4FF48070009001208DF80400002089
:105070008DF8060001208DF8070000208DF805004E
:1050800069460248FEF7F6FC1CBD00000014024011
:10509000704710B54FF4A06000F066F810BD000036
:1050A0002DE9F0410446002500270F26E07810B1D5
:1050B000E078012800D103E0862122A003F04AFE17
:1050C0006078102800DA03E087211EA003F042FE7A
:1050D000A078102800DA03E088211AA003F03AFE35
:1050E000E07818B31D48006800F4E060C0F5E060A7
:1050F000C0F30725C5F10400C7B22E416078B8405F
:10510000C5B2A078304005432807050E1448217821
:105110004554207800F01F01012088402178491172
:10512000890001F1E021C1F8000109E0207800F0D8
:105130001F01012088400B492278521141F82200BA
:10514000BDE8F0812E2E5C4C6962726172696573F4
:105150005C7372635C6D6973632E63000CED00E039
:1051600000E400E080E100E010B50446B4F5E06F33
:105170000BD0B4F5C06F08D0B4F5A06F05D0B4F56E
:10518000806F02D0B4F5407F00D103E0722104A00B
:1051900003F0E0FD084820430849086010BD000006
:1051A0002E2E5C4C69627261726965735C73726306
:1051B0005C6D6973632E63000000FA050CED00E07E
:1051C0002DE9F04105460E461446002711480078A7
:1051D00018B112202070BDE8F0812878012808D08D
:1051E000022807D0032802D0042804D100E000BF21
:1051F00000BF00BF02E001202070ECE700BFFAF71B
:10520000DDFF07462E613846FAF7DCFF00202070EC
:1052100000BFE0E79C00002010B500F015F801F099
:105220002FFA01F04BFA01F06BFA01F0F9F901F0F5
:10523000B9F901F0D5FA01F0FFFA01F09FFA00F098
:10524000D1FF00F019F810BD0748802102E0491E87
:10525000002204C00029FAD1044A054B1A6000223A
:10526000044B1A807047000064F9002060FB0020A6
:10527000E0000020E40000207047000006480078AD
:10528000012808D105480078FF2804D20348007897
:10529000401C024908707047A50000209C000020B7
:1052A00010B500241A480078012830D1FAF786FF9B
:1052B00004461848007820B116480078401E154969
:1052C000087014480078F8B913480078E0B901F084
:1052D00017FB12481249097850F82100114908605B
:1052E0000F4800781049097888420DD00D480068B1
:1052F000806B401C0B49096888630C480068401C9F
:105300000A490860FAF77AFF2046FAF75BFF10BDFA
:10531000A50000209C0000209D00002000E8002047
:105320009F000020B40000209E000020900000207C
:1053300070B5044600262078012801D0002070BDF9
:10534000FAF73CFF06466568002060603046FAF7D1
:1053500039FF2846F3E7000070B5054600261048DF
:10536000007808B1002070BDFAF728FF06460D4806
:105370000468006820B10B4800684068094908606B
:105380003046FAF71FFF4CB1012020700020208129
:10539000656005A02061204601F0F6F82046E2E7AE
:1053A0009C000020940000203F0000002DE9F04107
:1053B00005460F4614464FF000082878012804D00F
:1053C000012020700020BDE8F0813648007818B137
:1053D000022020700020F6E73348007818B10D2035
:1053E00020700020EFE7FAF7E9FE80466E6846B1CC
:1053F000002068604046FAF7E5FE00202070304645
:10540000E1E72A48006890F8300040F002002749A0
:10541000096881F8300000202449096881F83100CA
:1054200022480068C762284601F070F84046FAF743
:10543000C9FE01F02BFAFAF7C1FE80461B4800684E
:1054400090F8310020B101280DD002280AD105E0E2
:1054500016480068066A002020700DE000260E2025
:10546000207009E000BF29461048006801F038F8B4
:1054700000260A20207000BF00BF00200B490968E9
:1054800081F830000949096881F831000749096845
:10549000C8610649096808624046FAF793FE30463B
:1054A00091E700009C0000209D000020AC0000203F
:1054B00070B504460D4600262078012801D0012051
:1054C00070BDFAF77BFE0646A07A60B10023022287
:1054D0002946204600F0C2FF3046FAF773FE01F07D
:1054E000D5F90020ECE7606820B13046FAF76AFE93
:1054F0001420E5E765603046FAF764FE0020DFE738
:105500002DE9F04106460F464FF00008204800788C
:1055100010B10020BDE8F081FAF750FE80461D482A
:105520000468006820B11B48006840681949086099
:105530004046FAF747FEFCB1FAF740FE80461648AF
:105540000568D5B100680068134908604046FAF75D
:1055500039FE6E6006EB8700A860EE602E61AF82B8
:105560000020E882022020700020208165600BA0CE
:105570002061204601F008F808E0064800686060F5
:10558000044804604046FAF71DFE00242046C1E7A7
:105590009C00002094000020C40000203F00000078
:1055A0002DE9F0470446894615464FF0000A207859
:1055B000022804D0012028702046BDE8F087354835
:1055C000007818B10F2028702046F6E7FAF7F6FDAC
:1055D0008246A07A10B14FF0010801E04FF00008B8
:1055E000B9F1000F03D0B9F1010F49D121E0B8F1B1
:1055F000000F17D128A02061666828480068306035
:105600002648066000202070254800686060002061
:105610002081234804605046FAF7D4FD002028700A
:10562000002705E05046FAF7CDFD492028702746AF
:105630002DE005E0002304221946204600F00EFF6D
:10564000A07A0028F6D114A020616668134800688B
:1056500030601248066000202070114800686060C9
:10566000002020810E4804605046FAF7ABFDB8F1E7
:10567000010F01D101F00AF900202870002706E08F
:105680005046FAF79FFD07202870274600BF00BF4D
:10569000384692E79C0000203F000000C400002034
:1056A0009400002070B505460026FAF787FD0646EF
:1056B0006C686068E060606820610020E0823046CD
:1056C000FAF780FD002070BD2DE9F04707468846B7
:1056D00015464FF000093878022804D001202870C0
:1056E0000020BDE8F0873C48007818B102202870FF
:1056F0000020F6E73948007818B10D202870002006
:10570000EFE7FAF75BFD81467C68E08A98B1216992
:10571000081D20610E68E08A401EE082A1682069B1
:10572000884201D1606820614846FAF74BFD0020AD
:1057300028703046D5E72A48006890F8300040F0DD
:1057400004002749096881F83000002024490968CD
:1057500081F8310022480068C0F82C80384600F0FB
:10576000D5FE4846FAF72EFD01F090F8FAF726FD2F
:1057700081461B48006890F8310020B101280DD007
:1057800002280AD105E016480068066A0020287041
:105790000DE000260E20287009E000BF39461048B1
:1057A000006800F09DFE00260A20287000BF00BFA0
:1057B00000200B49096881F830000949096881F81F
:1057C000310007490968C861054909680862484607
:1057D000FAF7F8FC304684E79C0000209D0000208A
:1057E000AC0000202DE9F04105460E460027287840
:1057F000022802D00120BDE8F081FAF7DFFC07465D
:10580000A87A60B1002304223146284600F026FE23
:105810003846FAF7D7FC01F039F80020EBE76C685E
:10582000E08AA18A884204DB3846FAF7CBFC1E20C6
:10583000E1E7E168081DE0600E60E08A401CE0825C
:10584000D4E90210884201D16068E0603846FAF776
:10585000B9FC0020CFE7000010B500240B48007809
:10586000012811D1FAF7AAFC04460948007840B98A
:1058700008480078FF2804D206480078401C0549F3
:1058800008702046FAF79EFC10BD0000A50000201D
:105890009C0000209D00002010B5002413480078D3
:1058A000012821D1FAF78AFC044611480078C0B1DA
:1058B0000F480078401E0E4908700846007860B90D
:1058C0000C48007828B92046FAF77CFC00F0DEFF8F
:1058D0000AE02046FAF776FC06E02046FAF772FC6A
:1058E00002E02046FAF76EFC10BD0000A500002083
:1058F0009D0000209C00002070B505460026104841
:10590000007808B1002070BDFAF758FC06460D4833
:105910000468006820B10B480068406809490860C5
:105920003046FAF74FFC4CB103202070258100204F
:10593000606005A02061204600F026FE2046E2E7D8
:105940009C000020940000203F0000002DE9F0475B
:105950000446884615464FF000092078032804D0F5
:10596000012028702046BDE8F0872D48007818B146
:105970000F2028702046F6E7FAF720FC8146A07A2F
:1059800008B1012700E00027B8F1000F03D0B8F1FB
:10599000010F3AD119E08FB922A0206100202070B8
:1059A000214800686060002020811F48046048464C
:1059B000FAF708FC00202870002605E04846FAF7B0
:1059C00001FC49202870264626E005E0002301223C
:1059D0001946204600F042FDA07A0028F6D111A019
:1059E0002061002020701048006860600020208145
:1059F0000D4804604846FAF7E5FB012F01D100F09D
:105A000045FF00202870002606E04846FAF7DAFB3A
:105A100007202870264600BF00BF3046A3E70000DD
:105A20009C0000203F000000940000202DE9F04180
:105A300005460E46144600272878032803D0012087
:105A40002070BDE8F0813148007810B1022020704C
:105A5000F7E72F48007810B10D202070F1E7FAF732
:105A6000ADFB0746288940B12889401E2881384669
:105A7000FAF7A8FB00202070E3E72648006890F8BA
:105A8000300040F001002349096881F8300000200F
:105A90002049096881F831001E480068C66228461E
:105AA00000F034FD3846FAF78DFB00F0EFFEFAF710
:105AB00085FB07461748006890F8310020B101289F
:105AC00009D0022806D102E0002020700BE00E2051
:105AD000207008E000BF29460E48006800F000FD75
:105AE0000A20207000BF00BF00200A49096881F821
:105AF00030000849096881F8310006490968C86121
:105B00003846FAF75FFB00BF9BE700009C000020CF
:105B10009D000020AC00002070B5044600252078D0
:105B2000032801D0012070BDFAF748FB0546A07A92
:105B300060B1002301221946204600F08FFC284660
:105B4000FAF740FB00F0A2FE0020ECE720894FF6B8
:105B5000FF71884207D22089401C20812846FAF72D
:105B600031FB0020DFE72846FAF72CFB3320DAE789
:105B700010B50B48007890B900F0C2FE09480078D3
:105B80000949087009480749097850F8210008496F
:105B900008600846006807490860FAF716FB10BD60
:105BA000A50000209F0000209E00002000E80020AB
:105BB000B4000020AC000020704700002DE9FE4F2B
:105BC00006460F4690461C464FF00009FAF7F6FAD3
:105BD00081461F48007828B14846FAF7F3FA3C207E
:105BE000BDE8FE8F1B4850F8240060BB0120194916
:105BF00041F824004846FAF7E5FA002342463946C0
:105C0000304600F06FF98246002000900190034674
:105C1000024651460290204600F088FE054635B9FE
:105C20000D48007801280CD100F030FE09E0FAF7A9
:105C3000C5FA81460020074941F824004846FAF792
:105C4000C1FA2846CCE74846FAF7BCFA2820C7E74D
:105C50009C00002000E80020A50000202DE9F04F66
:105C600085B081468A4693461C46DDE90F78129D31
:105C700000200390FAF7A2FA03902348007830B18D
:105C80000398FAF79FFA3C2005B0BDE8F08F1F4853
:105C900050F8240088BB01201C4941F824000398D7
:105CA000FAF790FA2A464146384600F0F9FE2B46AC
:105CB0005A465146484600F015F904901198CDE92E
:105CC000008002953A4620460E9B049900F02EFE75
:105CD000064636B90E48007801280CD100F0D6FDF2
:105CE00009E0FAF76BFA03900020084941F8240014
:105CF0000398FAF767FA3046C6E7FFE70398FAF722
:105D000061FA2820C0E700009C00002000E8002085
:105D1000A5000020704700002DE9F041054600274E
:105D20004748007810B14020BDE8F0811F2D01D117
:105D30003E20F9E7FAF742FA0746FF2D03D1414822
:105D4000006890F83250404850F8254024B9384651
:105D5000FAF738FA4320E7E7012C04D13846FAF77E
:105D600031FA3D20E0E714F8340F3849085C6178D7
:105D700088432178354A505414F834091146085C98
:105D800030B994F8361032480078884330490870AA
:105D9000E06918B12046E16900F0A2FB666A16B11D
:105DA000304600F02BFC0020E06284F8300084F8DC
:105DB000310028480078FF2804D226480078401C8B
:105DC000244908703846FAF7FDF900F045FBFAF768
:105DD000F5F907461F48007820B11E480078401E9C
:105DE0001C490870204600F041F81B480078401E0E
:105DF000194908700020144941F82500A06930B9FC
:105E000000206169886115496069086005E0D4E98E
:105E100005014861D4E90510886111480068606196
:105E20000F4804600FA0E0643846FAF7CBF90E483B
:105E30000078012801D100F029FD002074E700005E
:105E40009C000020AC00002000E80020A100002001
:105E5000A00000209D000020A6000020B800002027
:105E6000B00000203F000000A500002070477047F0
:105E70002DE9F04106460F4614464FF0000815483C
:105E8000007818B112202070BDE8F081FAF796F979
:105E90008046FF2E03D11048006890F832600F480A
:105EA00050F826502DB94046FAF78CF9432020705F
:105EB000EAE7012D05D14046FAF784F94320207026
:105EC000E2E7EF644046FAF77DF90020207000BF5A
:105ED000DAE700009C000020AC00002000E8002071
:105EE0007047000070B5044610464FF0807505609D
:105EF000051F28462C60214E051F28462E604FF0B6
:105F00001236051F28462E604FF00336051F28461F
:105F10002E604FF00236051F28462E607610051FB2
:105F200028462E60051F284629604FF01136051FB0
:105F300028462E604FF01036051F28462E604FF081
:105F40000936051F28462E604FF00836051F2846E3
:105F50002E604FF00736051F28462E604FF006369C
:105F6000051F28462E604FF00536051F28462E6077
:105F70004FF00436051F28462E6070BD896A000860
:105F80002DE9F04105464FF00008FAF717F9804671
:105F9000FF2D05D12048006890F83250012608E016
:105FA0001D48006890F83200A84201D1012600E0A7
:105FB00000261A4850F825402CB94046FAF702F955
:105FC0004820BDE8F081012C04D14046FAF7FAF8E8
:105FD0004320F6E794F834701148C05D94F835100A
:105FE00088430F49C8550846C05D30B994F836104B
:105FF0000C48007888430B49087094F8300040F052
:10600000080084F830004046FAF7DCF8012E01D190
:1060100000F03CFC0020D4E7AC00002000E80020A9
:10602000A1000020A00000207047000070B50546C8
:1060300000261748007800B170BD1648007800B1FE
:10604000FAE71DB3FAF7BAF806461348006890F865
:1060500034401248005D1049096891F835108843B2
:106060000E4908550846005D40B90B48006890F895
:1060700036100B48007888430949087006480068C4
:10608000C5623046FAF79EF800F000FC00BFD3E787
:106090009C0000209D000020AC000020A1000020FA
:1060A000A000002070B50025FAF788F805460348DF
:1060B00004682846FAF786F8204670BDC80000201C
:1060C00070B5002600F072F8FAF778F80646314805
:1060D0000068401C2F4908603046FAF773F82E48D4
:1060E0000078012853D12D48007820B1012804D030
:1060F000022809D103E001250BE0002509E0012574
:1061000001202649087004E0012500202349087079
:1061100000BF00BF05B970BD2148046833E0FAF73D
:106120004DF80646E06A50B3E06A401EE062E06A5D
:1061300028BB94F8300000F0370040B114F8300F5D
:1061400000F0C800207001206070303C02E00020A8
:1061500084F8310094F8300000F0080078B9343445
:10616000A0781049097808430E49087020780E4934
:10617000085C6178084314F834190B4A5054646978
:106180003046FAF71FF894F832001F28C7D100BF35
:10619000C1E70000C8000020A5000020BC000020CE
:1061A000B8000020A0000020A100002010B5074882
:1061B0000088401C05490880084600880A2803DB3F
:1061C0000020088000F004F810BD0000E40000206A
:1061D00010B503480068FFF79FFC0446204610BD39
:1061E000D8000020F8B54FF42071284800F0EEFAEE
:1061F0004021274800F0EAFA002514E0681C86B226
:1062000005EB8500214901EBC00406EB860001EB9C
:10621000C00764202070002084F82500E7601DA0DE
:106220002062681C85B20F2DE8D305EB8500174965
:1062300001EBC00464202070002084F82500E06099
:1062400014A020620020144908601449088010201E
:10625000134908800D48134908600120FFF74CFBE3
:10626000114908600020FFF747FB104908606A46A3
:106270000FA10D480068FEF7A3FF6A4611A10B4865
:106280000068FEF79DFF00F027F8F8BDA4F4002099
:1062900024F900203F000000D0000020CE000020A4
:1062A000CC000020DC000020D4000020D80000201A
:1062B00075432F4F532D494920546D724C6F636BBA
:1062C0000000000075432F4F532D494920546D7233
:1062D0005369676E616C000000B587B00320002130
:1062E00080220A4BCDE90132CDE903104FF6FD7053
:1062F0000123074A00900748FFF7B0FC06AA06A151
:106300000120FFF7B5FD07B000BD000024F7002015
:1063100020F900209563000875432F4F532D4949FC
:1063200020546D720000000070B50B46032580F804
:106330002550012B05D1154EC56936683544456198
:106340000CE085692DB9114EC56936683544456143
:1063500004E00E4E8569366835444561057D05F0DB
:1063600007040B4D05EBC4010D682DB9086000252D
:10637000C56001258D8006E00A680860C260106172
:106380008D886D1C8D800025056170BDD0000020BA
:1063900024F9002008B500BF00BF6A4600211A4852
:1063A0000068FFF743FBFFF757FA18480068401CE6
:1063B000164908600846007800F00708144800EB0A
:1063C000C8073C681AE0E6681049606909688842B5
:1063D00013D1204600F01EF894F82400022804D1BE
:1063E00001212046FFF7A0FF02E0022084F82500EB
:1063F000656815B12046A168A8473446002CE2D153
:10640000FFF74AFAC9E70000D8000020D0000020BA
:1064100024F9002030B5057D05F007040D4D05EB8E
:10642000C4031D68854205D1C168196039B10025D2
:106430000D6104E00169C268CA6002B11161012501
:1064400080F825500025C56005619D886D1E9D80E2
:1064500030BD000024F90020704700002DE9F04F06
:1064600005460F4690469946A87A19490E5C05F1F3
:106470000B00805D11F800B00BEBC60000F0FF0AC6
:10648000144850F82A4000202034E0602760207C27
:1064900020EA0800207484F81190207C203C00F051
:1064A000080068B994F836000B49097808430A498E
:1064B00008700A48805D94F83510084307498855EC
:1064C0002946204600F00CF85046BDE8F08F000049
:1064D0000E54040800E80020A0000020A1000020C5
:1064E00010B590F8342001F10B039B5C90F8354017
:1064F000A34301F10B04A35423469B5C23B98B7A7D
:1065000090F83640A3438B7210BD000010B51B4AB3
:106510001268D061194A126892F8343000F10B0207
:10652000D25C164B1B6893F835301A43134B1B682B
:1065300093F8344000F10B031A55827A0F4B1B6815
:1065400093F836301A4382720C4A126892F834106B
:106550000B4A525C094B1B6893F835309A43084B41
:106560005A541A46525C42B9044A126892F83630BC
:10657000044A12789A43034B1A7010BDAC000020F5
:10658000A1000020A0000020014600228A72002005
:1065900005E0002301F10B021354421CD0B2042881
:1065A000F7D370472DE9F0415021114800F00EF962
:1065B00000250DE0681C86B20D4800EB051400EBC9
:1065C00006170020207067600AA0E060681C85B292
:1065D000042DEFD3064800EB051400202070606006
:1065E00004A0E060024804490860BDE8F0810000B2
:1065F000B0E500203F0000009800002030B50146C3
:106600004A6808682AB9CC68606028B100254560EE
:1066100002E0106000B142608B6800255D6230BD11
:1066200070B54FF42071134800F0D0F8002411E049
:10663000601C85B204EB84000E4901EB800305EB7E
:10664000850001EB8006002018705E600AA01861CA
:10665000601C84B21F2CEBD304EB8400054901EBD2
:10666000800300201870586003A018610846034991
:10667000086070BD30E300203F000000940000205F
:106680000020074908600749087007490870074952
:106690000870074908700749086007490860704793
:1066A000C80000209C0000209D000020A6000020C3
:1066B000A500002090000020A800002000210A4A28
:1066C0001170002004E00021084A1154411CC8B296
:1066D0000428F8D30021064A1170064A1170064AB0
:1066E0001160064A11607047A0000020A100002040
:1066F0009E0000209F000020B4000020AC0000207D
:1067000070B540F62C21184800F060F88021174839
:1067100000F05CF8002413E0601CC5B2C4EBC400B8
:1067200000EB4000104901EB8003C5EBC50000EB16
:10673000400001EB80065E610DA0D864601CC4B20D
:106740001E2CE9D3C4EBC40000EB4000064901EB6A
:1067500080030020586106A0D86400200549086025
:1067600001480549086070BD80E8002000E800206D
:106770003F000000B8000020B000002000B587B046
:106780000320002180220A4BCDE90132CDE903101C
:106790004FF6FF701F23074A00900748FFF75EFA85
:1067A00006AA06A11F20FFF763FB07B000BD00008B
:1067B00000E60020FCE70020616A000875432F4FC7
:1067C000532D49492049646C6500000004E0002213
:1067D00000F8012B4A1E91B20029F8D17047000041
:1067E00070B578211148FFF7F1FF00240EE004EBAB
:1067F00044000E4901EBC005601C00EB400001EBBA
:10680000C00068600AA06861601C84B2042CEED3EA
:1068100004EB4400054901EBC0050020686004A0BA
:10682000686108460349086070BD0000ACF20020B2
:106830003F000000C00000202DE9F0414FF4C0717E
:106840001048FFF7C3FF00240DE0601C86B204EB84
:1068500044000C4901EBC00506EB460001EBC00704
:106860002F60601C84B20F2CEFD304EB4400054969
:1068700001EBC00500202860084603490860BDE818
:10688000F081000024F30020C400002010B5002493
:10689000F9F794FC044613480078F8B912480078D8
:1068A000E0B900F02DF811481149097850F821009D
:1068B000104908600E4800780F49097888420DD0C9
:1068C0000C480068806B401C0A49096888630B48C3
:1068D0000068401C09490860F9F78BFC2046F9F76D
:1068E00071FC10BD9C0000209D00002000E80020ED
:1068F0009F000020B40000209E0000209000002097
:106900000649074A1278885C0649095C034A515CCB
:1069100001EBC001044A1170704700000E540408D6
:10692000A0000020A10000209F0000202DE9F84FCA
:1069300005460F4690469946DDE90AAB00200090D7
:10694000F9F73CFC00903F480468002C74D01834E0
:1069500054F8040C3B4908600098F9F733FC44F8FC
:10696000187CA576002020766076606144F814BC1F
:1069700044F80CAC44F8108C0C9824F8080C24F85B
:10698000069C0020E077E810207705F00700E0760D
:10699000217F01208840A077E17E01208840607738
:1069A00000206060E060A0602062A0626062E0623F
:1069B000206325A06063183C002606E0002104F156
:1069C000500040F82610701CC6B2012EF6DB20469F
:1069D000FFF7F2F82046FFF79DF9F9F7EFFB00907B
:1069E0001A4840F825401A48006860610020A061FC
:1069F0001748006810B116480068846114480460A4
:106A00003434A07813490978084312490870207873
:106A10001149085C6178084314F834190E4A50543F
:106A20000E480078401C0D4908700098F9F7CAFB21
:106A30000020BDE8F88FFFE70098F9F7C3FB42207C
:106A4000F7E70000B00000203F00000000E8002051
:106A5000B8000020A0000020A1000020A600002017
:106A6000002400BF00BFF9F7A9FB044605480068F1
:106A7000401C044908602046F9F7A4FBFFF7F7F92A
:106A8000F1E70000A800002010B504480068FFF7F7
:106A900027FAFF20FFF740F910BD0000AC000020EE
:106AA00002F0010343B102F002032BB102E0491EE0
:106AB000002308C00029FAD17047000070B50446D1
:106AC0000D461048204008B904B104E040F24441AA
:106AD0000DA002F03FF90DB1012D00D104E040F20C
:106AE000464109A002F036F92DB110480068204354
:106AF0000E49086004E00D480068A0430B49086097
:106B000070BD000000EE9B812E2E5C4C69627261AC
:106B1000726965735C7372635C73746D3332663271
:106B200078785F7263632E630000000030380240A3
:106B300070B504460D461048204008B904B104E081
:106B40004FF4A0610DA002F005F90DB1012D00D1A7
:106B500004E040F2015109A002F0FCF82DB1104808
:106B6000006820430E49086004E00D480068A04317
:106B70000B49086070BD000000EE9FDD2E2E5C4CBE
:106B800069627261726965735C7372635C73746D60
:106B90003332663278785F7263632E6300000000E0
:106BA0001038024070B504460D4624F0010008B9C3
:106BB00004B104E040F27F410CA002F0CBF80DB12B
:106BC000012D00D104E04FF4906108A002F0C2F85A
:106BD0002DB10F48006820430D49086004E00C48BF
:106BE0000068A0430A49086070BD00002E2E5C4C6E
:106BF00069627261726965735C7372635C73746DF0
:106C00003332663278785F7263632E63000000006F
:106C10003838024070B504460D461048204008B987
:106C200004B104E040F2B1410DA002F093F80DB1BF
:106C3000012D00D104E040F2B24109A002F08AF82F
:106C40002DB11048006820430E49086004E00D484B
:106C50000068A0430B49086070BD0000003601C900
:106C60002E2E5C4C69627261726965735C7372632B
:106C70005C73746D3332663278785F7263632E634F
:106C8000000000004038024070B504460D46104830
:106C9000204008B904B104E040F2D9410DA002F04F
:106CA00059F80DB1012D00D104E040F2DA4109A0FC
:106CB00002F050F82DB11048006820430E490860DA
:106CC00004E00D480068A0430B49086070BD000057
:106CD000CCA0F8FF2E2E5C4C6962726172696573FC
:106CE0005C7372635C73746D3332663278785F7292
:106CF00063632E630000000044380240F0B50021B9
:106D000000220024022500260223324F3F6807F0AC
:106D10000C0121B1042905D0082937D105E02E4FF7
:106D2000076036E02D4F076033E02A4F3F1F3F6872
:106D3000C7F38056274F3F1F3F6807F03F036EB1F0
:106D4000264FB7FBF3F7DFF88CC0ACF1040CDCF88E
:106D500000C0CCF3881C07FB0CF40CE01E4FB7FB03
:106D6000F3F7DFF870C0ACF1040CDCF800C0CCF332
:106D7000881C07FB0CF4174F3F1F3F68C7F3014700
:106D80007F1C7D00B4FBF5F7076002E0124F07603F
:106D900000BF00BF0F4F3F6807F0F0010909104F17
:106DA0007A5C0768D74047600A4F3F6807F4E051B4
:106DB000890A0B4F7A5C4768D7408760054F3F6868
:106DC00007F46041490B064F7A5C4768D740C760BB
:106DD000F0BD0000083802400024F40040787D0136
:106DE0003C0000201CB501217820FFF767FE002041
:106DF0008DF806008DF8070002208DF804000320AE
:106E00008DF80500012000906946E548FCF732FE48
:106E10000C220021E248FCF7FDFE022000906946AA
:106E2000DF48FCF727FE0C220121DD48FCF7F2FECB
:106E3000042000906946DA48FCF71CFE0C2202216F
:106E4000D748FCF7E7FE082000906946D448FCF7D5
:106E500011FE0C220321D248FCF7DCFE102000902A
:106E60006946CF48FCF706FE0C220421CC48FCF70B
:106E7000D1FE202000906946C948FCF7FBFD0C229A
:106E80000521C748FCF7C6FE4FF4805000906946C4
:106E9000C348FCF7EFFD0C221146C148FCF7BAFECF
:106EA0004FF4005000906946BD48FCF7E3FD0C220A
:106EB0000D21BB48FCF7AEFE4FF4804000906946C0
:106EC000B748FCF7D7FD0C220E21B548FCF7A2FE0F
:106ED0004FF4004000906946B148FCF7CBFD0C220E
:106EE0000F21AF48FCF796FE012000906946AD489F
:106EF000FCF7C0FD0C220021AA48FCF78BFE022003
:106F000000906946A748FCF7B5FD0C220121A54871
:106F1000FCF780FE042000906946A248FCF7AAFD19
:106F20000C2202219F48FCF775FE0820009069465C
:106F30009C48FCF79FFD0C2203219A48FCF76AFE4F
:106F40001020009069469748FCF794FD0C2204211C
:106F50009448FCF75FFE2020009069469148FCF7BA
:106F600089FD0C2205218F48FCF754FE4FF4006088
:106F7000009069468C48FCF77DFD0C220B218A4865
:106F8000FCF748FE4FF48050009069468648FCF7B5
:106F900071FD0C2211468448FCF73CFE4FF4005072
:106FA000009069468048FCF765FD0C220D217E4863
:106FB000FCF730FE4FF48040009069467A48FCF7B9
:106FC00059FD0C220E217848FCF724FE4FF40040B6
:106FD000009069467448FCF74DFD0C220F21724861
:106FE000FCF718FE0120009069466F48FCF742FD4F
:106FF0000C2200216C48FCF70DFE0220009069462F
:107000006948FCF737FD0C2201216748FCF702FEB6
:107010008020009069466548FCF72CFD0C22072172
:107020006248FCF7F7FD4FF48070009069465F48B6
:10703000FCF720FD0C2208215C48FCF7EBFD4FF427
:107040000070009069465948FCF714FD0C22092194
:107050005648FCF7DFFD4FF48060009069465348C6
:10706000FCF708FD0C220A215048FCF7D3FD4FF431
:107070000060009069464D48FCF7FCFC0C220B2197
:107080004A48FCF7C7FD4FF48050009069464748D6
:10709000FCF7F0FC0C2211464448FCF7BBFD4FF412
:1070A0000050009069464148FCF7E4FC0C220D2199
:1070B0003E48FCF7AFFD4FF48040009069463B48E6
:1070C000FCF7D8FC0C220E213848FCF7A3FD4FF446
:1070D0000040009069463548FCF7CCFC0C220F219B
:1070E0003248FCF797FD4FF48070009069462E48B7
:1070F000FCF7C0FC0C2208212B48FCF78BFD4FF459
:107100000070009069462848FCF7B4FC0C22092165
:107110002548FCF77FFD4FF48060009069462248C7
:10712000FCF7A8FC0C220A211F48FCF773FD4FF462
:107130008060009069461B48FCF79CFC0C220A21E9
:107140001848FCF767FD2020009069461648FCF7B8
:1071500091FC0C2205211448FCF75CFD10200090E6
:1071600069461148FCF786FC0C2204210E48FCF706
:1071700051FD0220009069460C48FCF77BFC0C2274
:1071800001210A48FCF746FD0120009069460748A6
:10719000FCF770FC0C2200210448FCF73BFD1CBDF1
:1071A0000014024000180240000C0240001002408F
:1071B0007047000010B504460CB1012C00D103E06B
:1071C000942103A001F0C6FD0A48046010BD000030
:1071D0002E2E5C4C69627261726965735C737263B6
:1071E0005C73746D3332663278785F73797363667B
:1071F000672E6300DC0027420CB500200190009050
:107200002D48006840F480302B49086000BF2A48B0
:10721000006800F4003000900198401C0190009834
:1072200018B90198B0F5A06FF1D12348006800F4B7
:10723000003010B10120009001E000200090009883
:10724000012838D11C48083000681B490831086003
:107250000846006840F4004008600846006840F4B2
:10726000A05008601548091F0860081F006840F01A
:107270008070091F086000BF0F48006800F00070B0
:107280000028F9D040F203700D4908600A48083020
:10729000006820F0030008490831086008460068CB
:1072A00040F00200086000BF03480830006800F0AA
:1072B0000C000828F8D10CBD00380240193C4005EC
:1072C000003C024010B50446042C01D0601D00B9FA
:1072D00003E0DB210BA001F03DFD042C08D14FF0B1
:1072E000E020006940F004004FF0E021086107E071
:1072F0004FF0E020006920F004004FF0E021086129
:1073000010BD00002E2E5C4C69627261726965735B
:107310005C7372635C6D6973632E630010B507481C
:107320000078012808D1FDF7A9FFFEF7C9FEFDF797
:10733000B7FF01200EF0EAFE10BD0000A5000020FE
:1073400010B51348006840F00100114908600020A2
:107350000F49083108600E4800680E4908400C4982
:1073600008600D48091D0860081F006820F480208F
:10737000091F0860002006490C31086000F010F871
:10738000FFF73AFF4FF000600449086010BD0000AD
:1073900000380240FFFFF6FE1030002408ED00E048
:1073A00010B5FCF733FB10BD10B50BF0CDF810BDD8
:1073B00010B540F22441104800F03EFAD0B10E481A
:1073C0000488001D048800210C48F9F755FF0B487C
:1073D000F9F7C4FF41F28831081A094908600949E0
:1073E0000648F9F73DFE01210448F9F745FF012061
:1073F0000549087010BD00000014014028640240D7
:1074000060000020008800105C00002000B587B0FC
:1074100001210846FFF752FB01211020FFF734FC41
:1074200007220A212948FCF7F5FB072209212748F2
:10743000FCF7F0FB4FF4C060019002208DF80800CB
:1074400000208DF80A0001208DF80B0002208DF835
:10745000090001A91D48FCF70DFB4FF4E130039032
:107460000020ADF81000ADF81200ADF814000C20AB
:10747000ADF816000020ADF8180003A9144800F07C
:1074800025FB0121124800F015F94021104800F0B9
:10749000B3F8012240F225510D4800F077FA01229D
:1074A00040F224410A4800F071FA25208DF80000CE
:1074B00000208DF801008DF8020001208DF80300F6
:1074C0006846FDF7EDFD07B000BD0000000002407A
:1074D0000010014010B5012211030248FCF790FD95
:1074E00010BD0000000802401CB501210420FFF778
:1074F000E5FA4FF48050009001208DF80400002040
:107500008DF806008DF8070002208DF80500694609
:107510000148FCF7AFFA1CBD0008024000B587B077
:10752000FFF7E2FF01210420FFF7C8FA01218804D8
:10753000FFF770FB07220B212D48FCF76BFB07229E
:107540000A212B48FCF766FB4FF480600190022073
:107550008DF8080000208DF80A008DF80B0002203D
:107560008DF8090001A92248FCF784FA4FF4006065
:10757000019002208DF8080001A91D48FCF77AFA55
:107580004FF4165003900020ADF81000ADF8120033
:10759000ADF814000C20ADF816000020ADF818006E
:1075A00003A9144800F092FA0121124800F082F871
:1075B0004021104800F020F8012240F225510D48EA
:1075C00000F0E4F9012240F224410A4800F0DEF91B
:1075D00027208DF8000000208DF801008DF80200B2
:1075E00001208DF803006846FDF75AFD07B000BD85
:1075F000000802400048004070B504460D461E4891
:1076000084420ED01D4884420BD01D48844208D0CD
:107610001C48844205D01C48844202D01B48844246
:1076200000D104E040F22B5119A001F093FB4FF67A
:107630009F40284008B905B104E040F22C5114A045
:1076400001F088FB05F40070B0F5007F11D10A4805
:10765000844208D00948844205D00948844202D0B7
:107660000A48844200D104E040F2315108A001F000
:1076700071FBE843208070BD0010014000440040D1
:1076800000480040004C0040005000400014014001
:107690002E2E5C4C69627261726965735C737263F1
:1076A0005C73746D3332663278785F7573617274AF
:1076B0002E63000070B504460D46164884420ED075
:1076C000154884420BD01548844208D0144884429F
:1076D00005D01448844202D01348844200D104E00B
:1076E0004FF4CD7111A001F035FB0DB1012D00D18A
:1076F00004E040F29B110DA001F02CFB25B1A08904
:1077000040F40050A08104E0A0894DF6FF710840CC
:10771000A08170BD001001400044004000480040BE
:10772000004C004000500040001401402E2E5C4CE4
:1077300069627261726965735C7372635C73746DA4
:107740003332663278785F75736172742E6300002D
:1077500070B505460C460026284885420ED02848BC
:1077600085420BD02748854208D02748854205D05E
:107770002648854202D02648854200D104E040F2E6
:10778000FB4124A001F0E6FA012C13D0802C11D08B
:10779000402C0FD0202C0DD0102C0BD0B4F5807FB6
:1077A00008D0B4F5007F05D0082C03D0042C01D0FC
:1077B000022C00D104E040F2FC4116A001F0CAFA0C
:1077C000B4F5007F11D10D48854208D00C488542A0
:1077D00005D00C48854202D00D48854200D104E016
:1077E00040F201510BA001F0B5FA2888204008B101
:1077F000012600E00026304670BD00000010014068
:107800000044004000480040004C00400050004050
:10781000001401402E2E5C4C6962726172696573BE
:107820005C7372635C73746D3332663278785F7543
:10783000736172742E6300002DE9F04705460C4613
:1078400000270026B046B146414885420ED0414847
:1078500085420BD04048854208D04048854205D03B
:107860003F48854202D03F48854200D104E040F2C3
:107870004F513DA001F06EFA282C27D040F227701E
:10788000844223D040F2266084421FD040F225502B
:1078900084421BD040F22440844217D040F6460078
:1078A000844213D040F66A1084420FD0B4F5587F5A
:1078B0000CD040F22530844208D0B4F5587F05D072
:1078C000B4F5187F02D0B4F5B07F00D104E04FF4D6
:1078D000AA6125A001F03EFA40F66A10844211D157
:1078E0001B48854208D01B48854205D01A4885426E
:1078F00002D01C48854200D104E040F255511AA044
:1079000001F028FAC4F3421804F01F06012000FA1F
:1079100006F6B8F1010F02D1A889064007E0B8F1D8
:10792000020F02D1288A064001E0A88A06402712E9
:10793000012000FA07F7288807401EB117B14FF061
:10794000010901E04FF000094846BDE8F08700005A
:10795000001001400044004000480040004C00403E
:1079600000500040001401402E2E5C4C6962726190
:10797000726965735C7372635C73746D3332663203
:1079800078785F75736172742E6300002DE9F0479B
:1079900004460D4617464FF00008C246C146002671
:1079A0003B4884420ED03B4884420BD03A48844244
:1079B00008D03A48844205D03948844202D0394838
:1079C000844200D104E040F2BC4137A001F0C2F98A
:1079D000282D19D040F22770854215D040F226603C
:1079E000854211D040F2255085420DD040F224400E
:1079F000854209D040F64600854205D040F66A101F
:107A0000854201D0602D00D104E040F2BD4126A0A6
:107A100001F0A0F90FB1012F00D104E040F2BE4106
:107A200021A001F097F940F66A10854211D118485B
:107A3000844208D01748844205D01748844202D0B7
:107A40001848844200D104E040F2C34116A001F07E
:107A500081F92646C5F3421805F01F0A012000FAF5
:107A60000AF9B8F1010F01D10C3605E0B8F1020FA7
:107A700001D1103600E0143627B1306840EA090021
:107A8000306003E0306820EA09003060BDE8F0872C
:107A9000001001400044004000480040004C0040FD
:107AA00000500040001401402E2E5C4C696272614F
:107AB000726965735C7372635C73746D33326632C2
:107AC00078785F75736172742E6300002DE9FF474B
:107AD00005460C460026B14600BFB0466D488542BB
:107AE0000ED06D4885420BD06C48854208D06C485A
:107AF000854205D06B48854202D06B48854200D153
:107B000003E0EA2169A001F025F9206820B170495D
:107B10002068884200D203E0EB2164A001F01AF94A
:107B2000A08818B1A088B0F5805F00D103E0EC21F7
:107B30005EA001F00FF9E08858B1E088B0F5805FF1
:107B400007D0E088B0F5005F03D0E088B0F5405F73
:107B500000D103E0ED2155A001F0FCF8208938B1F7
:107B60002089B0F5806F03D02089B0F5C06F00D1B7
:107B700003E0EE214DA001F0EDF860894FF6F371BE
:107B8000084010B9608900B103E0EF2147A001F07F
:107B9000E1F8A08958B1A089B0F5807F07D0A0890D
:107BA000B0F5007F03D0A089B0F5407F00D103E09D
:107BB000F0213EA001F0CEF8A08980B13548854281
:107BC00008D03548854205D03448854202D0364831
:107BD000854200D103E0F52134A001F0BBF82E8AE4
:107BE00026F44056E08806432E82AE8941F20C60AE
:107BF0008643A08821890843618908430643AE81F2
:107C0000AE8A26F44076A0890643AE826846FFF726
:107C100075F82048854202D02348854202D1DDF81C
:107C20000C9001E0DDF80890A88900F4004040B114
:107C300009EBC90000EB091021684900B0FBF1F71E
:107C400007E009EBC90000EB091021688900B0FBCF
:107C5000F1F76420B7FBF0F006013009642101FB65
:107C60001078A88900F4004040B1322000EBC80031
:107C7000B0FBF1F000F00700064308E0322000EB13
:107C800008106421B0FBF1F000F00F0006432E81D4
:107C9000BDE8FF870010014000440040004800405C
:107CA000004C004000500040001401402E2E5C4C5F
:107CB00069627261726965735C7372635C73746D1F
:107CC0003332663278785F75736172742E630000A8
:107CD000E170720010B504460D4884420ED00D4884
:107CE00084420BD00C48844208D00C48844205D012
:107CF0000B48844202D00B48844200D104E04FF488
:107D00000B7109A001F026F8A088C0F3080010BD8F
:107D1000001001400044004000480040004C00407A
:107D200000500040001401402E2E5C4C69627261CC
:107D3000726965735C7372635C73746D333266323F
:107D400078785F75736172742E63000070B50446B5
:107D50000D46124884420ED0114884420BD011487F
:107D6000844208D01048844205D01048844202D092
:107D70000F48844200D104E04FF407710DA000F0D9
:107D8000E9FFB5F5007F00DA04E040F21D2109A00B
:107D900000F0E0FFC5F30800A08070BD00100140B6
:107DA0000044004000480040004C004000500040AB
:107DB000001401402E2E5C4C696272617269657319
:107DC0005C7372635C73746D3332663278785F759E
:107DD000736172742E63000000BFFEE70FB4054BA1
:107DE00010B503A9044A029800F01AF910BC5DF816
:107DF00014FB000099E90008D40100200FB4084BDF
:107E000010B504A902AA039800F00AF9044602A9D1
:107E1000002000F09CFC204610BC5DF814FB000024
:107E20004F87000800487047E00100202DE9F04727
:107E300082460F4C10480D4E0E4F001B4FF00008AD
:107E400020F007054FF0010900221146504607F0C7
:107E5000E5FD002802D1306810B10020BDE8F087B0
:107E60003C60C4E90058C6F80090EDE7DC01002052
:107E7000FC850120D8010020F8A5012002E008C8F7
:107E8000121F08C1002AFAD170477047002001E094
:107E900001C1121F002AFBD1704700002DE9FF5FCE
:107EA00082B00021DDE90430020DDDF840B003436B
:107EB00018D044F61050A2F2FF3242431514119824
:107EC00001281FD0A5EB0B00401C5FEA000A4FF011
:107ED00000064E4FDFF83891B046504615D5CAF12E
:107EE000000413E0119801244AA3012801D16FEA8C
:107EF0000B010298119AC0E90031C0E9024206B0B4
:107F0000BDE8F09FCBF10000DFE704460021404AC6
:107F1000491842EB0450CDE9001012E0E00707D009
:107F200032463B4640464946F8F75FFC8046894664
:107F300032463B4610461946F8F757FC06460F46B0
:107F40006410002CEAD1DDE90401DDE90023BAF177
:107F5000000F06DAF8F749FC42464B46F8F745FCB5
:107F600005E0F8F7B4FC42464B46F8F7B0FC04468F
:107F70000E460022284BF8F719FD03D84FF0FF30CA
:107F8000014607E00022254B20463146F8F786FBE4
:107F9000F8F768FE102409E0002C0ADB0A2200230F
:107FA000F8F764F9039B30321A55641E50EA010257
:107FB000F2D1641C039AC4F111031444119A012AEA
:107FC00003D0012208430DD10AE0084304D0002069
:107FD0004FF0110B119072E7A3EB0B056D1E0DE036
:107FE0005B4504DD4FF0000205F1010504E003DA12
:107FF0004FF00002A5F10105002AECD0029811997A
:10800000C0E90231C0E9004579E7000000001440F2
:108010000000F03F300000000000F0430000E03FAF
:108020002DE9FF4F95B09B468946064600250FE295
:10803000252877D100242746F84A0121059400E03D
:10804000044316F8013F203B01FA03F01042F7D138
:1080500030782A2811D06FF02F033078A0F1300249
:10806000092A16D8059A44F0020402EB820203EBB7
:1080700042021044761C0590EFE759F8042B059254
:10808000002A03DA504244F40054059044F00204FC
:10809000761C30782E2816D116F8010F44F004040F
:1080A0002A280DD06FF02F023078A0F13003092B71
:1080B00009D807EB870302EB4303C718761CF3E7E5
:1080C00059F8047B761C30786C280FD006DC4C28DD
:1080D00017D068280DD06A2814D104E0742810D075
:1080E0007A280FD10DE044F400140AE044F480141F
:1080F00001E044F440147278824202D104F5801405
:10810000761C761C307866280BD013DC582877D084
:1081100009DC002875D04528F6D04628F4D0472839
:108120001AD19DE118E0632835D0642879D06528FC
:1081300012D195E1702873D008DC6728F1D0692846
:108140006FD06E280DD06F2806D1B5E073282CD0E3
:10815000752875D0782874D05A46179990476D1CA9
:1081600075E1C4F30250022809D003280DD0D9F8D4
:10817000001004280DD00D6009F1040967E1D9F859
:108180000010EA17C1E90052F6E7D9F800100D8097
:10819000F2E70D70F0E719F8041B8DF800100020CD
:1081A0008DF80100EA46012003E059F804AB4FF0D6
:1081B000FF3061074FF0000102D40DE008F101012A
:1081C0008846B9420FDA8045F8DB1AF80810002912
:1081D000F4D108E008F1010188468142FADB1AF87F
:1081E00008100029F6D105985B46A0EB0807214648
:1081F0003846179A00F094FA284400EB080507E087
:108200004DE029E10DE01AF8010B5A461799904705
:10821000B8F10108F7D25B4621463846179A13E1B8
:1082200042E00A220092C4F302524FF0000A022AEE
:1082300008D059F804CB032A4FEAEC710AD00DE0BC
:1082400029E02AE009F1070121F00702F2E802C162
:10825000914609E00FFA8CFC4FEAEC71042A03D135
:108260004FFA8CFC4FEAEC71002907DA0A4600212C
:10827000DCF1000C61EB02012D2202E0220504D5A5
:108280002B228DF80420012203E0E20701D02022F6
:10829000F7E7904659E00A2102E010220DE0102194
:1082A0004FF0000A00910BE010224FF0000A44F05A
:1082B00004040827009203E008224FF0000A00920D
:1082C000C4F30252022A05D059F804CB0021032A34
:1082D00008D009E009F1070121F00702F2E802C124
:1082E000914605E01FFA8CFC042A01D10CF0FF0C2A
:1082F0004FF00008220728D5702806D0009B83F095
:10830000100353EA0A0305D00EE040228DF8042042
:10831000012208E05CEA010206D030228DF8042038
:108320008DF8050002229046009B83F0080353EA73
:108330000A030AD15CEA010201D1620705D53022A5
:108340008DF804204FF001087F1E582804D034A077
:1083500003900EA802900DE036A0F9E75346604660
:10836000009AF7F783FF84460398825C0298401EC8
:10837000029002705CEA0100F0D1029806A9081A86
:1083800000F1200A600702D524F4803400E00127C0
:10839000574502DDA7EB0A0000E0002000EB0A01D0
:1083A000009005984144401A0590E00306D45B46CE
:1083B0002146179A059800F0B3F90544002706E016
:1083C00001A85A46C05D179990476D1C7F1C474510
:1083D000F6DBE0030CD55B462146179A059800F0C2
:1083E0009FF9054404E030205A46179990476D1CC8
:1083F0000099481E00900029F5DC08E002980299D7
:108400005A460078491C0291179990476D1CBAF1A1
:108410000001AAF1010AF1DC65E100000928010070
:1084200030313233343536373839616263646566EA
:1084300000000000303132333435363738394142AC
:10844000434445460000000000F058F90544761CFE
:10845000307800287FF4ECAD19B02846BDE8F08FE5
:10846000620700D4062709F1070222F0070CFCE896
:108470000223E14603F000485FEA080C02D00FF245
:10848000702C0DE05FEA045C02D50FF2682C07E067
:108490005FEAC47C02D00FF2602C01E0AFF2700CF6
:1084A0004FF0FF3823F00043CDF850C065280CD0C2
:1084B00006DC452809D046281DD047283DD13DE09F
:1084C000662818D067287ED138E00021112F01DB03
:1084D000112000E0781CCDE9000106A90EA8FFF7E5
:1084E000DDFCDDE90F010E9A03910021009207F1F6
:1084F000010A04914DE04FF000400097CDE90110D2
:1085000006A90EA8FFF7CAFCDDE90F0203920E9B35
:1085100011990022DDF80CA00093049211B9791C86
:1085200000EB010AB7EB0A0004D4C0F1FF3007F1F9
:10853000010A0490AAEB0700019044E0012F00DA41
:1085400001270021112F01DD112000E03846CDE97F
:10855000000106A90EA8FFF7A1FCDDE90F010E9AA4
:108560000391002104910092BA4621070CD403998B
:10857000514500DA8A46BAF1010F05DD009AAAF1E9
:108580000101515C302908D0B84202DA10F1040F21
:1085900006DA0121CDE9011015E0AAF10101E9E7B0
:1085A000002805DC049901440491AAEB000102E0D3
:1085B000411C514500DD8A460499401A401C019037
:1085C0004FF000400290200704D40198504501DB91
:1085D000CDF8048000208DF84F0002980DF14F0770
:1085E000B0F1004F25D02B200E9002984FF00208DA
:1085F00000280CDA404202902D200E9007E00A215C
:108600000298F8F7EBF93031029007F8011DB8F144
:108610000001A8F10108F2DC02980028EFD1791ED0
:108620000E980870307800F0200040F0450007F800
:10863000020D12A8C01B00F107081498007800B1C1
:10864000012000EB0A01019801EBE071059841441B
:10865000401A401E0590E00306D45B462146179A57
:10866000059800F05DF805441498007818B15A4652
:10867000179990476D1CE00324D55B462146179A55
:10868000059800F04DF805441CE00498002807DB2D
:10869000DDE90301884203DD0098405C179901E0A1
:1086A000179930205A469047049805F10105401C5F
:1086B00004900198401E019004D12E205A4617992B
:1086C00090476D1CBAF10001AAF1010ADDDC05E05A
:1086D00017F8010B5A46179990476D1CB8F1000125
:1086E000A8F10108F4DC5B462146179A0598ABE631
:1086F0002D0000002B000000200000002DE9F041BB
:10870000044600251E461746880404D405E0394671
:108710002020B0476D1C641EF9D52846BDE8F081C5
:108720002DE9F041044600251E469046C80301D5B8
:10873000302700E02027880404D505E0414638466C
:10874000B0476D1C641EF9D52846BDE8F0810A6863
:10875000531C0B601070704770B506460D46242000
:10876000FFF764FB0446621D13A130460BF0A0FE28
:1087700015A130460BF087FEE07018A130460BF0D3
:1087800082FEA07019A130460BF07DFE60831CA113
:1087900030460BF078FE2080A869406810B9A869BF
:1087A000446008E0A969486800E0006A016A00299D
:1087B000FBD1046200BF70BD226964656E74696696
:1087C000696572223A220000227746756E637469E9
:1087D0006F6E436F6465223A0000000022736C6183
:1087E000766541646472657373223A00227265672C
:1087F000697374657241646472657373223A000030
:10880000227265676973746572427974654E756D1D
:10881000223A000070B5064635462020FFF706FBD9
:1088200004460020E06136A130460BF02CFE607556
:1088300036A130460BF027FEE07537A130460BF02D
:1088400022FEA075621C39A130460BF031FE0C20CF
:10885000FFF7ECFAA06139A12846F7F768FD054655
:1088600011E02146284600F047F900BF37A128460D
:10887000F7F75DFD0546412028706D1C28785D28BE
:1088800001D1354600E0ECE700BF607D032824D12C
:10889000354621A128460BF0F6FDA0751BA1284600
:1088A0000BF0F1FDE0752AA12846F7F740FD0546DB
:1088B0009DB110E021462846FFF74EFF23A1284630
:1088C000F7F735FD0546412028706D1C28785D2896
:1088D00001D1354600E0EDE700BF2148D0F8E800BF
:1088E00018B91F48C0F8E84009E01D49D1F8E80070
:1088F00000E0C069C1690029FBD1C46100BF70BD3F
:108900002270726F746F636F6C223A00226461741C
:108910006154797065223A00226269674C69747407
:108920006C65466F726D6174223A00002264657650
:108930006963654964223A22000000002273656E73
:10894000736F7244617461223A5B00007D00000025
:1089500022636F6D6D616E6444617461223A5B00E5
:10896000047A002070B5054633A128460BF08BFD34
:108970003349C88233A128460BF085FD304981F880
:10898000F20033A128460BF07EFD2D4981F8F0005E
:1089900032A128460BF077FD2949C1F8EC0032A13D
:1089A00028460BF070FD264981F8F10031A12846D8
:1089B0000BF069FD2249C1F8C4004A1C31A12846C8
:1089C0000BF076FD1E4AA43231A128460BF070FD53
:1089D0001B4A4A3232A128460BF06AFD184A183267
:1089E00034A128460BF064FD154A7C3236A1284696
:1089F0000BF05EFD124A903237A128460BF058FD6D
:108A000039A12846F7F793FC044611E07CB12046D3
:108A1000FFF700FF00BF37A12046F7F788FC0446A8
:108A200041202070641C20785D2801D101E070BDD8
:108A3000ECE700BF00BFFAE722706F7274223A00C1
:108A4000047A00202273746F70426974223A000025
:108A50002264617461426974223A00002262617585
:108A60006472617465223A0022636865636B4269CF
:108A700074223A0022696E626F756E6454696D6586
:108A8000223A000022686F7374223A22000000002C
:108A9000226465766963654964223A220000000019
:108AA00022636F6D6D616E64546F706963223A2248
:108AB00000000000226D657373616765546F706913
:108AC00063223A220000000022757365726E616DA8
:108AD00065223A22000000002270617373776F7282
:108AE00064223A22000000006465766963654C697F
:108AF000737400007D0000002DE9F84380460C46A9
:108B0000607D012804D0022803D003286ED13AE00A
:108B100000BF3020FFF78AF9054636A140460BF02A
:108B2000B2FCE861AA1D38A140460BF0C1FC0D2142
:108B300000200AF055FD07463A4637A140460BF0A3
:108B4000B7FC002609E007EB46006A4636A1F7F7B6
:108B50003BFC9DF80000A855761C062EF3DB394639
:108B600000200AF02BFDA069806810B9A06985601B
:108B700008E0A169886800E0C06AC16A0029FBD1E9
:108B8000C56200BF33E02820FFF750F90546AA1C54
:108B90001DA140460BF08CFC25A140460BF073FC58
:108BA00085F8200025A140460BF06DFC687028A1D7
:108BB00040460BF068FC287029A140460BF063FC8E
:108BC000E8822CA140460BF05EFCE883A0690068B7
:108BD00010B9A069056008E0A169086800E0406A72
:108BE000416A0029FBD1456200BF00E000BF00BF21
:108BF000BDE8F883226964656E74696669657236DA
:108C00003435223A00000000226964656E7469669A
:108C1000696572223A2200002264657669636549BB
:108C200044363435223A2200253268687800000044
:108C30002270726563697365223A0000227246757C
:108C40006E6374696F6E436F6465223A00000000C2
:108C500022736C61766541646472657373223A00B5
:108C600022726567697374657241646472657373B7
:108C7000223A0000227265676973746572427974E2
:108C8000654E756D223A00002DE9F04105460E460D
:108C9000002447E0F7F792FA074604EB4400244922
:108CA00051F83000C8BB04EB440041F8305038465E
:108CB000F7F788FA002004EB44011D4A02EBC101DA
:108CC000486004EB440102EBC101088104EB44015C
:108CD00002EBC10148812878102804D10EB101208F
:108CE00002E0002000E0012004EB4401104A02EB06
:108CF000C1018881002004EB440102EBC101C8815D
:108D000004EB440102EBC101086104EB440102EBF6
:108D1000C10148612046BDE8F081FFE73846F7F71A
:108D200051FA641C082CB5DB4FF0FF30F3E700006C
:108D3000A05B012010B5044600BF00BF04F022FA7A
:108D40000022034941F288300DF0D0F810BD000038
:108D5000358D00087047000010B50246002309E079
:108D6000064800680078107004480068401C034CF6
:108D700020605B1C8B42F3DB084610BDB001002075
:108D800070B504460D4600202071401EE062294661
:108D9000204609F02BFC08B1032070BD94F82E1278
:108DA00094F82F0241EA00204AF65521884201D06A
:108DB0000220F2E794F86900010694F8680041EA9D
:108DC000004194F8670041EA002094F866100843D7
:108DD00020F07F400D49884201D10020DDE794F862
:108DE0008500010694F8840041EA004194F883006C
:108DF00041EA002094F88210084320F07F400349A4
:108E0000884201D10020C8E70120C6E7464154004E
:108E1000024600E0521C107810B110788842F9D157
:108E20001078704730B502460B46002004460146D4
:108E300021E001EB41001D4D55F82000C8B101EBC8
:108E4000410055F820001568A84213D101EB4100FC
:108E5000164D05EB800040689568A8420AD101EBE9
:108E60004100124D05EB80000089D588A84201D150
:108E700003E00124491C0329DBD300BF032906D1E9
:108E80000CB9022B01D1002030BD1220FCE743B900
:108E900001EB4100054D05EB80004089B0F5807F76
:108EA00001D11020F0E70020EEE700000CE30020E5
:108EB00010B5014600200DE000EB4002074B53F8CF
:108EC00022208A4205D1002200EB4003034C44F8E3
:108ED0002320401C0328EFD310BD00000CE300202A
:108EE0000246891E5069801E884201D800207047C2
:108EF0009378906A01FB0300F9E700002DE9F04741
:108F000005460C46207820F04000401E00EB800112
:108F100001EBC00600274FF0010800BF1A48C05DF2
:108F2000205C1949C95D2144497840EA0129B8F11A
:108F3000000F10D0484605F0C5FA8046FF2E07D234
:108F40003146761C35F8110005F0BCFA404508D0D2
:108F50000020BDE8F0874FF6FF70814501D000206A
:108F6000F7E7781C07460D28D8D3207800F040009A
:108F700038B1B8F1000F04D035F8160008B1002060
:108F8000E7E70120E5E70000D45304082DE9F047A6
:108F900004468946B9F1000F06D1E76817B1606948
:108FA000B84215D8012713E04946204605F086FD52
:108FB0000646022E02D20120BDE8F087701C08B9D7
:108FC0003046F9E76069B04201D93046F4E74F46D0
:108FD0003D4600BF6D1C6069A84204D80225BD4211
:108FE00001D90020E8E72946204605F067FD06463E
:108FF00006B909E0701C08B1012E01D13046DBE74B
:10900000BD42E7D10020D7E700BF6FF0704229468C
:1090100020460CF073F98046B8F1000F08D1B9F181
:10902000000F05D02A46494620460CF067F98046D5
:10903000B8F1000F0BD1E5602069401C78B12069C0
:10904000401E2061607940F00100607107E0B8F1D6
:10905000010F02D14FF0FF3000E001200546284605
:10906000AAE700002DE9F34F83B081460498006819
:10907000019002E00198401C0190019800782F288F
:10908000F8D0019800785C28F4D0D9F820A0002509
:109090002F4600BF38467F1C01990C5C202C03DB57
:1090A0002F2C01D05C2C00D132E0FF2D03D3062001
:1090B00005B0BDE8F08FE4B2812C13DBE0B2FE28EE
:1090C00010DC38467F1C01990E5C402E01DB7E2EA1
:1090D00005DD802E01DBFE2E01DD0620E8E706EB34
:1090E000042084B20121204605F0AEF904460CB9F3
:1090F0000620DDE7802C06DA214671A0FFF788FE06
:1091000008B10620D4E728466D1C2AF81040C1E7B4
:1091100000BF0198C11904980160202C01DA0420D5
:1091200000E00020804608E0681E3AF81040202C3D
:1091300002D02E2C00D002E06D1E002DF4D100BF15
:109140000DB90620B4E700202AF815000B222021D3
:10915000D9F8180009F07EF8002700E07F1C3AF8E3
:1091600017002028FAD03AF817002E28F6D00FB1B1
:1091700048F0030800E06D1E25B1681E3AF81000A3
:109180002E28F8D10020064602904FF0080B00BFB1
:1091900038467F1C3AF8104004B963E0202C03D015
:1091A0002E2C04D1AF4202D048F00308F0E7029819
:1091B000584501D2AF4214D1BBF10B0F02D148F098
:1091C00003084FE0AF4201D048F00308AF4200D996
:1091D00048E02F46082002904FF00B0BB006060E19
:1091E000D6E7802C09DB204605F06CF900210090C1
:1091F00005F02AF9044648F00208FF2C11DDABF116
:1092000001000299884204D848F00308CDF808B05C
:10921000BEE72212D9F818300298411C02911A5464
:1092200019E024B1214629A0FFF7F2FD18B15F240F
:1092300048F003080FE0412C04DB5A2C02DC46F016
:10924000020608E0612C06DB7A2C04DC46F00106FD
:10925000A4F1200084B2D9F818300298411C029180
:109260001C5495E700BFD9F818000078E52803D111
:109270000520D9F818100870BBF1080F01D1B0060D
:10928000060E06F00C000C2803D006F0030003289D
:1092900001D148F0020808F0020058B906F00300B6
:1092A000012801D148F0100806F00C00042801D173
:1092B00048F00808D9F8180080F80B800020F7E67D
:1092C000222A3A3C3E3F7C7F000000002B2C3B3D95
:1092D0005B5D00002DE9F843054600BF012009F061
:1092E00071F94FF4105101200AF07AF9814649468C
:1092F00018A00CF0C9F94846FFF734FB4946012095
:109300000AF05CF905F052FC06464FF00008D6F86A
:10931000E8701BE000246A464FF47A711048006838
:10932000FCF7D2F9044624B94FF47A70FCF77EFEBC
:109330000BE0002021680AF041F9214600200AF0E4
:109340003DF94FF47A70FCF771FE00BF002FE1D1B8
:10935000BDE8F8836465766963652E7478740000EF
:109360001400002030B50246531E1A46032B1BD2B0
:1093700002EB42030D4C04EB83035989B1F5807F66
:1093800000D1002109B14B1E99B202EB4203074CF8
:1093900004EB8303598129B9002302EB4204034DF6
:1093A00045F82430002000E0022030BD0CE300200E
:1093B00010B56FF00400FDF785FF104800681049F4
:1093C000B0FBF1F00F4908700C4800680C49B0FB85
:1093D000F1F44FF47A70444301200B4908804FF0B8
:1093E000E020006940F002004FF0E02108610846EB
:1093F0004461006940F00100086110BD00000020D8
:1094000000127A00660000206800002070B5044653
:109410000D4600BF1CB90DA0FEF7E0FC70BD00BFFB
:1094200000BF00BF606A78B1606A007B08280BD17A
:1094300000BF00BF2868616A496A884204D100BF42
:1094400000BF204600F020FA00BFE7E76E657469B0
:109450006620213D204E554C4C0000007CB5064650
:1094600000BF1EB941A0FEF7B9FC7CBD00BF746A05
:1094700000BF1CB944A0FEF7B1FCF6E700BF00BF77
:1094800000BF606B401C90B100BF00BF606B1E301E
:109490003C21B0FBF1F5B5F5803F01D34FF6FF75E8
:1094A000A583A08B08B90120A08300BF00BFA06BDB
:1094B000401C90B100BF00BFA06B1E303C21B0FB30
:1094C000F1F5B5F5803F01D34FF6FF75E583E08BED
:1094D00008B90120E08300BF00BFA08BE18B884268
:1094E00004DBE08B002801DD0020A083A07B10B10D
:1094F000A06A019010E094F824007F2802DCFF218C
:10950000019108E0C02803DB6FF07F41019102E088
:109510004FF6FF71019100BFE06A0090684608B104
:10952000009838B9606A019908400090009840F0AE
:109530008070009000BF00BF04F1240130460AF0A3
:10954000FDFE00BF00BF01A930460AF079FF00BF51
:1095500000BF694630460AF0E8FE30460AF078FF60
:109560000A21204601F036F900BF7EE76468637087
:109570005F62696E643A206E6574696620213D20E1
:109580004E554C4C00000000646863705F62696E69
:10959000643A206468637020213D204E554C4C0095
:1095A0002DE9F0410646746A00BF00BF082120463D
:1095B00001F010F9002204F12401304603F010FC00
:1095C00005460DB100BF00BF607B401C60734FF4C7
:1095D000FA7707F2F310394690FBF1F0608300BF91
:1095E00000BFBDE8F081000010B51248046800BF5C
:1095F00000BF1BE0606AC0B1606AC18B481E626A2E
:10960000D083012905D100BF00BF204601F0E4F955
:109610000BE0606A818B481E626A9083012904D145
:1096200000BF00BF204601F0C3F92468002CE1D13F
:1096300010BD0000100100202DE9F04106460C4647
:10964000174600BF36B95AA0FEF7C8FB6FF00D00F1
:10965000BDE8F08100BF00BF2CB95DA0FEF7BEFBE6
:109660006FF00500F4E700BF00BF206910B160A0F3
:10967000FEF7B4FB00BF00BF606910B166A0FEF743
:10968000ADFB00BF00224FF49A7110460AF02AFF8A
:109690002061206920B900BF00BF4FF0FF30D7E73D
:1096A00000BF20694089B0F59A7F02D264A0FEF71E
:1096B00095FB00BF607B20B971480068401C704971
:1096C00008606F480068206000BF00BF20694068E4
:1096D00060610120616908706169487096F82A002C
:1096E0006169887000206169C870206807F062FEB7
:1096F0006169486000206169088161694881616928
:10970000C860082F09D0042F07D0032F08D1207B71
:10971000052802D0207B042802D170686169C860E6
:10972000002061690861616948616169886100259B
:109730000DE096F82A00A84203DD06F12B00405DFB
:1097400000E0002061691C314855681C85B2102D6D
:10975000EFD3002505E0002160692C304155681CDD
:1097600085B2402DF7D3002505E0002160696C30FB
:109770004155681C85B2802DF7D342486169C1F814
:10978000EC0000202083002504E06069F03045559E
:10979000681C85B2442DF8D301223521204600F003
:1097A00067FA3946204600F081FA002050E70000B1
:1097B000646863705F6372656174655F6D73673A57
:1097C000206E6574696620213D204E554C4C00008A
:1097D000646863705F6372656174655F6D73673A37
:1097E000206468637020213D204E554C4C000000E1
:1097F000646863705F6372656174655F6D73673A17
:1098000020646863702D3E705F6F7574203D3D204D
:109810004E554C4C00000000646863705F637265D5
:109820006174655F6D73673A20646863702D3E6D87
:1098300073675F6F7574203D3D204E554C4C0000A2
:10984000646863705F6372656174655F6D73673AC6
:1098500020636865636B2074686174206669727345
:109860007420706275662063616E20686F6C64207E
:1098700073747275637420646863705F6D736700DE
:10988000E8000020638253632DE9F84305466C6AC3
:10989000002600BF00BF0C21204600F09BFF0422E1
:1098A00021462846FFF7C8FE06460EBB0422322199
:1098B000204600F0DDF9606A07F0A3FD80464146CE
:1098C000204600F023FA204600F086FA228BF03280
:1098D00091B220690BF0DAFA009543230E4A216910
:1098E000606810F08BFD204600F018F800BF01E022
:1098F00000BF00BF607B401C607342F2107707F22C
:10990000F3104FF4FA7190FBF1F0608300BF00BFD9
:109910003046BDE8F8830000A055040810B50446A1
:1099200000BF1CB90EA0FEF759FA10BD00BF00BF62
:10993000206910B912A0FEF751FA00BF00BF60699C
:1099400010B919A0FEF74AFA00BF206910B12069CA
:109950000BF08CF900202061606100BFE5E700009A
:10996000646863705F64656C6574655F6D73673AA6
:10997000206468637020213D204E554C4C0000004F
:10998000646863705F64656C6574655F6D73673A86
:1099900020646863702D3E705F6F757420213D20D8
:1099A0004E554C4C00000000646863705F64656C49
:1099B0006574655F6D73673A20646863702D3E6DF2
:1099C00073675F6F757420213D204E554C4C00002D
:1099D000F8B505466C6A002600BF00BF0020606233
:1099E0000621204600F0F6FE012221462846FFF718
:1099F00023FE0646002E3AD100BF00BF02223921C5
:109A0000204600F035F9298D204600F0C9F90422DE
:109A10003721204600F02CF90121204600F046F9BC
:109A20000321204600F042F91C21204600F03EF9B7
:109A30000621204600F03AF9204600F0CDF900BF9B
:109A400000BF228BF03291B220690BF01FFA00BFE9
:109A500000BF00954323164A2169606810F0CEFCD0
:109A600000BF00BF2046FFF759FF00BF01E000BF65
:109A700000BF607B401C6073607B062803DA617B5B
:109A80000120884000E03C2000EB4001C1EBC01009
:109A90004FF6FF7101EAC00707F2F3104FF4FA71B5
:109AA00090FBF1F0608300BF00BF3046F8BD0000BE
:109AB000A055040810B5104804681AE0606AB8B1EF
:109AC000606A408B012805DD606A408B401E616A38
:109AD00048830DE0606A408B012809D1606A408BA1
:109AE000401E616A488300BF00BF204600F088FF27
:109AF0002468002CE2D110BD10010020F8B5064604
:109B0000746A0020A062E0622448C07810B1244842
:109B1000C06820632148007918B12148006960635A
:109B200002E0206B400860631C48407918B11C4873
:109B30004069A06301E0206BA063A06800696062D7
:109B40001648807938B11649886907F033FCA0625D
:109B50000120A07301E00020A0731048C07920B15B
:109B60000F49C86907F026FCE06200250EE005F108
:109B700008010B4A52F8210007F01CFC00906946CE
:109B8000284601F077FE681CC5B200BF05F1080049
:109B90000249085C08B1022DE9DBF8BD8CFB00200E
:109BA00064FB002070B50446656A00BF00BF204614
:109BB0000AF0A6FB094920460AF0C0FB07492046E7
:109BC0000AF0B3FB054920460AF03AFC0C2128466E
:109BD00000F000FE2046FFF7FBFE70BD9C55040818
:109BE00070B505466C6A00BF00BF0B48807878B13D
:109BF0000A49886807F0DEFB206200BF00BFA0684A
:109C00000069606200BF00BF284600F061FD01E00E
:109C100000BF00BF70BD00008CFB002064FB002073
:109C200070B505466C6A04B970BD207B042809D064
:109C300003DC98B1032812D107E0052803D00A28D5
:109C40000DD101E000BF00BF00BF28460AF058FB5D
:109C500000206073284600F093FB06E005E000203A
:109C600060732846FFF7B4FE00BF00BF00BFDBE70C
:109C700070B504460E46154600BF208B801C284454
:109C8000442802D90848FEF7A9F800BF218B481CD8
:109C900020836069F0304654218B481C2083606922
:109CA000F030455470BD00004C58040870B50446AF
:109CB0000D4600BF208B442802D305A0FEF78EF886
:109CC00000BF218B481C20836069F030455470BD73
:109CD000646863705F6F7074696F6E5F62797465DA
:109CE0003A20646863702D3E6F7074696F6E735FA5
:109CF0006F75745F6C656E203C20444843505F4F25
:109D00005054494F4E535F4C454E000070B50446C9
:109D10000D4600BF208B001D442802D910A0FEF77D
:109D20005DF800BF290E228B501C20836069F03043
:109D30008154C5F30741228B501C20836069F030A9
:109D40008154C5F30721228B501C20836069F030B9
:109D50008154228B501C20836069F030855470BD83
:109D6000646863705F6F7074696F6E5F6C6F6E674D
:109D70003A20646863702D3E6F7074696F6E735F14
:109D80006F75745F6C656E202B2034203C3D204441
:109D90004843505F4F5054494F4E535F4C454E001F
:109DA00070B504460D4600BF208B801C442802D9A4
:109DB0000848FEF713F800BF290A228B501C2083A5
:109DC0006069F0308154228B501C20836069F03030
:109DD000855470BD0858040810B5044600BF1CB96E
:109DE00017A0FDF7FBFF10BD00BF00BF606910B9F1
:109DF0001CA0FDF7F3FF00BF00BF208B442802D357
:109E000023A0FDF7EBFF00BFFF21228B501C208316
:109E10006069F030815406E00021228B501C2083C1
:109E20006069F0308154208B442803D3207E00F0F9
:109E3000030010B1208B4428EED300BFD3E700000D
:109E4000646863705F6F7074696F6E5F747261696C
:109E50006C65723A206468637020213D204E554C39
:109E60004C000000646863705F6F7074696F6E5FB0
:109E7000747261696C65723A20646863702D3E6D1E
:109E800073675F6F757420213D204E554C4C0A005E
:109E9000646863705F6F7074696F6E5F747261691C
:109EA0006C65723A20646863702D3E6F7074696FE0
:109EB0006E735F6F75745F6C656E203C2044484321
:109EC000505F4F5054494F4E535F4C454E0A00006F
:109ED0002DE9F34F89B089460020069005900A21AC
:109EE000DC48F6F70DFAB9F80A002C2804DA6FF00E
:109EF00001000BB0BDE8F08FD9F80410099881601B
:109F00004FF0F00BB9F80800079000BF4C460AE08C
:109F10006089ABEB00001FFA80FB61890798401A4B
:109F200080B20790246814B160895845F0DD14B9F7
:109F30006FF00100DDE75F46DDF81CA06068089067
:109F40004CE10898C05D049000264FF0FF38B81C23
:109F500080B203906189781C814203DD791C0898E6
:109F6000455C07E0206818B120684068007800E090
:109F7000002005462E460498342865D00BDC0328C3
:109F800025D003DC80B1012874D113E006282CD041
:109F90003328F9D14BE0352863D0362871D03A28E0
:109FA0007CD03B28F0D186E0002005460646781E8E
:109FB00087B291E000BF042D05D0A7A0FDF70EFFEA
:109FC0006FF0050095E700BF4FF0060884E0042617
:109FD00000BFB54205DAA3A0FDF700FF6FF0050052
:109FE00087E700BF4FF0070876E000BFE91705EBF1
:109FF00091718910A5EB810129B19FA0FDF7EEFEBB
:10A000006FF0050075E700BF082D01DA284600E073
:10A010000820064600BFB54205DA92A0FDF7DEFE35
:10A020006FF0050065E700BF4FF0080854E000BF7F
:10A03000042D05D088A0FDF7D1FE6FF0050058E78C
:10A0400000BF4FF0030847E000BF012D05D08EA0F0
:10A05000FDF7C4FE6FF005004BE700BF4FF00008AE
:10A060003AE000BF012D08D087A0FDF7B7FE6FF0E2
:10A0700005003EE72CE004E010E000BF4FF00108CF
:10A080002AE000BF042D05D073A0FDF7A7FE6FF0F6
:10A0900005002EE700BF4FF002081DE000BF042DB1
:10A0A00005D06DA0FDF79AFE6FF0050021E700BF17
:10A0B0004FF0040810E000BF042D05D066A0FDF7A6
:10A0C0008DFE6FF0050014E700BF4FF0050803E0B8
:10A0D000002600BF00BF00BF00BFA81C384487B2E5
:10A0E000002E5FDD0020029000BF00BFB8F1000F1E
:10A0F00002DBB8F10A0F02DB66A0FDF76FFE00BFBE
:10A10000544810F8080078BB042E01DA304600E00D
:10A110000420019002A92046039B019A0AF034FD15
:10A12000042E22DD00BFF11706EB91718910A6EB1A
:10A13000810129B15CA0FDF751FE6FF00500D8E662
:10A1400000BF0120434901F80800029807F032F9E6
:10A150005A4941F82800301FC6B20398001D80B24A
:10A16000039008F10108C0E71BE0042E04D1029817
:10A1700007F047F902900CE000BF012E05D050A077
:10A18000FDF72CFE6FF00500B3E600BF9DF8080058
:10A19000029001202F4901F808004849029841F82F
:10A1A000280000BF6089B84217DC6089381A87B27E
:10A1B0006089AAEB00001FFA80FA57450CDABAF161
:10A1C000000F09D0246800BF14B942A0FDF706FEB5
:10A1D00000BF6068089000E008E000BF34B1089854
:10A1E000C05DFF2802D05745FFF6ABAE00BF19484F
:10A1F0000078D0B1314908680021164A1170012851
:10A2000003D10121069100BF0EE0022803D10121F4
:10A21000059100BF08E0032804D1012105910691B2
:10A2200000BF01E000BF00BF00BF069830B10020B2
:10A2300006904FF06C0BEC20079067E6059830B164
:10A24000002005904FF02C0B6C2007905EE600205C
:10A250004FE600008CFB00206C656E203D3D2034F5
:10A26000000000006C656E203E3D206465636F64F5
:10A27000655F6C656E0000006C656E2025203420E3
:10A280003D3D2030000000006C656E203D3D2031DA
:10A2900000000000636865636B206465636F64653C
:10A2A0005F696478000000006465636F64655F6CDB
:10A2B000656E20252034203D3D20300064FB0020C9
:10A2C000696E76616C6964206465636F64655F6C58
:10A2D000656E00006E657874207062756620776127
:10A2E00073206E756C6C0000F8B505466C6A00BF93
:10A2F00000BF0421204600F06DFA032221462846C3
:10A30000FFF79AF90646EEB9022239212046FFF7F7
:10A31000AFFC298D2046FFF743FD2046FFF75CFD8B
:10A32000228BF03291B220690AF0B0FD00954323F0
:10A33000124A2169606810F061F82046FFF7EEFAD2
:10A3400000BF01E000BF00BF607B401C6073607B0A
:10A350000A2804DA607B4FF47A71484301E042F244
:10A36000107087B207F2F3104FF4FA7190FBF1F01E
:10A37000608300BF00BF3046F8BD0000A055040850
:10A380002DE9F84305466C6A00BF00BF0321204653
:10A3900000F020FA032221462846FFF74DF9064631
:10A3A0005EBB022239212046FFF762FC4FF4107198
:10A3B0002046FFF7F5FC042232212046FFF758FC27
:10A3C000606A07F01EF8804641462046FFF79EFC73
:10A3D0002046FFF701FD228BF03291B220690AF08E
:10A3E00055FD00954323134A2169606810F006F873
:10A3F0002046FFF793FA00BF01E000BF00BF607B7B
:10A40000401C6073607B0A2804DA607B4FF47A7129
:10A41000484301E042F2107087B207F2F3104FF4A4
:10A42000FA7190FBF1F0608300BF00BF3046BDE8D9
:10A43000F8830000A05504082DE9F05F8146154619
:10A44000DDF828B04F467C6AD5F804A000BF00BFF5
:10A4500000BF00BF00BF00BF00BFA06810B143A095
:10A46000FDF7BCFC00BF68892C2802DA00BF00BFE2
:10A4700075E09AF80000022802D000BF00BF6EE02D
:10A4800000260CE007F12B00815D0AF11C00805DC5
:10A49000814202D000BF00BF61E0701CC6B297F8D5
:10A4A0002A00B042EEDCDAF8040006F0AAFF2168C8
:10A4B000884202D000BF00BF51E029462046FFF786
:10A4C00007FD10B100BF00BF49E000BF00BF2C482E
:10A4D000407810B900BF00BF41E02A4890F80480DE
:10A4E000B8F1050F18D100BF00BF207B012806D1AD
:10A4F0003846FFF703FB3846FFF752F82EE0207B83
:10A50000032805D0207B042802D0207B052825D1F4
:10A510003846FEF7A3FF21E0B8F1060F11D1207BEA
:10A52000032808D0207B012805D0207B042802D0F6
:10A53000207B052805D100BF00BF3846FFF732FB5E
:10A540000CE0B8F1020F09D1207B062806D100BF2C
:10A5500000BF002060833846FFF742FB00BF0020A9
:10A56000A06028460AF082FBBDE8F09F7265706C1F
:10A5700079207761736E27742066726565640000C8
:10A580008CFB002064FB0020F8B505466C6A00BF18
:10A5900000BF0021204600F01DF90020206260620B
:10A5A000A062E062A0636063206307222146284620
:10A5B000FFF742F80646AEB92046FFF70DFC228BA6
:10A5C000F03291B220690AF061FC0095432304F156
:10A5D0002002216960680FF011FF2046FFF79EF905
:10A5E00000BF01E000BF00BF607B401C6073607B68
:10A5F0000A2804DA607B4FF47A71484301E042F2A2
:10A60000107087B207F2F3104FF4FA7190FBF1F07B
:10A61000608300BF00BF284609F072FE0649284645
:10A6200009F08CFE0449284609F07FFE02492846BD
:10A6300009F006FF3046F8BD9C550408F8B50546FC
:10A640006C6A00BF00BF0521204600F0C3F803225A
:10A6500021462846FEF7F0FF0646F6B902223921C8
:10A660002046FFF705FB298D2046FFF799FB204682
:10A67000FFF7B2FB228BF03291B220690AF006FCA0
:10A680000095432304F12002216960680FF0B6FEB3
:10A690002046FFF743F900BF01E000BF00BF607B29
:10A6A000401C6073607B0A2804DA607B4FF4FA6117
:10A6B000484301E044F6206087B207F2F3104FF4FC
:10A6C000FA7190FBF1F0608300BF00BF3046F8BD27
:10A6D0002DE9F84305466C6A00BF00BF0121204602
:10A6E00000F078F8032221462846FEF7A5FF06462B
:10A6F000002E4CD1022239212046FFF7B9FA298DCC
:10A700002046FFF74DFB042232212046FFF7B0FA26
:10A71000606A06F076FE804641462046FFF7F6FA6C
:10A72000042236212046FFF7A3FA206A06F069FECC
:10A73000804641462046FFF7E9FA042237212046A9
:10A74000FFF796FA01212046FFF7B0FA03212046D1
:10A75000FFF7ACFA1C212046FFF7A8FA0621204695
:10A76000FFF7A4FA2046FFF737FB228BF03291B2B5
:10A7700020690AF08BFB00954323154A2169606824
:10A780000FF03CFE2046FFF7C9F800BF01E000BF14
:10A7900000BF607B401C6073607B062803DA617B2E
:10A7A0000120884000E03C2000EB4001C1EBC010DC
:10A7B0004FF6FF7101EAC00707F2F3104FF4FA7188
:10A7C00090FBF1F0608300BF00BF3046BDE8F88326
:10A7D000A0550408027B8A4203D001730022427311
:10A7E0004283704770B50546002600BF2DB93FA0D3
:10A7F000FDF7F4FA6FF00D0070BD00BF6C6A00BF8A
:10A8000000BF15F8310F20F00800287015F8310945
:10A8100000F0200020B900BF00BF6FF00D00EBE793
:10A82000288DB0F5107F04DA00BF00BF4FF0FF3075
:10A83000E2E774B900BF00BF3C2007F007FC044604
:10A8400024B900BF00BF4FF0FF30D5E76C6200BFF6
:10A8500014E000BF00BF606810B160680FF088FDB1
:10A8600000BF206910B125A0FDF7B8FA00BF00BFF6
:10A87000A06810B127A0FDF7B1FA00BF3C21204627
:10A88000F5F73EFD0FF036FD6060606820B900BF4F
:10A8900000BF4FF0FF30AFE76068007A40F0200063
:10A8A000616808724422204960680FF07FFB4322F0
:10A8B0001D4960680FF0D2FB2A461C4960680FF002
:10A8C00053FD00BF00BF2846FFF782F806462EB1B1
:10A8D000284600F02DF84FF0FF308DE795F8310055
:10A8E00040F0080085F83100304685E76E657469F0
:10A8F0006620213D204E554C4C000000706275666C
:10A9000020705F6F7574207761736E277420667294
:10A91000656564007265706C79207761736E277469
:10A9200020667265656400009C55040839A400081F
:10A9300070B5054600BF1DB911A0FDF74FFA70BDF7
:10A9400000BF6C6A95F8310020F0080085F83100EE
:10A9500000BF00BF8CB1606820B160680FF008FDD7
:10A960000020606000BFA06810B10CA0FDF736FAAF
:10A9700000BF00212046FFF72DFF00BFDFE70000EA
:10A98000646863705F73746F703A206E6574696693
:10A9900020213D204E554C4C000000007265706C2B
:10A9A00079207761736E2774206672656564000094
:10A9B00070B505466C6A00BF00BF207B012805D03A
:10A9C000207B0A2802D0207B052804D100BF00BFCD
:10A9D0002846FFF733FE70BD70B505466C6A00BFB0
:10A9E00000BF207B012805D0207B0A2802D0207BD5
:10A9F000052804D100BF00BF2846FFF775FC70BDD5
:10AA000070B505466C6A00BF00BF207B0C2802D0E1
:10AA1000207B062805D100BF00BF2846FEF7D8FFDF
:10AA20004FE0207B012811D100BF00BF607B0528CB
:10AA300003DC2846FFF74CFE43E000BF00BF28467A
:10AA4000FFF7A2FD2846FEF7C3FF3AE0207B082867
:10AA50000CD100BF00BF607B012803DC2846FEF755
:10AA60009FFD2EE02846FEF7F9FC2AE0207B052812
:10AA700005D100BF00BF2846FFF7E0FD21E0207BA5
:10AA8000042811D100BF00BF607B082803DC2846E2
:10AA9000FFF72AFC15E000BF00BF2846FFF774FD52
:10AAA0002846FEF795FF0CE0207B032809D1607B48
:10AAB000022803DA2846FFF763FC02E02846FEF787
:10AAC00087FF70BD10B5044600BF00BFFEF78CFDC8
:10AAD000002203494EF660200BF008FA10BD00007A
:10AAE000C5AA000810B5044600BF00BFFEF7E2FF8C
:10AAF000002203494FF4FA700BF0F8F910BD000082
:10AB0000E5AA00082DE9F04104460E460021204642
:10AB100000F04FFA0546EDB9002700BF2169206813
:10AB200007F064FD054605B113E060690078E5288B
:10AB300002D06069007820B9781C0746B04201D184
:10AB400007E000270121204600F07FF80546002D90
:10AB5000E4D000BF042D00D107252846BDE8F081D0
:10AB60002DE9F04704460021204600F022FA07466E
:10AB700017B13846BDE8F0874FF0FF09CA464FF6D7
:10AB8000FF70A08400BF2169206807F02FFD0746F1
:10AB900007B157E065692E780EB9042752E0E87ACC
:10ABA00000F03F08E52E05D008F0080040B1B8F1EC
:10ABB0000F0F05D04FF0FF094FF6FF70A0843AE069
:10ABC000B8F10F0F1CD1206A78B306F0400030B105
:10ABD00095F80DA026F04006B146E088A0844E45C9
:10ABE0000AD1687B504507D12946206AFEF786F9CD
:10ABF00010B1A9F1010000E0FF2000F0FF091AE008
:10AC0000B9F1000F05D128460AF0D4FF504500D114
:10AC100018E0A069C07A00F0010038B90B2228467C
:10AC2000A16907F031F908B90CE004E04FF0FF0921
:10AC30004FF6FF70A0840021204600F006F807467A
:10AC4000002FA0D000BF384694E72DE9F04104461C
:10AC50008846E088461CB0B208B1206910B90420CB
:10AC6000BDE8F08106F00F0000286CD12069401C7F
:10AC70002061E06828B920680089B04263D80420C8
:10AC8000EEE720688078401E00EA161000285AD1AE
:10AC9000E168206803F012FF0546012D01D802206B
:10ACA000DEE7681C08B90120DAE720684069A8429D
:10ACB00043D8B8F1000F01D10420D1E7E168206842
:10ACC000FEF764F905460DB90720C9E7012D01D14A
:10ACD0000220C5E7681C08B90120C1E720680AF016
:10ACE000DDFF08B10120BBE7216801F130004FF41E
:10ACF0000072002107F0AEFA29462068FEF7F0F84E
:10AD00002168C86200270EE00120216808712068D0
:10AD10000AF0C4FF08B10120A2E72068C06A401C05
:10AD20002168C8627F1C20688078B842ECD820680F
:10AD3000C06AC01B2168C86200BFE5602946206860
:10AD4000FEF7CEF82061E6802068303006F00F0173
:10AD500000EB41106061002082E72DE9F05F0446BE
:10AD60008A464FF0FF09CB4604274EE02169206850
:10AD700007F03CFC074607B14AE0666935780DB933
:10AD8000042745E0F07A00F03F08E52D09D02E2D8C
:10AD900007D0B8F1080F01D1012000E00020504594
:10ADA00002D04FF0FF0929E0B8F10F0F1AD105F0DA
:10ADB000400030B196F80DB025F04005A946E08876
:10ADC000A0844D450AD1707B584507D13146206A91
:10ADD0000AF078F910B1A9F1010000E0FF2000F0BD
:10ADE000FF090BE0B9F1000F04D130460AF0E2FE92
:10ADF000584502D04FF6FF70A08409E0002120469C
:10AE0000FFF723FF074607B102E020690028ADD114
:10AE100000BF0FB1002020613846BDE8F09F2DE94A
:10AE2000FE4F0446D4F81880D4F820900C224146F6
:10AE3000684607F03CF800BF9DF80B0000F00100E9
:10AE400020B3002088F80B00206201260CE0334676
:10AE50004A466946404603F0CDFD2046FFF780FE96
:10AE6000054605B102E0761C642EF0D300BF642EC7
:10AE700002D10720BDE8FE8F042D01D02846F9E756
:10AE80009DF80B0088F80B00C4F820909DF80B008B
:10AE900000F0020060B1002600E0761C39F81600D0
:10AEA0000028FAD106F119000D21B0FBF1F700E0FE
:10AEB000012739462046FFF725FE054645BB781E8B
:10AEC000071E25D0E088C11B204600F072F8054619
:10AED000F5B9A0690AF06EFE824600BF21692068BC
:10AEE00007F084FB054605B111E0FAB253466169EB
:10AEF000206A03F0C9FC0120216808710021204666
:10AF0000FFF7A3FE054615B9781E071EE6D100BF60
:10AF1000C5B92169206807F069FB054695B920226B
:10AF20000021606907F096F90B22D4E9050106F0CB
:10AF3000BEFFA069C07A00F01800616908730120A3
:10AF400021680871284695E770B50446E688A08C0C
:10AF50004FF6FF72904201D1304600E0A08C0146CE
:10AF6000204600F026F805460DBB00BF2169206889
:10AF700007F03CFB054605B115E020220021606981
:10AF800007F068F9E52061690870012021680871FF
:10AF9000E088B04200D306E000212046FFF755FECE
:10AFA0000546002DE2D000BF042D00D10225284621
:10AFB00070BD2DE9F04104460E46E680A568012DDE
:10AFC00003D020684069A84202D80220BDE8F08181
:10AFD0002DB920680078032801D12068456A45B959
:10AFE00020680089B04201D80220EFE72068476A54
:10AFF0001EE0206880784FEA001812E02946206899
:10B0000003F05CFD0546681C08B90120DEE7022D4F
:10B0100003D320684069A84201D80220D6E7A6EBF6
:10B0200008064645EAD229462068FDF759FF07463B
:10B03000E5600FB90220C9E707EB16102061206810
:10B04000303006F00F0100EB411060610020BDE7D9
:10B050000146012009B9002000E000BF00BF704791
:10B060002DE9F04105460E4614460427F5B901279F
:10B0700036B1012E06D0022E0AD0032E12D10CE0DA
:10B08000002711E0F9F73EFD400A206000270BE0A1
:10B090004FF400702080002706E04FF4007020601D
:10B0A000002701E0042700BF00BF01E0042700BF24
:10B0B00000BF3846BDE8F0812DE9F04104460D4659
:10B0C00016461F464FF000085CB93B464FF400722D
:10B0D00031462846F9F7A6FD00B901E04FF0010816
:10B0E00002E04FF0040800BF00BF4046BDE8F08119
:10B0F0000146012009B9002000E000BF00BF7047F1
:10B100002DE9F04104460D4616461F464FF0000853
:10B1100084B93B464FF4007231462846F9F7EAFD00
:10B1200000B906E03A46314606A0FCF757FE4FF05C
:10B13000010802E04FF0040800BF00BF4046BDE830
:10B14000F08100004E414E445F57726974654D7541
:10B150006C7469536563746F727328292045727229
:10B160006F722120736563746F72203D2025642CFB
:10B1700020636F756E74203D202564200D0A000049
:10B1800010B5002404E0204600F006F8601CC4B2AC
:10B19000042CF8DB10BD000070B50646C6EBC600F7
:10B1A00000EB80003E4901EBC00400BF042E02DB2F
:10B1B0003CA0FCF713FE00BF2078002866D00128D1
:10B1C00004D0022815D0032861D154E00220207059
:10B1D000002060700120A0700020E070607832468E
:10B1E00004F10C0100F08AFA05460DB100BF00BF62
:10B1F00053E0A078401EC0B2A07000283AD1E07899
:10B20000401CC0B2E070042828D16078401C02289D
:10B2100012DA6078401C2A4901EB800060B1607846
:10B22000401C51F8200038B16078401C607001204B
:10B23000A0700020E07030E000BF00BFD4F8100123
:10B2400038B1002104F10C00D4F81031D4F81421E5
:10B25000984700202070C4F810011EE0E078A0702C
:10B260006078324604F10C0100F048FA05460DB151
:10B2700000BF00BF11E0A068401EA06028B900BF59
:10B2800000BF00202070C4F8100106E005E000BFF8
:10B290000CA0FCF7A3FD00BF00BF00BF70BD000005
:10B2A00098FB0020617272617920696E6465782074
:10B2B0006F7574206F6620626F756E647300000096
:10B2C000F4000020756E6B6E6F776E20646E735F96
:10B2D0007461626C6520656E747279207374617438
:10B2E000653A000010B5024600BF11F8013B03F0BB
:10B2F000C000C02800D110E009E010780C78A0420E
:10B3000001D0012010BD491C521C581EC3B2002B95
:10B31000F3DC521C08780028E7D100BF0020F1E7D9
:10B320002DE9F05F07468846914600240020064636
:10B33000834600251BE0C5EBC50000EB80003149CA
:10B3400001EBC004207800B913E0207803280CD169
:10B3500020792D490978081A584506DD20792A49AF
:10B360000978081A00F0FF0B2E46681CC5B2042DA0
:10B37000E1DB00BF042D18D1042E08DAC6EBC600AD
:10B3800000EB80001F4911F83000032805D000BFF2
:10B3900000BF4FF0FF30BDE8F09F3546C5EBC5005C
:10B3A00000EB8000174901EBC00400BF00BF012083
:10B3B000207015480078207113480078401C12490D
:10B3C0000870C4F81081C4F814913846F4F7C1FF2E
:10B3D000FF2803D23846F4F7BCFF00E0FF20824686
:10B3E0005246394604F10C00F4F771FF002104F1D4
:10B3F0000C0000F80A102846FFF7CEFE6FF004009C
:10B40000C9E7000098FB0020F00000202DE9F04182
:10B4100005460E46174698461248006840B13EB1B0
:10B4200035B1287820B12846F4F793FFFF2803D9D7
:10B430006FF00D00BDE8F081284605F091F9044653
:10B44000601C18B9284600F04BF80446601C10B187
:10B4500034600020EEE7424639462846FFF760FF99
:10B46000E8E70000EC00002008B5144820F00300D5
:10B470001349086013A005F073F9009000BF00BFE6
:10B4800014480068C0B90EF035FF1249086008463C
:10B49000006888B100BF00BF00220F490D48006856
:10B4A0000EF084FD00220D490A4800680EF05CFF92
:10B4B0006946002000F0DEF908BD0000FBFF002017
:10B4C000FC0000203230382E36372E3232322E3207
:10B4D00032320000EC0000209C55040875B50008CD
:10B4E00070B50546002427E0C4EBC40000EB8000E3
:10B4F000144911F8300003281CD1C4EBC40000EB40
:10B5000080000A4602EBC00000F10C012846F4F767
:10B5100027FF78B900BF00BF00BF00BF00BF00BF5A
:10B52000C4EBC40000EB8000064901EBC000D0F87A
:10B530000C0170BD601CC4B2042CD5DB4FF0FF3091
:10B54000F7E7000098FB0020014600BF11F8012B2F
:10B5500002F0C000C02800D108E002E0491C501EE3
:10B56000C2B2002AFADC08780028EFD100BF481CDC
:10B57000704700002DE9FE4F1546DDF830B02889F0
:10B58000B0F5007F02DD00BF00BFACE028891A28BB
:10B5900002DA00BF00BFA6E02A89002354480168F0
:10B5A000284609F0F1FA2989884279D1504806687D
:10B5B000308805F00CFF8046B8F1040F70DAC8EB54
:10B5C000C80000EB80004B4901EBC0042078022842
:10B5D00078D103202070F07800F00F006071B088FF
:10B5E00005F0F5FE8246F08805F0F1FE8146B07860
:10B5F00000F0800020B1607910B9BAF1010F02D0DB
:10B6000000BF00BF5FE03A4801680C3104F10C0054
:10B61000FFF768FE10B100BF00BF54E03448006877
:10B620000C30FFF791FF071D46E03846FFF78CFF0F
:10B63000074638680090786801903889ADF80800AE
:10B64000BDF80000B0F5807F2BD1BDF80200B0F549
:10B65000807F26D1BDF80800B0F5806F21D1019818
:10B6600005F0CFFEA0602449A068884201D90846B1
:10B67000A060D7F80A10C4F80C1100BF00BF00BFCB
:10B6800000BF00BF00BFD4F8100140B104F58671BF
:10B6900004F10C00D4F81031D4F81421984722E0BA
:10B6A00010E0BDF8080005F092FE07F10A01471806
:10B6B000A9F101001FFA80F9B9F1000FB5DC00BF54
:10B6C00000BF00E00FE0D4F8100138B1002104F110
:10B6D0000C00D4F81031D4F81421984700202070C1
:10B6E000C4F8100100BF284609F0C0FABDE8FE8F7B
:10B6F000FC00002098FB0020803A09002DE9F74F5C
:10B7000082B00746894600BF00BF00BF022F02DBA0
:10B7100040A0FCF763FB00BF00BF444800EB87007C
:10B7200018B1424850F8270010B941A0FCF756FB69
:10B7300000BF00224FF48871104608F0D3FE054682
:10B74000002D60D000BF286810B142A0FCF746FB76
:10B7500000BFD5F804800020C8F80000C8F8040035
:10B76000C8F80800049805F032FEA8F8000001208F
:10B7700088F802000002A8F8040008F10C044E4604
:10B78000761E00BF761CA346641C0020009007E0D4
:10B7900030782070641C0098401CC0B20090761C69
:10B7A00030782E2802D030780028F1D100988BF81C
:10B7B000000030780028E5D104F8010B4FF48070C8
:10B7C000ADF80400ADF8060001982060AA88201D9D
:10B7D000801A81B2284609F059FB144800EB870112
:10B7E0003522234800680EF039FC104800EB870230
:10B7F000352329461E4800680EF0E4FD824628469F
:10B8000009F034FA01E04FF0FF3A504605B0BDE8C8
:10B81000F08F0000646E7320736572766572206F1E
:10B820007574206F6620617272617900F4000020E7
:10B83000646E732073657276657220686173206E22
:10B840006F2049502061646472657373207365745E
:10B850000000000070627566206D7573742062656B
:10B8600020696E206F6E6520706965636500000059
:10B87000EC00002002280ADA054A12683AB131B118
:10B8800029B10A681AB1034A0B6842F820307047A0
:10B89000EC000020F400002010B5044600BF00BFFB
:10B8A00000F00AF8002203494FF47A700AF01EFBF8
:10B8B00010BD000099B8000810B50448006818B120
:10B8C00000BF00BFFFF75CFC10BD0000EC000020D3
:10B8D00010B504462068407878B120684078022886
:10B8E0000BD000BF20680078102802D01FA0FCF702
:10B8F00075FA00BFFB20207130E02068406858B323
:10B9000020680078102827D1207A032806D02068E4
:10B910004078022802D1F32020711FE0207A00F045
:10B92000010010B1206808F007F800BF2068D0F8C7
:10B930002C0118B92068D0F8280110B113A0FCF729
:10B940004DFA00BF0420216848702068C0F82C41DF
:10B95000206800F029F810BDFA202071216801F15B
:10B960000C000AF09AFA00BFF5E700006D73672D2E
:10B970003E636F6E6E2D3E74797065203D3D204EA6
:10B980004554434F4E4E5F5443500000616C726506
:10B990006164792077726974696E67206F722063C1
:10B9A0006C6F73696E6700002DE9F047044600BFB5
:10B9B00014B95BA0FCF712FA00BF00BF2078102872
:10B9C00002D05BA0FCF70AFA00BF00BF6078042831
:10B9D00002D05FA0FCF702FA00BF00BF606810B998
:10B9E00064A0FCF7FBF900BF00BFD4F82C0110B92C
:10B9F00065A0FCF7F3F900BFD4F82C01067A06F035
:10BA0000010706F00208032E01D1012000E000200A
:10BA10008146B9F1000F03D0002160680AF066FC8E
:10BA20006068007E012804D1002160680AF0F5FBFF
:10BA30001BE03FB1002160680CF022FF002160682C
:10BA40000AF0EBFBB8F1000F03D0002160680DF0A5
:10BA5000F9F8B9F1000F08D00422002160680BF05A
:10BA600081FF002160680AF091FFB9F1000F04D056
:10BA700060680AF03DFC054605E0424639466068CC
:10BA80000DF002F9054675BB0020D4F82C110871A1
:10BA9000C4F82C016070B9F1000F09D06060D4F8CF
:10BAA000300128B1002204212046D4F830319847D3
:10BAB00047B1D4F8300128B1002211462046D4F80D
:10BAC00030319847B8F1000F08D0D4F8300128B1D0
:10BAD000002202212046D4F83031984704F10C00AE
:10BAE0000AF0DBF91AE0FFE700BF6068007E01287A
:10BAF00002D12CA0FCF772F900BF334960680DF049
:10BB0000A1F80422314960680BF02CFF30496068CD
:10BB10000AF03CFF214660680AF0E8FBBDE8F087C8
:10BB2000696E76616C696420636F6E6E0000000060
:10BB30007468697320697320666F72207463702063
:10BB40006E6574636F6E6E73206F6E6C79000000AB
:10BB5000636F6E6E206D75737420626520696E2050
:10BB60007374617465204E4554434F4E4E5F434C91
:10BB70004F53450070636220616C72656164792087
:10BB8000636C6F7365640000636F6E6E2D3E63754A
:10BB90007272656E745F6D736720213D204E554C47
:10BBA0004C000000436C6F73696E672061206C6904
:10BBB0007374656E20706362206D6179206E6F749E
:10BBC000206661696C210000DD5A01087552010888
:10BBD00001C5000810B504462068406810B9F4207B
:10BBE00020715CE02068007800F0F000102812D08E
:10BBF000202808D0402847D12268A168506809F061
:10BC000018FC20714AE0A2892368A16858680EF0E8
:10BC100025FA207142E02068407810B1F7202071A9
:10BC200031E0206809F09CFFA2892368A168586868
:10BC30001E4B0AF065FC2071207920BB216891F829
:10BC40002411C1F3400003212268517000BF40B1AC
:10BC5000216891F8241141F00401226882F824112E
:10BC600007E0216891F8241121F00401226882F88C
:10BC7000241100BF10B1FB21217103E02168C1F83C
:10BC80002C4110BD00BF09E000BF09A0FCF7A6F8D9
:10BC900000BFFA20207100BF00BF00BF00BF2168B5
:10BCA00001F10C000AF0F9F800BFEAE7C9BC00088E
:10BCB000496E76616C6964206E6574636F6E6E2088
:10BCC00074797065000000002DE9F047054689464B
:10BCD00016462C461CB96FF00500BDE8F08700BF82
:10BCE0006078032802D027A0FCF778F800BF00BFD7
:10BCF000D4F82C0138B994F8240100F0040010B9EC
:10BD000028A0FCF76BF800BFD4F82C0110B1D4F8D0
:10BD10002C0106712078102803D116B9204609F0AD
:10BD20001FFF94F82401012121EA900700BF94F835
:10BD3000240120F0040084F8240100BF0020C4F88E
:10BD40002C01607077B900BFF4F738FA804694F997
:10BD5000080010F1090F01DB002020724046F4F7C3
:10BD600031FA00BFD4F8300128B100220221204668
:10BD7000D4F8303198471FB104F10C000AF08DF867
:10BD80000020AAE7636F6E6E2D3E737461746520A8
:10BD90003D3D204E4554434F4E4E5F434F4E4E4522
:10BDA0004354000028636F6E6E2D3E63757272659A
:10BDB0006E745F6D736720213D204E554C4C2920D9
:10BDC0007C7C20636F6E6E2D3E696E5F6E6F6E5F62
:10BDD000626C6F636B696E675F636F6E6E656374D1
:10BDE0000000000010B504462068407898B1206833
:10BDF000407802280FD02068407803280BD000BF7D
:10BE000020680078102802D039A0FBF7E7FF00BFB8
:10BE1000FB2020715FE000BF20684078032808D134
:10BE2000206890F8240100F0040010B938A0FBF756
:10BE3000D5FF00BF206807F07FFD2068406800281C
:10BE400035D02068007800F0F000102811D02028AC
:10BE500006D0402826D12168486809F04BFB22E033
:10BE6000002021684968C861216848680EF080FA9E
:10BE700019E000BF2068D0F82C0118B92068D0F86C
:10BE8000280110B12AA0FBF7A9FF00BF04202168F8
:10BE90004870032020722068C0F82C412068FFF70A
:10BEA00083FD10BD00BF00BF0020216848602068EE
:10BEB000D0F8300128B1206800221146D0F8303186
:10BEC00098472068D0F8300128B12068002202216C
:10BED000D0F830319847216801F10C0009F0E3FFF8
:10BEE00020B1216801F10C0009F0D7FF00BFD8E7AD
:10BEF0006D73672D3E636F6E6E2D3E747970652095
:10BF00003D3D204E4554434F4E4E5F54435000003C
:10BF1000626C6F636B696E6720636F6E6E656374CE
:10BF200020696E2070726F67726573730000000085
:10BF3000616C72656164792077726974696E6720DB
:10BF40006F7220636C6F73696E67000010B50446F2
:10BF50002068007800F0F000202806D121684868A9
:10BF60000EF0B0F80020207101E0FA202071216865
:10BF700001F10C0009F091FF10BD000010B504465E
:10BF80002068406800284DD0207C28B12168A06836
:10BF900049680968016004E02168A0684968496847
:10BFA0000160002020712068007800F0F000102867
:10BFB00025D020280CD040282DD1207C28B1206805
:10BFC0004068017CE068018001E0F320207128E0F6
:10BFD000207C28B120684068418AE06801800DE03B
:10BFE00020684068007C00F0040010B9F320207144
:10BFF00004E020684068818AE068018011E0207CCC
:10C0000018B120684068408B02E020684068808B4F
:10C01000E168088005E000BF06A0FBF7DFFE00BF77
:10C0200000BF01E0F3202071216801F10C0009F04C
:10C0300034FF10BD696E76616C6964206E6574634F
:10C040006F6E6E5F747970650000000010B5044675
:10C05000002020712068406810B9204608F0C0FF19
:10C06000216801F10C0009F018FF10BD70B50446FD
:10C070000020207120684068B0B120680078102846
:10C0800012D1A56800BFB5F5803F02D34FF6FF700F
:10C0900000E0A8B206462168486831460CF02AFC48
:10C0A000AD1B002DEFD100BF216801F10C0009F09C
:10C0B000F4FE70BD70B50446206890F9080010F1D8
:10C0C000090F03DA2068007A207140E0F320207124
:10C0D0002068406800283AD02068007800F0F0001E
:10C0E000202819D0402830D1A068083010B1A068AD
:10C0F000806838B9A26811682268506809F01AFA95
:10C10000207108E0A36803F10802196823685868E1
:10C1100009F01AFA207119E0A068083010B1A0687F
:10C12000806838B9A2681168226850680EF040F93A
:10C13000207109E0A568AB8905F108022968256826
:10C1400068680EF03FF9207100E000BF00BF216871
:10C1500001F10C0009F0A1FE70BD000010B504460D
:10C16000206890F9080010F1090F03DA2068007ABE
:10C17000207133E02068007810282DD120684078A5
:10C1800010B1FB20207129E02068406808B301202D
:10C190002168487000BF2068D0F82C0118B92068C9
:10C1A000D0F8280110B111A0FBF718FE00BF00BFA6
:10C1B000E06810B914A0FBF711FE00BF2068C0F8BA
:10C1C0002C4100202168C1F82801206800F026F8E1
:10C1D00010BDF320207101E0FA202071216801F1E7
:10C1E0000C0009F05AFE00BFF2E70000616C7265B6
:10C1F0006164792077726974696E67206F72206359
:10C200006C6F73696E6700006D73672D3E6D7367A9
:10C210002E772E6C656E20213D2030002DE9F84FE1
:10C2200004460020009094F8240100F0020028B990
:10C23000D4F82C01007C00F0040008B1012000E0DB
:10C2400000200746D4F82C0190F8108000BF14B9E4
:10C2500073A0FBF7C3FD00BF00BF6078012802D0C8
:10C2600073A0FBF7BBFD00BF00BFD4F82C0110B9D1
:10C2700077A0FBF7B3FD00BF00BF606810B97BA0DB
:10C28000FBF7ACFD00BF00BFD4F82811D4F82C0197
:10C29000C068814202D37BA0FBF7A0FD00BFD4F8A9
:10C2A0001C01E0B109F0DAFDD4F82C114969401AFB
:10C2B000D4F81C11884212DB01200090D4F8280128
:10C2C00030B96FF006050021D4F82C01C16097E069
:10C2D0000025D4F82811D4F82C01C16090E0D4F8DE
:10C2E0002C018068D4F8281100EB010BD4F82C0144
:10C2F000C068D4F82811A0EB010ABAF5803F04D336
:10C300004FF6FF7648F0020801E01FFA8AF66068EF
:10C31000B0F86690B14507DA4E461FB126B96FF006
:10C32000060519E048F0020800BFD4F82801811979
:10C33000D4F82C01C068814202D95FA0FBF74EFD02
:10C3400000BF43463246594660680DF01FF8054667
:10C350000DB1681C58BB00BFA7B1D4F82C01C06850
:10C36000B0420FD9D4F8300128B13246032120461B
:10C37000D4F83031984794F8240140F0100084F844
:10C38000240114E06068B0F8660040F66931884224
:10C3900004DD6068B0F86800082808DBD4F83001D4
:10C3A00028B1324603212046D4F830319847D5B918
:10C3B000D4F828013044C4F82801D4F82811D4F85E
:10C3C0002C01C068814200D04FB1D4F82811D4F8B4
:10C3D0002C01C160012000900020C4F82801606891
:10C3E0000AF09EFF0CE0681C20B91FB960680AF0D3
:10C3F00097FF05E0012000900021D4F82C01C160D6
:10C40000009850B1D4F82C0105710020C4F82C011B
:10C41000607004F10C0009F040FD0020BDE8F88FC9
:10C42000636F6E6E20213D204E554C4C0000000085
:10C43000636F6E6E2D3E7374617465203D3D204EBA
:10C440004554434F4E4E5F5752495445000000003B
:10C45000636F6E6E2D3E63757272656E745F6D7381
:10C460006720213D204E554C4C000000636F6E6EDE
:10C470002D3E7063622E74637020213D204E554C1A
:10C480004C000000636F6E6E2D3E77726974655FBD
:10C490006F6666736574203C20636F6E6E2D3E631D
:10C4A000757272656E745F6D73672D3E6D73672E66
:10C4B000772E6C656E000000646F5F77726974653B
:10C4C0006D6F72653A20696E76616C6964206C6587
:10C4D0006E67746821000000002100E0491C0329F8
:10C4E00006D201EB4100054A52F820000028F5D1A0
:10C4F000032901D0012070470020FCE70CE3002055
:10C500002DE9F04707460E463C4600BF14B938A057
:10C51000FBF764FC00BF00206060F3F74FFE81462C
:10C5200026724846F3F74EFE657800206070D4F816
:10C53000300128B1002204212046D4F83031984738
:10C54000D4F8300128B1002211462046D4F8303109
:10C550009847D4F8300128B1002202212046D4F8AF
:10C560003031984704F1100009F071FC20B100212E
:10C5700004F1100009F05EFC04F1940009F067FC7E
:10C5800020B1002104F1940009F054FC012D03D0E6
:10C59000042D01D0032D21D194F82401C0F380088B
:10C5A00000BF94F8240120F0040084F8240100BFA7
:10C5B000B8F1000F11D100BFD4F82C0110B910A0B0
:10C5C000FBF70CFC00BFD4F82C0106710020C4F866
:10C5D0002C0104F10C0009F060FC07E000BFD4F866
:10C5E0002C0110B10DA0FBF7F9FB00BFBDE8F087EF
:10C5F000636F6E6E20213D204E554C4C00000000B4
:10C60000636F6E6E2D3E63757272656E745F6D73CF
:10C610006720213D204E554C4C000000636F6E6E2C
:10C620002D3E63757272656E745F6D7367203D3D5C
:10C63000204E554C4C000000F8B5064600200090F6
:10C6400096F83100C0F3001000284FD02CA0FBF763
:10C65000C5FB2F480068002842D0002000904FF40E
:10C66000805200210120F6F7ADFA00BF0098401C6F
:10C67000009001210846F6F7C7F900F0200018B92C
:10C68000244900988842F1D310210120F6F7BCF923
:10C69000044604F0040020B14FF400601C49086215
:10C6A00002E000201A49086204F0020018B10020DC
:10C6B0001749486103E04FF4804015494861164826
:10C6C0000568134840691249096A0843054312483E
:10C6D00005604FF6FF70F5F702FA0F480568056030
:10C6E000F6F7F6F90D4807F0B3FE07E00CA0FBF7EC
:10C6F00075FBF6F7FDF9094807F002FEF8BD0000EA
:10C700006E6574776F726B2069732075700000001E
:10C71000B4D90020FFFF0400008002407CD9002033
:10C720006E6574776F726B20697320646F776E002B
:10C730002DE9FC4705468846164600BF25B94EA0A0
:10C74000FBF74CFBBDE8FC8700BF70892A2805DA9F
:10C7500000BF00BF304608F089FAF3E7776807F1B9
:10C760000E042088B0F5807F08D12079062805D1F5
:10C770006079042802D16088082805D000BF00BF76
:10C78000304608F073FADDE7D4F80E000190A06996
:10C790000090281D08B1686810B94FF0000907E043
:10C7A00000986968884201D1012000E0002081469C
:10C7B000B9F1000F01D0012000E00220034604F18E
:10C7C000080201A9284600F027FDE088B0F5807F27
:10C7D00003D0B0F5007F45D13DE000BF00BFB9F107
:10C7E000000F2FD000BF00BF022004F0F0FDE0805A
:10C7F000D4F80E00A0616868C4F80E0000BF95F878
:10C800002A00062802D02048FBF7E8FA00BFA068FB
:10C81000C4F81200A089E082A0683860A089B880BE
:10C82000D8F80000A060B8F80400A081D8F8000093
:10C83000C7F80600B8F80400788131462846AA698E
:10C84000904707E0281D08B1686808B900BF01E0FB
:10C8500000BF00BF09E000BF00BF01A92846FCF7E8
:10C86000D5FD02E000BF00BF00BF00BF304608F0AA
:10C87000FDF900BF66E700006E6574696620213D22
:10C88000204E554C4C0000006459040870B5054614
:10C89000002412E004EB8400094901EB8000867C4F
:10C8A0004EB104EB840001EB80008068A84202D105
:10C8B000204600F037F9601CC4B20A2CEADB70BDD8
:10C8C000E46C01202DE9FE4F064688464FF00A0928
:10C8D000CA460A270024002002900190BB4600901F
:10C8E00000BF69E004EB8400674901EB8000857CB0
:10C8F0000A2F04D11DB900BF00BF67B25AE0002D56
:10C9000058D000BF012D04D0022D02DA5FA0FBF742
:10C9100065FA00BF6EB104EB84015B4A02EB810152
:10C9200030684968884204D100BF00BF60B2BDE8EA
:10C93000FE8F012D2AD104EB8400534951F82000C9
:10C9400088B104EB840001EB8000C17C0098814237
:10C9500030DB4FFA84FB04EB84004B4901EB800091
:10C96000C07C009026E004EB8400474901EB800086
:10C97000C17C029881421DDB4FFA84F904EB8400EC
:10C98000414901EB8000C07C029013E0022D11DBD5
:10C9900004EB84003C4901EB8000C17C019881429A
:10C9A00008DB4FFA84FA04EB8400374901EB80007E
:10C9B000C07C0190601CC4B20A2C93DB08F002001A
:10C9C00020B90A2F07D108F0010020B900BF00BF2D
:10C9D0004FF0FF30ABE70A2F02DAFCB200BF2EE0C7
:10C9E000BAF10A0F0EDA0AF0FF0400BF00BF00BF61
:10C9F00004EB8400244951F8200010B133A0FBF768
:10CA0000EDF912E0B9F10A0F03DA09F0FF0400BFF3
:10CA10000BE0BBF10A0F03DA0BF0FF0400BF04E0E8
:10CA200000BF00BF4FF0FF3081E700BF0A2C02DBE0
:10CA30002CA0FBF7D3F900BF204600F073F800BF2D
:10CA40000A2C02DB27A0FBF7C9F900BF00BF04EBEB
:10CA500084000D4901EB8000807C10B126A0FBF71B
:10CA6000BDF900BF36B104EB8401074A02EB810136
:10CA700030684860002004EB8401034A02EB810126
:10CA8000C87460B253E70000E46C012073746174F1
:10CA900065203D3D204554484152505F5354415418
:10CAA000455F50454E44494E47207C7C207374615D
:10CAB0007465203E3D204554484152505F535441D7
:10CAC00054455F535441424C450000006172705F11
:10CAD0007461626C655B695D2E71203D3D204E5531
:10CAE0004C4C000069203C204152505F5441424C64
:10CAF000455F53495A4500006172705F7461626C12
:10CB0000655B695D2E7374617465203D3D204554FD
:10CB1000484152505F53544154455F454D5054591C
:10CB20000000000010B5044604EB8400194951F8D8
:10CB3000200070B100BF00BF04EB8401154A52F819
:10CB4000210008F093F8002004EB8401114A42F818
:10CB50002100002004EB84010E4A02EB810188745D
:10CB600004EB840102EB8101C87404EB840102EB45
:10CB70008101886004EB840102EB8101486004EBD1
:10CB80008400114601EB800003490A68C26089886D
:10CB9000018210BDE46C0120EA5504082DE9FC4730
:10CBA00004460F461546A94600BF14B951A0FBF72D
:10CBB00015F900BF00BF17B952A0FBF70FF900BF6E
:10CBC00000BF15B952A0FBF709F900BF0E21384686
:10CBD00008F0ECF828B100BF00BF6FF00100BDE81D
:10CBE000FC872146286802F041FF10B1DFF8308150
:10CBF00077E0287800F0F000E02815D101208DF8CA
:10CC0000000000208DF801005E208DF80200687899
:10CC100000F07F008DF80300A8788DF80400E87814
:10CC20008DF80500E8465BE02868A1680840D4E973
:10CC300001121140884210D0288880B24FF6A961B5
:10CC400088420AD004F10C0020B1E06810B104F170
:10CC50000C0902E06FF00300C1E73248007800EBF6
:10CC60008000314901EB8000807C022812DB2D49D5
:10CC7000097801EB81012C4A02EB8101D9F800000F
:10CC80004968884206D1274802783946204600F094
:10CC90004DF8A4E700261BE006EB8600224901EBD5
:10CCA0008000807C022811DB06EB86011E4A02EB25
:10CCB0008101D9F800004968884207D119490E70EE
:10CCC000F2B23946204600F031F888E7701C46B2CF
:10CCD0000A2EE1DB3A464946204600F081F87EE71D
:10CCE00000BF434604F12B023946204600F022FAE9
:10CCF00075E700006E6574696620213D204E554C35
:10CD00004C0000007120213D204E554C4C0000008D
:10CD100069706164647220213D204E554C4C0000C6
:10CD2000E4550408AC010020E46C012070B5054610
:10CD30000E46144600BF04EB84001C4901EB800042
:10CD4000807C022802DA1AA0FBF748F800BF04EB47
:10CD50008400164901EB8000807C022817D104EB87
:10CD6000840001EB8000C07CE42810DB04EB84002D
:10CD70000A4602EB8000011D284600F0C3F930B9D5
:10CD8000032004EB8401094A02EB8101887404EB5F
:10CD90008400064901EB800000F10C0305F12B0231
:10CDA0003146284600F0C6F970BD0000E46C012051
:10CDB0006172705F7461626C655B6172705F6964FF
:10CDC000785D2E7374617465203E3D204554484162
:10CDD00052505F53544154455F535441424C4500B7
:10CDE0002DE9F05F80460F46164608F12B094FF0FB
:10CDF000FF3A4146386802F039FE38B9387800F019
:10CE0000F000E02802D00FB1386828B900BF00BF99
:10CE10006FF00D00BDE8F09F01213846FFF752FD8D
:10CE20000446002C06DA00BF00BF0EB100BF00BFF1
:10CE30002046EFE704EB8400534901EB8000807C3F
:10CE400030B9012004EB84014F4A02EB8101887460
:10CE500000BF04EB84004C4901EB8000807C01287A
:10CE600009D004EB840001EB8000807C022802DA08
:10CE700046A0FAF7B3FF00BF04EB8400424901EB80
:10CE80008000807C012800D03EB93946404600F041
:10CE900039F982460EB95046BCE700BF16B945A025
:10CEA000FAF79CFF00BF04EB8400374901EB8000D8
:10CEB000807C02280FDB42490C7004EB840032496D
:10CEC00001EB800000F10C034A463146404600F079
:10CED00031F9824656E004EB84002B4901EB8000D7
:10CEE000807C01284ED14FF0000B354611E000BF89
:10CEF00068892989884204D1286810B131A0FAF7DD
:10CF00006DFF00BF287B012802D04FF0010B02E02B
:10CF10002D68002DEBD100BFBBF1000F10D0298987
:10CF20000022032007F0DEFA05466DB1314628469F
:10CF300007F05EFD40B1284607F098FE002503E0AB
:10CF40003546284608F03EF8BDB104EB84000E4992
:10CF500051F8200040B100BF00BF04EB84010A4A31
:10CF600052F8210007F082FE04EB8400064941F8E4
:10CF700020504FF0000A00BF03E000BF00BF4FF099
:10CF8000FF3A00BF504645E7E46C01206172705FD4
:10CF90007461626C655B695D2E7374617465203DBC
:10CFA0003D2050454E44494E47206F722053544116
:10CFB000424C45007120213D204E554C4C00000054
:10CFC000AC0100206E6F207061636B657420717519
:10CFD0006575657320616C6C6F7765642100000076
:10CFE0002DE9F84F0746884691469A46DDF828B065
:10CFF0000020009000BF17B930A0FAF7EFFE00BF85
:10D0000000222A21032007F06DFA05462DB900BF42
:10D0100000BF4FF0FF30BDE8F88F00BF68892A28B5
:10D0200002DA2AA0FAF7DAFE00BF6E6806F10E04F3
:10D0300000BF00BF0D9804F0CAF9E08000BF97F868
:10D040002A00062802D02E48FAF7C8FE00BFDAF8F8
:10D050000000A060BAF80400A0810B980168C4F831
:10D0600012108088E082D9F800003060B9F804001E
:10D07000B080D8F80000C6F80600B8F80400708147
:10D08000DBF80000C4F80E000C980068A0614FF4B3
:10D09000807020800820608006202071042060714C
:10D0A0004FF4C160B08129463846BA699047009074
:10D0B000284607F0DBFD00250098ACE76E65746933
:10D0C0006620213D204E554C4C000000636865638E
:10D0D0006B20746861742066697273742070627565
:10D0E000662063616E20686F6C6420737472756370
:10D0F00074206574686172705F686472000000007B
:10D10000645904087FB504460D4600BF00BF0121E5
:10D11000064A201D04F12B038DE825000391044AE3
:10D1200019462046FFF75CFF04B070BDEA550408BD
:10D13000E45504082DE9F04104460E46174698468A
:10D14000756800BF94F82A00062802D00C48FAF748
:10D1500045FE00BFD8F800002860B8F80400A88099
:10D160003868C5F80600B88868810820A88100BF23
:10D1700000BF31462046A2699047BDE8F08100001B
:10D180006459040870B500BF00BF00243FE004EB01
:10D190008400204901EB8000857C35B304EB8400DA
:10D1A00001EB8000C07C401C04EB8401194A02EBB7
:10D1B0008101C87404EB8400114601EB8000C07C3F
:10D1C000F0280DDA04EB840001EB8000807C01285C
:10D1D0000CD104EB840001EB8000C07C022805DB4D
:10D1E00000BF00BF2046FFF79DFC0EE004EB84006B
:10D1F000084901EB8000807C032806D1022004EB63
:10D200008401044A02EB81018874601CC4B20A2CB8
:10D21000BDDB70BDE46C01202DE9F04706460D46EC
:10D220001746984600BF96F82A00062802D02DA07F
:10D23000FAF7D4FD00BF00BF00BF5DB1286848B158
:10D240003146286802F012FC20B9287800F0F0007E
:10D25000E02805D100BF00BF6FF00D00BDE8F087EA
:10D2600041462846FFF72EFB0446002C01DA2046F3
:10D27000F4E7022004EB8401244A02EB8101887464
:10D2800004EB8400114601EB8000866000BF00BF04
:10D2900004EB840001EB80003968C160B988018229
:10D2A000002004EB840102EB8101C87404EB8400CC
:10D2B000114651F8200098B104EB840051F82090F9
:10D2C000002004EB840142F821003B4606F12B02CA
:10D2D00049463046FFF72EFF484607F0C7FC00BF1F
:10D2E0000020BBE76E657469662D3E6877616464F3
:10D2F000725F6C656E203D3D204554484152505F41
:10D300004857414444525F4C454E0000E46C0120B4
:10D310002DE9F04104460E464FF00E0860890E28B4
:10D3200000DC4EE0656800BF00BFAF89287800F0E0
:10D330000100B0B12878012809D1687888B9A878A7
:10D340005E280ED1607B40F01000607309E0062279
:10D350001E492846F3F712F818B9607B40F0080020
:10D360006073082F03D0B7F5C16F25D117E096F889
:10D37000310000F0200000B923E0C8F1000001B244
:10D38000204607F013FD28B100BF11A0FAF726FDD3
:10D3900000BF16E03146204602F096FC0DE096F8FC
:10D3A000310000F0200000B90BE0224606F12B010D
:10D3B0003046FFF7BDF900E003E000BF0020BDE804
:10D3C000F081204607F052FC0020F8E7E4550408FD
:10D3D00043616E2774206D6F7665206F76657220CD
:10D3E00068656164657220696E207061636B657445
:10D3F0000000000010B5044600BF14B914A0FAF7ED
:10D40000EDFC00BF652084F832006E213320015509
:10D41000134860611348A061204603F091FB124855
:10D42000006820B90020F8F767FA0F4908600F4834
:10D43000006820B90120F8F75FFA0C49086003235F
:10D440000B4A21460B48F8F7B9FB002010BD00003D
:10D450006E6574696620213D204E554C4C000000DD
:10D460009DCB0008E10C0108A0010020A4010020D0
:10D47000E064012079D4000808B50646354600BFAF
:10D480006A4600210A480068F8F7D0FA00BF28462B
:10D4900003F0AAFB0446002CF2D0294620462A6954
:10D4A000904720B100BF00BF204607F0DFFBEEE74A
:10D4B000A001002010B50446012001F0B9FB0022B4
:10D4C000AFF20F014FF47A7008F010FD10BD0000AC
:10D4D0002DE9F05F0746884617B3D7F81841002CAE
:10D4E00018DAF2F76BFE8346D7F8180100280CDA39
:10D4F000B8F1000F04D1D7F81801401EC7F8180181
:10D500005846F2F75FFEBDE8F09FD7F8184158463D
:10D51000F2F758FE204601F073FB05460DB9F2E71D
:10D52000F1E7F2F74BFE8346B8F1050F17D2DFE8BB
:10D5300008F003080D1013006889401C00B26881D0
:10D5400013E06889401E00B268810EE00120A881C6
:10D550000BE00020A88108E00120E88105E000BF81
:10D5600038A0FAF73BFC00BF00BF00BF686918B9DC
:10D570005846F2F727FEC6E700BF364806685AE06D
:10D580007069002848D18146B5F90A0000280FDDEE
:10D59000B16869B1E11704EB5171C910B268515C0F
:10D5A00004F0070301229A40114009B14FF001092C
:10D5B000A88990B1B9F1000F0FD1F16869B1E117F5
:10D5C00004EB5171C910F268515C04F007030122A9
:10D5D0009A40114009B14FF00109E88990B1B9F1C1
:10D5E000000F0FD1316969B1E11704EB5171C91016
:10D5F0003269515C04F0070301229A40114009B1DD
:10D600004FF00109B9F1000F05D00120706106F15A
:10D61000180008F042FC00BF0F48D0F800A05846A0
:10D62000F2F7D0FDF2F7CAFD83460B480068824549
:10D6300000D0A2E73668002EA2D15846F2F7C2FD0C
:10D6400000BF60E7756E6B6E6F776E206576656EF6
:10D6500074000000900100209401002070B5054680
:10D66000284600F04DFD04465CB928460CF05CFFEE
:10D67000044634B9686AFBF775FE04460CB900200D
:10D680002860204670BD00002DE9F74F90B091460C
:10D6900010A801F08FFA0F900F98002803DA0B20E2
:10D6A00013B0BDE8F08F1198012801DD1320F7E7D2
:10D6B000A9F1010000EA090008B11320F0E7FE49D2
:10D6C0000F9851F820B0BBF1000F01D10C20E7E713
:10D6D00000208BF800000F98C0B20C9000200B9037
:10D6E0000C98FDF7B5FC0190019800F0010008B11D
:10D6F0000320D5E7019800F0040008B10A20CFE725
:10D7000000BF04AA01210C98FDF7AAFC10B90498E7
:10D71000802801D20120C3E7119808B1002000E061
:10D720003F2080460498A0EB08000490B9F1000F58
:10D7300013D14FF4FA610498B0FBF1F00A904FF066
:10D74000000A01E00AF1010ADC4830F81A100A98D0
:10D750008142F7D8DA4830F81A904FEA5929B9F1DE
:10D76000000F01D14FF00109B9F1800F01D94FF03D
:10D7700080090498B0FBF9F7012540F6F67087425E
:10D7800000D302254FF6F670874200D30325032D00
:10D790000AD1082000EB870000F2FF10460A202083
:10D7A00003900020029011E0012D05D107EB470006
:10D7B000401C4008C01C01E07800001D064606F22F
:10D7C000FF10460A01200390202002900398404455
:10D7D00007900798304406900299069808440590EF
:10D7E00005984844A0EB08000499884201D90E200E
:10D7F00056E709AA03210C98FDF732FC28B90998CD
:10D8000018B10998B0F5004F01D901200990099984
:10D8100005980844401E491E8843099009990598B7
:10D82000081A0990032D08D1099903980844039018
:10D83000099907980844079001E009980644DDE932
:10D840000301081A811B0298081AB0FBF9F7022D90
:10D8500003D140F6F670874205D3032D05D14FF66C
:10D86000F670874201D20E201AE7032D02D10C2058
:10D870000D9010E0012D06D10498B0F5803F02D242
:10D8800001200D9007E00498B0F5803F01D20420FC
:10D8900000E006200D9000BF119810B1F0200E900E
:10D8A00044E04FF4007200210BF1300004F0D2FC90
:10D8B0000BF5F77401206070A0700020E0700D98E7
:10D8C0002071FE206071049840443F21B0FBF1F0CC
:10D8D000FF21B0FBF1F009903F21099841EA900047
:10D8E000A0710998E0713F20207200216172A1723D
:10D8F000E172049820730498010A61730498010C82
:10D90000A1730498010EE17355218BF82E12AA2100
:10D910008BF82F12012300220BF130010C98FDF738
:10D92000EFFB08B10120BBE6F8200E900BF13004AC
:10D930004FF400720021204604F08CFC0B2261A100
:10D94000204604F0B4FA4FF4007A84F80BA04FEAB2
:10D950001A21217384F80D900398A0730398010A8B
:10D96000E17301202074032D01D1002001E04FF468
:10D970000070824684F811A04FEA1A21A17404981D
:10D98000B0F5803F05D20498E0740498010A21752F
:10D9900010E0049884F820000498C0F307212120A7
:10D9A00001550498C0F30741222001550498010E47
:10D9B000232001550E9860753F2020760021617666
:10D9C000FF20A076E17684F81C804FEA1821617769
:10D9D0004FEA1841A1774FEA1861E17701F0E2F8C8
:10D9E0000990032D3ED1099884F843000998C0F3AB
:10D9F0000721442001550998C0F3074145200155EE
:10DA00000998010E4620015584F82460C6F30721C9
:10DA100025200155C6F3074126200155310E272048
:10DA20000155022084F82C0000212D2001552E20C4
:10DA300001552F200155012084F830003120015577
:10DA4000062084F8320033200155802084F84000FD
:10DA5000292084F8420013221DA104F1470004F09C
:10DA600026FA1FE0099884F827000998C0F30721D7
:10DA7000282001550998C0F307412920015509982C
:10DA8000010E2A200155A675310AE175802084F81F
:10DA90002400292084F82600132212A104F12B006F
:10DAA00004F005FA552084F8FE01AA2140F2FF1087
:10DAB0000155012342461FE000E30020E253040821
:10DAC000F8530408EBFE904D53444F53352E30006D
:10DAD0004E4F204E414D45202020204641543332A8
:10DAE000202020004E4F204E414D45202020204632
:10DAF000415420202020200021460C98FDF700FBF7
:10DB000008B10120CCE5032D06D1012308F106025E
:10DB100021460C98FDF7F4FA079808904FF0000A98
:10DB200061E04FF400720021204604F093FB0E9850
:10DB30000990032D14D0012D01D1624801E06FF04E
:10DB4000FF00099908430990099820700998000A74
:10DB500060700998000CA0700998000EE07019E040
:10DB6000099860F0FF000990099820700998000A50
:10DB700060700998000CA0700998000EE070FF20FA
:10DB80002071FF216171A171E17120726172A17236
:10DB90000F21E1720898411C024601230891214699
:10DBA0000C98FDF7ADFA08B1012079E54FF4007249
:10DBB0000021204604F04EFB012009900EE0089859
:10DBC000411C02460123089121460C98FDF798FA62
:10DBD00008B1012064E50998401C09900998B042F9
:10DBE000EDD30AF1010ABAF1000F9AD0032D01D149
:10DBF000484600E00298824600BF0898411C024651
:10DC00000123089121460C98FDF77AFA08B101200A
:10DC100046E5AAF10100B0F1000AEED1032D46D18C
:10DC20005220207060706120A0704120E07072204E
:10DC300084F8E401722140F2E51001554121401CB5
:10DC400001556121401C0155781E84F8E801C0F39C
:10DC5000072140F2E9100155781EC0F307414FF447
:10DC6000F5700155781E010E40F2EB1001550220AF
:10DC700084F8EC01002140F2ED100155401C0155E3
:10DC8000401C0155552084F8FE01AA2140F2FF10E6
:10DC90000155012308F1010221460C98FDF730FAE5
:10DCA000012308F1070221460C98FDF729FA00220A
:10DCB00011460C98FDF7D4F908B10120F0E40020DA
:10DCC000EEE4000000FFFF00F7B582B016460398AF
:10DCD000019001A800F06EFF0546002D02DA0B202E
:10DCE00005B0F0BD0F4850F8254024B12046FBF7A1
:10DCF000DFF800202070029810B10020029908700F
:10DD00000849029841F82500029808B1012E01D077
:10DD10000020E5E7002203A902A800F0EFFB074678
:10DD20003846DDE700E300202DE9F743ADF50E7D31
:10DD30000546164625B909200DF5117DBDE8F0838D
:10DD40000020286006F01F0626F001028FA984A893
:10DD500000F0D4FB0746002F72D181A88A9001A859
:10DD60008C9084A88F9900F0CFFD0746899C6FB9ED
:10DD70000CB906270AE026F0010008B1012000E0F6
:10DD80000020014684A8FBF74DF8074606F01C006A
:10DD9000002856D077B1042F08D1FEF79DFB18B1AB
:10DDA00084A8FDF73CF800E01220074646F008067C
:10DDB000899C09E0E07A00F0110008B1072703E030
:10DDC00006F0040000B10827002F38D106F0080043
:10DDD000A8B300F0E7FE804684F80E804FEA1821D1
:10DDE000E1734FEA184121744FEA18616174002011
:10DDF000E072207700216177A177E177214684984E
:10DE000002F0F6FD81460021204607F0CBFE0120FE
:10DE100084990871B9F1000F11D08498D0F82C8042
:10DE20004946849807F024FE074647B9A9F1010046
:10DE30008499C8604146849804F0D8FB07460FE0F7
:10DE400042E06FB9E07A00F0100008B1042707E063
:10DE500006F0020020B1E07A00F0010000B10727CF
:10DE6000B7B906F0080008B146F020068498C06AE9
:10DE7000E8612C6226F0010008B1012000E00020DA
:10DE8000014684A801F026FD6862686A00B902278D
:10DE9000D7B9AE710020E8712146849802F0A8FD40
:10DEA0002861E07F0106A07F41EA0041607F41EAEE
:10DEB0000020217F0843E8600020A860A8618498C2
:10DEC00028602868C088A880384635E733B5ADF5A6
:10DED000057D04461CB909200DF5077D30BD0022E3
:10DEE00086A984A800F00AFB0546002D33D184984A
:10DEF000206081A8A06101A820622046869900F0D8
:10DF000003FD05460DBB606958B16069C07A00F039
:10DF1000100028B16169849802F06AFDA06000E0F9
:10DF2000052595B98498C088A08000212046FDF77A
:10DF300040F805464DB9A06840B10021204601F0E7
:10DF4000C9FCE061E06900B9122501E00020E06150
:10DF5000042D00D105250DB1002020602846BBE727
:10DF60002DE9FF4F83B0044615469A46DDF810B000
:10DF70000020CAF8000020460CF0D6FA0290029861
:10DF800018B1029807B0BDE8F08FE07908B1E079E8
:10DF9000F8E7A07900F0010008B90720F2E7D4E91A
:10DFA0000210401A00900098854200D9009DA2E01E
:10DFB0002089C0F3080000287ED120688078401EA8
:10DFC000A16800EA512000F0FF09B9F1000F17D154
:10DFD000A06810B92069019004E06169206800F030
:10DFE0006DFD01900198022802D20220E071C9E77C
:10DFF0000198401C10B90120E071C3E701986061ED
:10E0000061692068FAF76CFF064616B90220E071D4
:10E01000B8E74E444FEA5528B8F1000F29D009EB74
:10E02000080021688978884203D920688078A0EBAD
:10E03000090821684878434632465946FDF73CF8BE
:10E0400010B10120E0719DE7A07900F0400068B1B7
:10E05000A069801B404509D2A169891B0BEB4120B7
:10E060004FF4007204F1280103F021FF4FEA482722
:10E0700037E0A069B04220D0A07900F0400078B12C
:10E0800021684878012304F12801A269FDF738F8D6
:10E0900010B10120E07175E7A07920F04000A07177
:10E0A000216848780123324604F12801FDF704F87D
:10E0B00018B10120E07165E700E0A6612089C0F396
:10E0C0000800C0F50077AF4200D92F462089C0F381
:10E0D000080204F1280011183A46584603F0E7FEFA
:10E0E00000BFBB44A0683844A060DAF800003844A0
:10E0F000CAF80000ED1B002D7FF45AAF002041E765
:10E100002DE9F041044620460CF00EFA0746002F98
:10E110004CD1A07900F02000002847D0A07900F071
:10E12000400078B121684878012304F12801A269F0
:10E13000FCF7E6FF10B10120BDE8F081A07920F0E6
:10E140004000A071E169206804F050FA0746002FF2
:10E150002CD1256AE87A40F02000E872207B2877ED
:10E16000A089010A6977E068010CA977E068010ECF
:10E17000E9772846216907F015FD00F013FD0646F2
:10E18000AE75310AE975310C2976310E69760020B9
:10E19000A8740021E974A07920F02000A07101206A
:10E1A00021680871206807F015FD07463846C3E767
:10E1B00071B5ADF5177D012297A98DA800F09EF9E4
:10E1C0000446002C4FD180A89390CDF854D28DA84E
:10E1D000979900F099FB044600BF24B902218DA84D
:10E1E000FAF720FE0446002C3DD1929E0EB906247B
:10E1F00004E0F07A00F0010000B1072431468D9868
:10E2000002F0F6FB0546ECB9F07A00F01000C8B158
:10E21000022D01D2022415E028228DA983A803F043
:10E2200046FE8595022183A8FCF7C3FE04464CB93F
:10E23000002183A8FCF791FD044604B90724042CAF
:10E2400000D100247CB98DA8FCF77EFE044654B9A9
:10E2500025B129468D9807F00BFC04461CB98D9812
:10E2600007F0B8FC044620460DF5187D70BD2DE979
:10E27000FF4F83B0044615469B460498019000204A
:10E28000CBF8000020460CF04FF90290029818B12C
:10E29000029807B0BDE8F08FE07908B1E079F8E7BF
:10E2A000A07900F0020008B90720F2E7A06828442E
:10E2B000A168884200D20025B5E02089C0F308009B
:10E2C000002877D120688078401EA16800EA51209C
:10E2D00000F0FF0ABAF1000F1ED1A06838B9276913
:10E2E00057B900212068FAF751FE074604E061693A
:10E2F0002068FAF74BFE074607B997E0012F02D1D5
:10E300000220E071C5E7781C10B90120E071C0E778
:10E310006761206900B92761A07900F0400078B1F9
:10E3200021684878012304F12801A269FCF7E8FE7E
:10E3300010B10120E071ACE7A07920F04000A0719D
:10E3400061692068FAF7CCFD064616B90220E07133
:10E350009FE756444FEA5529B9F1000F2BD00AEB3D
:10E36000090021688978884203D920688078A0EB69
:10E370000A09216848784B4632460199FCF7C0FEED
:10E3800010B10120E07184E7A069801B48450ED2DE
:10E39000A069801B019A02EB40214FF4007204F146
:10E3A000280003F084FDA07920F04000A0714FEA1E
:10E3B00049282BE013E0A069B0420FD0D4E9020154
:10E3C00088420BD2216848780123324604F12801A3
:10E3D000FCF772FE10B10120E0715AE7A6612089B6
:10E3E000C0F30800C0F50078A84500D9A8462189E7
:10E3F000C1F3080204F1280150184246019903F0C4
:10E4000056FDA07940F04000A07100BF0198404443
:10E410000190A0684044A060DBF800004044CBF8C5
:10E420000000A5EB0805002D7FF447AF00BFD4E93D
:10E430000201884201D9A068E060A07940F0200084
:10E44000A071002025E700002DE9F04102460F46AB
:10E45000802A01DA10462FE01FB1184B45F22056F2
:10E4600002E0174B45F220560025102416E0A6EBDB
:10E47000050C0CEBDC7805EB68014FEA410C33F836
:10E480001CC0944500D10BE04FEA410C33F81CC08E
:10E49000944501DA0D4600E00E46641E002CE6D1DC
:10E4A00000BF34B14FF0010C0CEB410C33F81CC031
:10E4B00001E04FF0000C6046BDE8F08190FB0208DF
:10E4C0000CA701080246002100E0491C094830F869
:10E4D000110020B1074830F811009042F5D10548ED
:10E4E00030F8110018B1044830F811007047104698
:10E4F000FCE7000014500408F45104082DE9F74F1C
:10E5000088B0002108980160099800F053FB07903B
:10E510000798002803DA0B200BB0BDE8F08FD6492E
:10E52000079851F820400CB90C20F5E708980460D2
:10E53000207878B16078FCF7DBFD804608F00100B8
:10E5400040B90A9820B108F0040008B10A20E3E7B6
:10E550000020E1E700202070079860706078FCF7E9
:10E5600077FD804608F0010008B10320D4E70A983F
:10E5700020B108F0040008B10A20CDE70027394691
:10E580002046FAF7FDFB0546012D01D06DBB2CE0BE
:10E59000002614E004F5F77101EB0610017951B182
:10E5A000C17A0A06817A42EA0142417A42EA0121AD
:10E5B000027A114300E000214DF82610761C042E4B
:10E5C000E8D3002606B1761E00BF5DF8267027B19D
:10E5D00039462046FAF7D4FB00E0022005461DB17B
:10E5E000701C06460428F0D300BF032D01D1012082
:10E5F00092E70DB10D208FE73B20015D94F83C00C0
:10E6000041EA0020B0F5007F01D00D2084E74620CC
:10E61000015D94F8470041EA0029B9F1000F0ED1DD
:10E6200094F85700010694F8560041EA004194F826
:10E63000550041EA002094F8541040EA0109C4F85A
:10E6400018904020005DE070E078012804D0E07868
:10E65000022801D00D205FE7E07809FB00F93D209A
:10E66000005DA070A07818B1A078411E084008B1E4
:10E670000D2051E74120015D94F8420041EA00205D
:10E680002081207A00F00F0008B10D2044E74320DC
:10E69000015D94F8440041EA002BBBF1000F0ED15C
:10E6A00094F85300010694F8520041EA004194F8AE
:10E6B000510041EA002094F8501040EA010B3E203E
:10E6C000015D94F83F0041EA00200490049808B9E5
:10E6D0000D2021E704984844218900EB1110069091
:10E6E0000698834501D20D2016E70698ABEB000093
:10E6F000A178B0FBF1FABAF1000F01D10D200BE7C0
:10E70000012540F6F670824500D302254FF6F670DB
:10E71000824500D303250AF102006061E761049895
:10E720003844206206983844A062032D16D120890F
:10E7300008B10D20F0E694F85F00010694F85E0041
:10E7400041EA004194F85D0041EA002094F85C1031
:10E750000843606260698000059014E0208908B970
:10E760000D20D9E6206A48446062022D02D160691A
:10E77000400007E0207D00F00100616901EB4101EC
:10E7800000EB51000590A169059800F2FF10B1EB74
:10E79000502F01D20D20BFE64FF0FF302061E06026
:10E7A00080206071032D5AD194F8601094F86100B4
:10E7B00041EA0020012852D1791C204603F016FFBF
:10E7C000E8BB0020607194F82E1294F82F0241EA01
:10E7D00000204AF65521884241D13320005D0106D0
:10E7E0003220005D41EA00413120005D41EA002015
:10E7F00094F8301008432149884230D194F8170228
:10E80000010694F8160241EA004194F8150241EA23
:10E81000002094F814120843194988421FD194F833
:10E820001B02010694F81A0241EA004194F8190209
:10E8300041EA002094F818120843206100E00EE03D
:10E8400094F81F02010694F81E0241EA004194F870
:10E850001D0241EA002094F81C120843E060257074
:10E8600008480088401C80B206490880E0802046A5
:10E87000FAF71EFB00204FE600E3002052526141F0
:10E88000727241618C000020F0B504461D464D7344
:10E890000F27CF7200270F738F76BC4681F81BC0FD
:10E8A000571E07EB870C0CEBC706002738463B4684
:10E8B00000BF4FF6FF77B84203D03746761C34F8D6
:10E8C0001700DFF840C01CF803C001F80C00071265
:10E8D000DFF830C01CF803C08C448CF8017008B914
:10E8E0004FF6FF705F1C3B460D2FE2D34FF6FF77CC
:10E8F000B84202D034F816700FB942F040020A70E4
:10E90000F0BD0000D45304082DE9F34104460198FA
:10E9100000782F2803D0019800785C2802D1019854
:10E92000401C01900020A06001980078202807D2A8
:10E9300000212046FCF73DFB05460020606128E0F1
:10E9400000BF01A92046FAF78DFB054605B11FE07F
:10E950002046FCF705F90546A069C67A3DB1042DAD
:10E9600004D100BF06F0040000B9052510E006F050
:10E97000040000B10CE06769F87A00F0100008B9F3
:10E98000052505E03946206802F032F8A060D8E796
:10E9900000BF2846BDE8FC8170B504460D46E1B2D3
:10E9A0000548F9F7D3F900BF80210348F8F7D0FEF6
:10E9B0000028F9D0204670BD001001402DE9F0413B
:10E9C00004460D4666680020606020812061F1F7F2
:10E9D000F5FB0746002020603846F1F7F3FB3EB117
:10E9E0001DB1304606F042F902E0304604F016FE52
:10E9F000BDE8F0812DE9FC4707468A4690461E4651
:10EA00000B225146384603F052FA052E18D93046EB
:10EA100010E038F8021B00250AE00A4660F35F02A6
:10EA20001046491000F480320AB1234A50406D1C50
:10EA3000102DF2D3B8F80020002AEAD1064600BF14
:10EA4000072500BF06F00F0000F13009B9F1390FBA
:10EA500003DD09F1070000F0FF0928466D1E0DF8DF
:10EA600000903609002EEDD17E200DF8050000241F
:10EA70000BE0385D812807DB385DFE2804DC681E6A
:10EA8000A04200D106E0641C641CAC4202D2385D96
:10EA90002028EED100BF00BF082D04D228466D1CEF
:10EAA0001DF8001000E020212046641C3954082C79
:10EAB000F2D3BDE8FC870000211001002DE9F041F0
:10EAC00005460C46022C02D36869A04202D80120F8
:10EAD000BDE8F0812878012804D002282CD0032832
:10EAE0005AD13DE0274607EB5707286A00EB57212C
:10EAF000284603F07BFD00B150E0C7F3080105F1A3
:10EB0000300010F801807F1C286A00EB572128464E
:10EB100003F06CFD00B141E0C7F3080105F13000DE
:10EB2000405C48EA002804F0010010B14FEA1810D8
:10EB3000CEE7C8F30B00CBE7286A00EB1421284688
:10EB400003F054FD00B129E040F2FF1000EA440157
:10EB500005F130000E183078717840EA0120B7E7EF
:10EB6000286A00EBD411284603F040FD00B115E0FF
:10EB700040F2FF1000EA840105F130000E18F07831
:10EB80000006B17840EA0140717840EA012031780E
:10EB9000084320F070409BE7012099E700BF4FF049
:10EBA000FF3095E7004870470000E2440048704796
:10EBB000047A002070B502464FF0FF301568E5B1C9
:10EBC000116800E0491C0D78202D02D30D783A2DF4
:10EBD000F8D10D783A2D0FD1146814F8015BA5F126
:10EBE00030030A2B07D28C4205D1032B03D21846DF
:10EBF0004D1C2946156070BD002000BFFBE70000DA
:10EC00000146002901DB082903DB00BF00BF00200B
:10EC1000704701EB4100054B03EBC002106818B9C7
:10EC200000BF00BF0020F3E71046F1E7A05B012022
:10EC300070B5054600F030F804461548007800F03D
:10EC40000100D0B11248007800F0100050B1F4B9C2
:10EC5000104805F0B8FB0E48006820F010000C4981
:10EC6000086014E09CB10B4805F0C2FB084800683E
:10EC700040F010000649086009E044B1054801F081
:10EC80005FFF044805F0B4FB0248FBF7ABFD70BD25
:10EC90006C0000207CD9002010B501210846F3F754
:10ECA000B3FE00F0040008B1012010BD0020FCE715
:10ECB00010B50446204602F001F910BD2DE9F041DF
:10ECC00086B007460C46154600220121022002F0BC
:10ECD000F9FF0646002E04DA6FF0010006B0BDE829
:10ECE000F08145BB002000906B462A4A69463846B1
:10ECF000FCF78CFB0020059005E00A20F7F796F959
:10ED000005980A300590009818B90598B0F5FA6F83
:10ED1000F3DB0598B0F5FA6F05DB1FA0F9F75EF895
:10ED20006FF00100DAE7684601F0DEFD804601F091
:10ED300017FD029003E0384601F012FD029010200A
:10ED40008DF8040002208DF80500A0B202F03FFB10
:10ED5000ADF80600002003900490102201A930466F
:10ED600002F0E0F828B111A0F9F738F84FF0FF30C1
:10ED7000B4E740F6B8300590042005AB41F2060236
:10ED8000D11F0090304602F0A9FD0EA0F9F726F839
:10ED90003046A3E7F9F20008646E732067657420BB
:10EDA0006661696C757265200A000000636F6E6EA3
:10EDB00065637420736572766572206572726F7216
:10EDC000200D0A00636F6E6E656374207365727642
:10EDD00065722073756363657373200D0A0000000C
:10EDE0002DE9F05F05460E4617469846DDE90A9A7A
:10EDF0004FF0FF34424639462846FFF75FFF04468E
:10EE0000002C00DA12E032462946204600F040F895
:10EE10008346002C00DA09E052464946204600F0BD
:10EE2000D3F98346002C00DA00E000BF002C02DB9F
:10EE30002046FFF73DFF5846BDE8F09F2DE9F04121
:10EE400007460E46144610E04FF47A7231463846B3
:10EE500002F0BEFF0546002D03DC4FF0FF30BDE899
:10EE6000F081A4F57A7406F57A76B4F57A7FEBDC56
:10EE7000002C0ADD22463146384602F0A9FF05463D
:10EE8000002D02DC4FF0FF30E9E70120E7E700004A
:10EE90002DE9F04106460F4614464FF4806125489F
:10EEA000F1F72EFA24A12348F8F7A8FF24B924A1EA
:10EEB0002048F1F730FA03E021461E48F1F72BFA1B
:10EEC00020A11C48F1F727FA21A11A48F1F723FAEB
:10EED00039461848F1F71FFA1FA11648F1F71BFA37
:10EEE0001EA11448F1F717FA21A11248F1F713FAFD
:10EEF00026A11048F1F70FFA2AA10E48F1F70BFAF4
:10EF000015A10C48F1F707FA0A48F1F722FA05466D
:10EF100008492BA0F8F762FF2A460649304602F05E
:10EF200057FF0546002D03DC4FF0FF30BDE8F081B0
:10EF30000120FBE7647F01204745542000000000CA
:10EF40002F00000020485454502F312E310D0A005C
:10EF5000486F73743A2000000D0A0000436F6E6E14
:10EF6000656374696F6E3A20636C6F73650D0A0098
:10EF70004163636570743A206170706C6963617499
:10EF8000696F6E2F6A736F6E0D0A0000557365729C
:10EF90002D4167656E743A2073746D33326632307A
:10EFA000370D0A0043616368652D436F6E74726F9D
:10EFB0006C3A206E6F2D63616368650D0A00000076
:10EFC000257300002DE9F04180460D4614461E468B
:10EFD0004FF480612E48F1F793F92EA12C48F8F7F1
:10EFE0000DFF24B92DA12A48F1F795F903E0214638
:10EFF0002748F1F790F92AA12548F1F78CF940212B
:10F000002A48F1F77DF92A4629A12848F8F7F6FEA3
:10F0100026491F48F1F77FF928A11D48F1F77BF930
:10F020002BA11B48F1F777F930A11948F1F773F9D3
:10F0300034A11748F1F76FF939A11548F1F76BF9C9
:10F0400040211A48F1F75CF932463EA11748F8F71B
:10F05000D5FE16490E48F1F75EF917A10C48F1F7F5
:10F060005AF90B48F1F775F9074609493BA0F8F73B
:10F07000B5FE3A460649404602F0AAFE0746002F72
:10F0800003DC4FF0FF30BDE8F0810120FBE700001A
:10F09000647F0120504F5354200000002F000000D7
:10F0A00020485454502F312E310D0A006485012020
:10F0B000486F73743A2025730D0A0000436F6E6E1B
:10F0C000656374696F6E3A20636C6F73650D0A0037
:10F0D0004163636570743A206170706C6963617438
:10F0E000696F6E2F6A736F6E0D0A0000557365723B
:10F0F0002D4167656E743A2073746D333266323019
:10F10000370D0A0043616368652D436F6E74726F3B
:10F110006C3A206E6F2D63616368650D0A00000014
:10F12000436F6E74656E742D547970653A2061700A
:10F13000706C69636174696F6E2F6A736F6E0D0A0C
:10F1400000000000436F6E74656E742D4C656E6731
:10F1500074683A2025640D0A000000002573000041
:10F160002DE9F05F06460F4690469946DDE90ABA5A
:10F170004A4641463046FFF7A1FD0546002D00DA1C
:10F1800019E053463A4631462846FFF71BFF04462E
:10F19000002C00DA0FE0524659462846FFF74EFE93
:10F1A0000446002C00DA06E02846DDE90C1200F0E7
:10F1B00057F8044600BF002D02DB2846FFF778FD14
:10F1C0002046BDE8F09F00002DE9F04780460E463E
:10F1D000174600254FF400721F49404600F012F90F
:10F1E0000446002C02DC681EBDE8F0871A491BA00B
:10F1F000F8F7F4FD184800F02BF9814600BF4FF4F2
:10F2000000721549404600F0FDF80446124913A06B
:10F21000F8F7E4FD022C04DC00D104E04FF0FF30ED
:10F22000E2E7002CEBDC00BF002500BF00234FF419
:10F2300000720949404602F0FEF80446002C05DD44
:10F24000701922460449F1F742F82544002CEDDC00
:10F250003D604846C8E70000648301202573000034
:10F260002DE9F04780460E46174600254FF4007200
:10F270001F49404600F0C6F80446002C02DC681E18
:10F28000BDE8F0871A491BA0F8F7A8FD184800F060
:10F29000DFF8814600BF4FF400721549404600F088
:10F2A000B1F80446124913A0F8F798FD022C04DCCB
:10F2B00000D104E04FF0FF30E2E7002CEBDC00BFB0
:10F2C000002500BF00234FF400720949404602F0B8
:10F2D000B2F80446002C05DD701922460449F0F707
:10F2E000F6FF2544002CEDDC3D604846C8E70000F1
:10F2F00064830120257300002DE9F04105460C468A
:10F30000164620683060204601F0EEFA07463A467D
:10F31000294602A0F8F762FDBDE8F08125733A2581
:10F32000730D0A00FEB54FF47041012004F058F946
:10F3300004463221012004F053F90646194A1AA165
:10F340003046F8F75BFD02A8002341F69272314681
:10F35000CDE900401DA0FFF743FD0546C82D0ED1A5
:10F360001EA0F2F7B9F92046F0F7F3FF07463A4638
:10F3700021461AA00BF044F901201B4908702146D0
:10F3800011A0F8F72BFD294618A0029AF8F726FDE0
:10F390002146012004F012F93146012004F00EF953
:10F3A000FEBD0000E85300202F696F742F74726156
:10F3B0006E736D69742F6765745472616E736D69D5
:10F3C00074436F6E6669672F257300006770752E32
:10F3D00072696E677A6C652E636F6D00646576691D
:10F3E00063652E7478740000240000200D0A2072DA
:10F3F00065743D256420646174616C656E3D2564AF
:10F400000D0A00002DE9F84380460D4617460024FA
:10F41000002000900FE0002301226946404602F0E0
:10F420000AF80646002E01DC0A2000909DF8002014
:10F430002046641C2A54781EA04203DD9DF800007B
:10F440000A28E8D1002028552046BDE8F8830000AE
:10F450002DE9F0410446092210A12046F0F7A4FF4F
:10F4600028B1092210A12046F0F79EFF90B9093477
:10F470002078A0F130076078A0F13005A078A0F1E5
:10F4800030066420784305EB850100EB41003044F1
:10F49000BDE8F0814FF0FF30FAE7000048545450C7
:10F4A0002F312E3120000000687474702F312E31FE
:10F4B0002000000030B585B04FF400711148F0F71E
:10F4C0001FFF11480068F0F744FF054604A80D49E6
:10F4D0000D4A12680023CDE90025CDE9021041F65E
:10F4E00092720AA10EA0FFF73BFE0446054910A048
:10F4F000F8F774FC21460FA0049AF8F76FFC05B0EA
:10F5000030BD000004780020280000202F696F74AF
:10F510002F746573742F687474705465737400006D
:10F520006770752E72696E677A6C652E636F6D00F9
:10F53000257300000D0A207265743D256420646106
:10F5400074616C656E3D25640D0A000070B505465A
:10F550000C4622460321284600F052F970BD0000F7
:10F560002DE9FE4F04468946666830780007870E0D
:10F570007942204605F01AFC10B92089042802D2ED
:10F5800000BF00BFB9E0606890F800A0606890F824
:10F5900001B0BAF1000F03D0BAF1080F78D100E042
:10F5A000A6E001255948007800F0F000E02800D1DD
:10F5B000002556490868494600F058FA00B1002570
:10F5C00035B900BF00BF204605F050FBBDE8FE8FF7
:10F5D00000BF00BF2089082802D200BF00BF8CE016
:10F5E000204600F0EFF928B100BF00BF204605F02B
:10F5F0003DFBEBE72221204605F0D8FB00283BD05D
:10F600003946204605F0D2FB28B100BF40A0F8F7EC
:10F61000E5FB00BF75E021890022022004F062FFB3
:10F62000054615B900BF00BF6BE000BF698907F14F
:10F630000800814202D243A0F8F7D0FB00BF214668
:10F64000284605F0D5F928B100BF4CA0F8F7C6FB55
:10F6500000BF56E06E68784201B2284605F0A6FB6E
:10F6600028B100BF4FA0F8F7B9FB00BF49E0204622
:10F6700005F0FCFA2C460CE06FF02101204605F065
:10F6800095FB30B100BF47A0F8F7A8FB00BF38E0FA
:10F690002BE0D4F804801D480068F0604E480068F4
:10F6A0003061002088F80000A8F80200FF203072C6
:10F6B000002070813946204605F078FB20B100BF5C
:10F6C00046A0F8F78BFB0FE001200021FF230A463C
:10F6D000CDE9010900910D49204600F01BFC0546CB
:10F6E0000DB100BF00BF00BF02E000BF00BF00BF00
:10F6F00000BF204605F0BAFA68E7204605F0B6FAE2
:10F7000064E7204605F0B2FA00BF5FE78001002001
:10F7100069636D705F696E7075743A206D6F76699C
:10F720006E6720702D3E7061796C6F616420746F1C
:10F7300020697020686561646572206661696C6526
:10F74000640A0000636865636B20746861742066F6
:10F750006972737420706275662063616E20686FD1
:10F760006C642073747275637420746865204943F7
:10F770004D502068656164657200000069636D70BA
:10F780005F696E7075743A20636F7079696E672077
:10F79000746F206E65772070627566206661696C93
:10F7A00065640A0069636D705F696E7075743A20F4
:10F7B000726573746F72696E67206F726967696EC4
:10F7C000616C20702D3E7061796C6F6164206661A0
:10F7D000696C65640A0000007C01002043616E27AB
:10F7E00074206D6F7665206F766572206865616440
:10F7F000657220696E207061636B657400000000A3
:10F800002DE9FE4306460F469046002224210120A2
:10F8100004F068FE05461DB900BF00BFBDE8FE83C9
:10F8200000BF6889242802D21AA0F8F7D7FA00BFCF
:10F83000D6F8049000BF00BF00BF00BF00BF00BFEC
:10F8400000BF00BF00BF00BF6C68277084F8018054
:10F850000020A080E08071686A6802F108001C2224
:10F86000F0F735FD002060806989204600F0A0F89F
:10F870006080D9F80C00029001200021FF2302AA29
:10F88000CDE90010284600F01BFB284605F0EEF9F4
:10F8900000BFC3E7636865636B20746861742066AA
:10F8A0006972737420706275662063616E20686F80
:10F8B0006C642069636D70206D65737361676500AA
:10F8C00070B505460C4622460B212846FFF798FFE7
:10F8D00070BD000030B502460B4600211BE001EB75
:10F8E0004100324C54F820001468A04212D101EBC0
:10F8F00041002E4C04EB800040689468A04209D17E
:10F9000001EB4100294C04EB80000089D488A0421F
:10F9100000D102E0491C0329E1D300BF032927D10C
:10F92000002100E0491C032906D201EB41001F4CD5
:10F9300054F820000028F5D1032901D1002030BD62
:10F9400001EB4104194D106845F8240001EB410416
:10F9500005EB840490686060D08801EB410405EBFE
:10F9600084042081002001EB410405EB84046081C4
:10F9700043B101EB41000D4C04EB8000408908B11C
:10F980000020DCE713B14FF4807006E001EB41008A
:10F99000064C04EB80004089401C01EB4104034D00
:10F9A00005EB84046081481CC9E700000CE30020DB
:10F9B00070B504460D462946204602F0DAF9C043E8
:10F9C00080B270BD2DE9F04106460024002735467F
:10F9D00017E06989686802F0CCF90444A0B200EB32
:10F9E0001444688900EBD0714910A0EB410139B192
:10F9F000C7F10100C7B2E0B2C4F3072141EA002415
:10FA00002D68002DE5D127B1E0B2C4F3072141EA0A
:10FA10000024E04380B2BDE8F08100002DE9F04110
:10FA20000B3020F00706104D19E02068B04215D3C6
:10FA3000B0420AD9871B201DD4F80480F0F747FC98
:10FA4000A019C0E90078286004E060682860201DE3
:10FA5000F0F73DFC201D2660BDE8F081251D2C68D7
:10FA6000002CE2D10020F7E7D801002018B50246AB
:10FA70000092D04300B10AB9012018BD91F83100BD
:10FA800000F0020008B90020F7E74868904201D171
:10FA90000020F2E700988B681840D1E90134234038
:10FAA000984208D1886822EA00008C68E3439842B3
:10FAB00001D10120E1E70020DFE700002DE9F74F49
:10FAC0008CB004468946B9F82800089014200490A8
:10FAD0004FF0000860680B900B9EF08801F097FCD7
:10FAE00003900398C0F30C000790039800F40050B3
:10FAF00006902089143880B209900899A1F1140069
:10FB0000C11700EB5171C1F3CF010A91AAE0089827
:10FB100014380999884201DB012000E0002005909B
:10FB20000798C0F30C00069908430390059818B98C
:10FB3000039840F400500390059808B1099801E03B
:10FB40000A98C0001FFA80FB00221421022004F052
:10FB5000C9FC054625B94FF0FF300FB0BDE8F08F66
:10FB600000BF6089142802DA41A0F8F737F900BF16
:10FB7000142268680B99F0F7AAFB6E686168049814
:10FB80000844606061890498081A6081CDF808B063
:10FB90003FE061890298814201DD029800E06089BE
:10FBA0008046B8F1000F01D1246832E000F072F80D
:10FBB00007462FB9284605F059F84FF0FF30CCE73B
:10FBC00060683B4602224146CDE90008032004F06C
:10FBD0003BFE8246BAF1000F08D1384600F060F8CB
:10FBE000284605F043F84FF0FF30B6E7204605F011
:10FBF000E9F97C61264838615146284604F07AFECE
:10FC00000298A0EB080080B20290029800B124682C
:10FC100000BF02980028BCD1CDF81080039801F0F5
:10FC2000D6FBF0800BF1140188B201F0D0FB70809C
:10FC30000020708114213046FFF7BAFE7081D9F898
:10FC40001430294648460E9A9847284605F00EF883
:10FC50000998A0EB0B0080B209900A990798084414
:10FC600080B20790099800287FF451AF00BF74E775
:10FC700074686973206E65656473206120706275B5
:10FC80006620696E206F6E6520706965636521006E
:10FC9000A509010810B5062002F00CFC10BD0000FB
:10FCA00010B5044600BF14B904A0F8F797F800BFD8
:10FCB0002146062002F09AFB10BD00007020213D75
:10FCC000204E554C4C0000002DE9F05F06460F46D3
:10FCD0004FF0010A756828780421B1EB201F07D086
:10FCE00000BF00BF304604F0C1FF0020BDE8F09F18
:10FCF000287800F00F084FF6FF7000EA880868883F
:10FD000001F085FB81467089404502DB308948451A
:10FD10000EDA7089404501DA00BF00BF30894845DE
:10FD200001DA00BF00BF304604F0A0FF0020DDE78D
:10FD30004946304605F0AAF828695C490860E86839
:10FD40005B4908604FF0010B3C4600BF00BF00BF9D
:10FD500094F8310000F0010088B1201D78B160688E
:10FD600068B1524800686168884205D04F49086808
:10FD70002146FFF77BFE10B100BF00BF0DE0BBF1D5
:10FD8000000F04D04FF0000B4A48046800E02468DC
:10FD9000BC4200D12468002CD8D100BF84B9687A55
:10FDA00011280DD105EB080000BF00BF4188B1F557
:10FDB000884F04D100BF00BF3C464FF0000A00BF8F
:10FDC000BAF1000F15D03A48006890B13849086878
:10FDD0003946FFF74BFE28B93548007800F0F000AF
:10FDE000E02806D100BF00BF304604F03FFF0020EE
:10FDF0007CE734B900BF00BF304604F037FF002075
:10FE000074E7E8884FF63F71084048B100BF00BF73
:10FE1000304600F011F906460EB9002066E7756815
:10FE200000BF00BF00BF00BF234807602348056034
:10FE30003946304605F006FB68BB687A01280DD0CC
:10FE4000062806D011280ED1394630460AF044F96A
:10FE500020E03946304606F0FDFD1BE039463046CD
:10FE6000FFF77EFB16E0114908683946FFF7FEFDF3
:10FE700050B90E48007800F0F000E02804D075601A
:10FE800002213046FFF762FB304604F0EFFE00BF70
:10FE900000BF00BF00BF0020074908600749086095
:10FEA000034908600149086000BF1FE78001002086
:10FEB0007C01002010010020740100207801002046
:10FEC0002DE9FE4F05460F4616469846DDE90C9A89
:10FED00000BFE889012802D00BA0F7F77FFF00BF21
:10FEE000304600F011FC041E04D100BF00BF001F0B
:10FEF000BDE8FE8F4346324639462846CDE9009A92
:10FF0000029400F007F8F3E7702D3E726566203D1D
:10FF10003D2031002DE9F84F05460F4690469A46A0
:10FF2000DDF828B00C9E00BFE889012802D032A07D
:10FF3000F7F754FF00BFB8F1000F43D04FF014099A
:10FF40001421284604F032FF28B100BF00BF6FF033
:10FF50000100BDE8F88F6C6800BF6889142802D2E0
:10FF600028A0F7F73BFF00BF84F808A00B98607249
:10FF7000D8F80000206148464FEAE97109EB917119
:10FF8000C1F3870141F04001217084F801B0288954
:10FF900001F01DFA60800020E0802648008801F012
:10FFA00016FAA08023480088401C224908800FB11F
:10FFB000386810B97068E06001E03868E0600020DF
:10FFC000608103E06C6820690090E84600BF00BFD4
:10FFD000308D48B12889318D884205DD4246314651
:10FFE0002846FFF76BFDB4E700BF00BF4246294635
:10FFF000304673699847ACE7702D3E726566203DC8
:020000040801F1
:100000003D203100636865636B207468617420660D
:100010006972737420706275662063616E20686F08
:100020006C64207374727563742069705F686472A5
:1000300000000000840100202DE9F84F80460020D8
:100040000090D8F80450287800F00F001421B1EB8C
:10005000800F02D000BF00BFB4E0E88801F0D7F9FC
:10006000C0F30C004FF6FF7101EAC00A688801F086
:10007000CEF9297801F00F01A0EB81001FFA80FB77
:10008000404604F0ACFC06465248018888190A280C
:100090000CDD3146284600F0CBFA20B14D480088EF
:1000A00030440A2802DD00BF00BF8BE04A480468E4
:1000B00014E06069E968884209D1A0692969884229
:1000C00005D1A089A988884201D1012000E0002043
:1000D00010B100BF00BF03E000942468002CE8D1F9
:1000E00000BF34B93146284600F0D6F9044694B929
:1000F00068E0E88801F08BF9C0F30C0058B9E0899A
:1001000001F085F9C0F30C0028B11422294604F14E
:100110000800F0F7DCF82F48008830442D490880AB
:10012000A87900F0200040B9A07F40F00100A0773E
:100130000AEB0B00A08300BF00BF4146204600F041
:100140004DF8D0B3A08B1430A08360684068076876
:1001500060684568142204F108012846F0F7B7F8F2
:10016000A08B01F034F968800020E88068811421B8
:100170002846FFF71DFC6881D4F804800CE0D7F80E
:1001800004906FF01301384604F010FE39464046E3
:1001900004F0B0FBD9F80070002FF0D12046009990
:1001A00000F052F9404604F01AFC0A490988081A7E
:1001B000084908804046BDE8F88FFFE700BF00BF50
:1001C0000020F8E700BF00BF404604F04FFD0020CC
:1001D000F1E700008C010020880100202DE9FC5F80
:1001E00006460F4600254FF0010BD7F804A0BAF8D9
:1001F000020001F00CF99AF8001001F00F01A0EBD9
:10020000810080B20090BAF8060001F000F9C0F356
:100210000C004FF6FF7101EAC000019000BF00BF63
:100220007C68002020600198A080DDE9001008446F
:10023000E080D6F804902EE0D9F80480A088B8F8C1
:100240000410884210DAC4F800905DB1A088E988F3
:10025000884204DBE088B8F80410884200DD86E0BC
:100260002F6000E0776019E0A088B8F80410884299
:1002700000D17CE0A088B8F80610884200DA76E069
:1002800035B1E888B8F80410884201D04FF0000B6F
:10029000D8F800904546B9F1000FCDD100BFB9F1B3
:1002A000000F19D185B100BFE888A188884202DD1E
:1002B00035A0F7F793FD00BF2F60E888A18888423A
:1002C0000AD04FF0000B07E000BF706810B136A0F5
:1002D000F7F784FD00BF7760B07F00F001000028D1
:1002E00043D0BBF1000F3DD070684068808810B1EA
:1002F0004FF0000B36E02546D4F800900BE0D9F81B
:100300000440E888A188884202D04FF0000B05E045
:100310002546D4F80090B9F1000FF0D100BFBBF131
:10032000000F1FD000BF706810B92DA0F7F756FD61
:1003300000BF00BF70684068A04202D128A0F7F754
:100340004DFD00BF00BF206810B129A0F7F746FDA2
:1003500000BF00BFE088B18B884202D02DA0F7F724
:100360003DFD00BF5846BDE8FC9F0020FBE7384636
:1003700004F035FB33490988081A324908803846A9
:1003800004F074FC0020EEE7636865636B2066721E
:1003900061676D656E747320646F6E2774206F766D
:1003A00065726C61700000006E6F20707265766916
:1003B0006F757320667261676D656E742C2074684A
:1003C0006973206D7573742062652074686520669A
:1003D0006972737420667261676D656E74210000C6
:1003E00073616E69747920636865636B0000000057
:1003F00076616C69646174655F6461746167726180
:100400006D3A6E6578745F70627566213D4E554C2D
:100410004C00000076616C69646174655F646174AE
:10042000616772616D3A646174616772616D2065C4
:100430006E64213D646174616772616D206C656EEC
:10044000000000008C01002070B504460D460A48EB
:100450000068A04203D108492068086007E000BF97
:1004600015B906A0F7F7BAFC00BF2068286021463E
:10047000052001F0BBFF70BD8801002073616E692B
:10048000747920636865636B206C696E6B656420AA
:100490006C6973740000000070B505460E460520B7
:1004A00002F008F8044674B93146284600F0C0F856
:1004B000B04203DB052001F0FDFF04461CB900BF7C
:1004C00000BF002070BD20212046EFF719FF032058
:1004D000E07706480068206004480460142229463A
:1004E00004F10800EFF7F3FE2046EBE78801002057
:1004F0002DE9F04704468846002500BFA04502D1FB
:1005000033A0F7F76BFC00BFB8F1000F08D000BFB5
:10051000D8F80000A04202D030A0F7F75FFC00BF7F
:100520006068D0F80490B9F80400F8B96768D9F8A1
:1005300000006060142204F108017868EFF7C7FE3C
:1005400001213846FFF7BCF9384604F048FA064660
:1005500000BFA819B0F5803F02DB25A0F7F73EFCED
:1005600000BFA81985B2384604F080FB676817E021
:10057000D7F80490BA46D9F80070504604F02FFA24
:10058000064600BFA819B0F5803F02DB18A0F7F7B8
:1005900025FC00BFA81985B2504604F067FB00BFD8
:1005A000002FE5D141462046FFF74EFF00BF184817
:1005B0000088A84202DA17A0F7F710FC00BF144821
:1005C0000088401B124908802846BDE8F0870000DB
:1005D0007072657620213D206970720070726576B8
:1005E0002D3E6E657874203D3D20697072000000DC
:1005F00070627566735F6672656564202B20636C3C
:10060000656E203C3D20307866666666000000001E
:100610008C01002069705F72656173735F70627531
:1006200066636F756E74203E3D20636C656E0000DE
:100630002DE9F05F05468946002700BF0026B34636
:10064000B246194804681DE06069E968884207D12C
:10065000A0692969884203D1A089A988884201D06C
:10066000012000E0002048B10AF1010A0EB9264637
:1006700004E0E07FF17F884200DC2646206800B17C
:10068000A3462468002CDFD12EB159463046FFF72F
:100690002FFF804647444F4502DABAF1010FCDDC07
:1006A0003846BDE8F09F00008801002010B50446E0
:1006B00000BF00BF00F00AF8002203494FF47A702F
:1006C00005F014FC10BD0000AD06010870B5002651
:1006D0000C48046813E0E07F002807DDE07F401E3F
:1006E000E07700BF00BF2646246808E000BF00BFD7
:1006F0002546246831462846FFF7FAFE00BF002C45
:10070000E9D170BD8801002010B502461248016889
:100710000FE091F8310000F0010048B110688B68DB
:100720001840D1E901342340984201D1084610BD58
:1007300009680029EDD10948006830B10748006810
:1007400090F8310000F0010018B900BF00BF002090
:10075000EDE702480068EAE71001002014010020DC
:1007600038B504466946204600F006F808B10098FE
:1007700038BD4FF0FF30FBE72DE9FF4706468846BE
:100780006F46347800BF302C01DB392C03DD0020AC
:1007900004B0BDE8F08700254FF00A09302C0ED1D7
:1007A000701C06460478782C01D0582C05D14FF0E7
:1007B0001009701C0646047801E04FF0080900BFDC
:1007C000302C09DB392C07DCA4F1300005FB0905CE
:1007D000701C06460478F3E7B9F1100F1BD1302CDA
:1007E00001DB392C07DD612C01DB662C03DD412C9C
:1007F00011DB462C0FDC612C03DB7A2C01DC612140
:1008000000E0412104F10A00401A40EA0515701C7D
:1008100006460478D4E700BF00BF2E2C09D103A8F8
:10082000874201D30020B3E720C7701C0646047836
:10083000A9E700BF00BF6CB1202C0BD00C2C09D055
:100840000A2C07D00D2C05D0092C03D00B2C01D07D
:1008500000209DE76846381A012101EBA000052819
:100860002AD2DFE800F00305060F1B0000208FE707
:1008700028E0B5F1807F01D3002089E7009845EAA0
:1008800000651FE0B5F5803F01D3002080E70098A8
:100890000006019940EA0140054313E0FF2D01D90C
:1008A000002075E700980006019940EA014002998E
:1008B00040EA0120054305E000BF08A0F7F78EFAE3
:1008C00000BF00BF00BFB8F1000F04D0284600F001
:1008D00071FDC8F8000001205AE70000756E6861DC
:1008E0006E646C656400000010B504461022024975
:1008F000204600F003F810BD905B01202DE9FC4775
:1009000006460B4614464FF0000C3068019019461D
:1009100001AA00273CE0002500BF10784FF00A092B
:1009200090FBF9FA09FB1A0000F0FF08107890FB21
:10093000F9F0107008F1300000F0FF0A284605F1C8
:10094000010909F0FF050DF800A010780028E4D196
:100950000BE060460CF1010CA04202DB0020BDE878
:10096000FC871DF8050001F8010B281EA5F10109FF
:1009700009F0FF05EDD160460CF1010CA04201DB4E
:100980000020ECE72E2001F8010B521C781CC7B2A6
:10099000042FC0DB4FF00009481E014680F800908C
:1009A0001846DCE770B505462C4600BF14B90AA00E
:1009B000F7F714FA00BF00BFAC4202D009A0F7F766
:1009C0000DFA00BF606910B1606904F04FF920466C
:1009D000FFF766F970BD000070637220213D204E64
:1009E000554C4C00706372203D3D207000000000AB
:1009F00010B502468C7ECB7E44EA03201378032B8D
:100A000005D10C7D4B7D44EA032340EA034010BD31
:100A10002DE9F04F87B03BA4474800680690464850
:100A200008300068059044481030006804900021A8
:100A3000002055E002464FEAE07B00EB9B7B4FEA4B
:100A4000AB0BA0EB8B0B4FEACB0EDDF818B02BFAFB
:100A50000EFB0BF0FF031F0903F00F0C4FEAE07BC6
:100A600000EB9B7B4FEAAB0BA0EB8B0B4FEACB0E63
:100A7000DDF814B02BFA0EFB0BF0FF054FEA15184A
:100A800005F00F094FEAE07B00EB9B7B4FEAAB0BD5
:100A9000A0EB8B0B4FEACB0EDDF810B02BFA0EFB60
:100AA0000BF0FF064FEA161A06F00F02009207EB52
:100AB00008025244A25C0DF1040B01F1020E0BF886
:100AC0000E200CEB090B009A5A4414F802B00DF1F9
:100AD000040ECA1C0EF802B0421CD0B28A1CD1B25D
:100AE0000829A7DB00208DF80E004C208DF80400AB
:100AF00052208DF8050001A91048EFF74CFC07B013
:100B0000BDE8F08F303132333435363738396162F1
:100B1000636465666768696A6B6C6D6E6F7071722D
:100B2000737475767778797A4142434445464748ED
:100B3000494A4B4C4D4E0000107AFF1FE8530020ED
:100B400070B50446F0F73CFE062084F82A002148E0
:100B50000668022084F82B002C200655C6F30721D6
:100B60002D200155C6F307412E200155310E2F20AF
:100B7000015500213020015504F12B010020F1F72F
:100B8000A3FD40F2DC502085222084F831000522AC
:100B900011491248F0F746FF082211491148F0F7B1
:100BA000B7FE002506E00F4901EB05100121F0F723
:100BB000E1FE6D1C082DF6DB002507E0074901EB7F
:100BC00005104FF44001F0F755FF6D1C052DF5DBC6
:100BD00070BD0000107AFF1F6CAB00207C7B0020F2
:100BE000CC7B0020FC7A00202DE9F04F87B04FF03D
:100BF00000080024A1460027002003906846F1F772
:100C000077F89DE8070004AB07C3DDF810A0DDF816
:100C100014B0BAF1000F07D01FFA8AF10322104670
:100C200003F060FC804603E0002007B0BDE8F08FD1
:100C3000B8F1000F2ED0069E0024454628E06F89AB
:100C40004FF0000915E040F2F4531A1B0BEB0401BE
:100C50006B6803EB0900EFF73AFBF668D6F808B0CB
:100C600040F2F450001B3F1A40F2F450001B814444
:100C70000024381940F2F4518842E4D80BEB040107
:100C80006A6802EB09003A46EFF721FB3C442D6805
:100C9000002DD4D1069E0020039006E04FF00040C6
:100CA0003060F6680398401C03900B480068816828
:100CB00003988142F2D800200749096888600748F4
:100CC000406900F0800020B1802004494861002084
:100CD00088604046A9E700005400002000900240D0
:100CE0002DE9FC5F8B4639480068806800904FF022
:100CF000000900240026A24601AA00213448006809
:100D0000F4F794FE3148D0F8008000BF5D4644E01F
:100D1000D8F8000000F0004010B16FF0010743E088
:100D20006E894FF0000A25E040F2F4531A1B6B68FD
:100D300003EB0A01009B1819EFF7C9FAD8F80C80E9
:100D4000D8F8000000F0004010B16FF007072BE06A
:100D5000D8F80800009040F2F450001B361A40F218
:100D6000F450001B824440F2F450001B48441FFA28
:100D700080F90024301940F2F4518842D4D86A68CE
:100D800002EB0A01009A10193246EFF7A0FA344438
:100D900009EB06001FFA80F92D68002DB8D14846EE
:100DA000F1F7BEFD002700BF0A48406900F02000AF
:100DB00020B12020074948610020486004480068AD
:100DC000F4F7AAFE3846BDE8FC9F00004C00002066
:100DD000A40100200090024010B586B00021084612
:100DE00008F018FF00200590049003902748284938
:100DF000002203ABCDE90021029004AA05A92548F1
:100E000003F00AFA234803F073FA23480068112814
:100E100022D1204890F8310040F010001D4981F89F
:100E20003100084603F014FBF1F752FE1948F9F7B8
:100E3000D9FC02E00A20F5F7F9F816484068059950
:100E40008842F7D01348001DFFF74EFD04462146A7
:100E500012A0F6F7C3FF0CE00E4803F051FA0D485C
:100E600090F8310020F010000A4981F83100F1F7C4
:100E70003FFE1049074803F0A3FA00220E494FF441
:100E8000FA6005F033F806B010BD00008D9C010833
:100E9000F5D300087CD900206C00002064686370E2
:100EA0002069705F61646472206973202573200D6E
:100EB0000A00000039C60008B5D4000870B5054620
:100EC000002600BF00BF2846FDF79AFE04460CB975
:100ED000701E70BD206840B120680078102801D1D4
:100EE000012000E00020064606E000BF606810B167
:100EF00006A0F6F773FF00BF206802F0D1FC314670
:100F00002046FDF75BFD0020E3E70000736F636B95
:100F10002D3E6C61737464617461203D3D204E55BB
:100F20004C4C00002DE9F84F81460E46904648464D
:100F3000FDF766FE04461CB94FF0FF30BDE8F88FA0
:100F400000BFB8F1100F05D17078022802D106F069
:100F5000030050B122A0F6F741FF00BF2848806B84
:100F6000206100BF4FF0FF30E8E700BF37463E4644
:100F7000787830B900BF00BF206802F0A5FC0546B4
:100F800014E078680090B7F802A000BF00BF00BF6F
:100F900000BF00BF00BF504600F039FA83465A46F2
:100FA0006946206802F03EFC054600BF85B100BFDF
:100FB00000BF00BF6842102804D21148694250F8AF
:100FC000210000E00520206100BF4FF0FF30B5E7B1
:100FD00000BF00BF00BF0020206100BF00BFADE721
:100FE0006C7769705F636F6E6E6563743A20696ECB
:100FF00076616C69642061646472657373000000DB
:10100000A45504082DE9F04788B082468846154665
:101010009946109E00275046FDF7F2FD04461CB984
:10102000781E08B0BDE8F087B9F1000F00D036B9DE
:1010300000BF0E20206100BF4FF0FF30F1E7B8F194
:10104000000F3FD0B8F1060F4CD0A8F6FF70002873
:1010500065D141F20601681A8D4217D00ADC022DD3
:101060000FD0082D10D0202D0CD0A5F580500538BC
:1010700010BB0AE0012806D0022808D004281BD1A2
:101080000AE000BF00BF00BF00BF00BF00BF306864
:10109000042800D2162713E03068042800D216274F
:1010A00020680078202805D120684068007C00F086
:1010B000020000B1612703E000BF00BF5C2700BF52
:1010C00000BF30E0012D02D0022D05D100BF3068F5
:1010D000042800D2162703E000BF00BF5C2700BF32
:1010E00000BF20E03068042801D216271BE02068EA
:1010F0000078102801D0002093E7062D09D2DFE800
:1011000005F008030405060700BF00BF00BF00BFCD
:1011100003E000BF00BF5C2700BF00BF03E000BFCB
:1011200000BF5C2700BF00BF2FB100BF276100BF19
:101130004FF0FF3075E70194CDF808A0CDF80C8092
:101140000495CDF8149006968DF81C70012201A923
:10115000094808F02FFD216801F10C00002104F07E
:1011600004FE9DF91C7000BF276100BF17B14FF04E
:10117000FF3056E7002054E77D1101082DE9F047C4
:10118000064600BF16B97EA0F6F728FE00BFB0469F
:101190004646D8F80040D8F804A0D8F80890D8F807
:1011A0000C70D8F81050B9F1000F6ED0B9F1060FDD
:1011B0006CD0A9F6FF70002869D141F20601781AB7
:1011C0008F425DD00BDC022F10D0082F10D0202FC3
:1011D0000DD0A7F580500538002860D14BE00128DC
:1011E0002BD002280CD0042859D151E000BF00BFF9
:1011F00020684068007A3840286000BF00BF54E093
:101200002068007800F0F000102806D0202807D0D1
:10121000402808D1032028600BE00120286008E066
:101220000220286005E020680078286000BF00BF29
:1012300000BF00BF00BF00BF37E0206910B12069C8
:10124000732811D100BF206890F90800404210288F
:1012500007D2206890F9080040424C4951F820001C
:1012600000E00520206100BF206928600020206187
:1012700000BF00BF19E02068D0F81C01286014E00E
:101280002068D0F8200128600FE010E029E068E035
:1012900020684068007C00F00100286005E000BF85
:1012A0003BA0F6F79BFD00BF00BF00BF5FE0012F32
:1012B00008D0022F0DD120684068807A286000BFD6
:1012C00000BF0CE020684068407A286000BF00BF83
:1012D00005E000BF2EA0F6F781FD00BF00BF00BFF4
:1012E00045E0062F35D2DFE807F034030C14202C3C
:1012F00020684068807FC0F38010286000BF00BF76
:101300002DE020684068D0F88C00286000BF00BF46
:1013100025E020684068D0F88C004FF47A71B0FB6B
:10132000F1F0286000BF00BF19E020684068D0F8E5
:1013300090004FF47A71B0FBF1F0286000BF00BF5D
:101340000DE020684068D0F89400286000BF00BF1E
:1013500005E000BF0EA0F6F741FD00BF00BF00BFD3
:1013600005E000BF0FA0F6F739FD00BF00BF00BFCA
:10137000216801F10C0004F090FDBDE8F087000049
:1013800061726720213D204E554C4C00A455040845
:10139000756E68616E646C6564206F70746E616DEB
:1013A00065000000756E68616E646C6564206C6534
:1013B00076656C000146080601F47F4240EA02208F
:1013C00001F47F0240EA122040EA116070470146B2
:1013D0000806000C40EA1120704710B504F0ECFC40
:1013E00000F0ECFD01F034F802F06CFF00F0C0FCFE
:1013F00008F070FE05F02CFBFAF736F804F0E8FD73
:1014000010BD00B503461846FFF7D4FF00BD00B578
:1014100002461046FFF7DBFF00BD7CB504460D46D3
:101420001646002000900346324629460190204689
:1014300000F012F87CBD2DE9FC4104460D4616462D
:101440001F46002000903B46324629460190204628
:1014500000F002F8BDE8FC812DE9FF4F8BB0164685
:101460009846DDF8649000200A900025069000BFA1
:1014700000BF0B98FDF7C4FB04461CB9681E0FB0F3
:10148000BDE8F08F00BF00BF00BF606810B16068AA
:101490000A9062E008F0080028B9206890F824015A
:1014A00000F00200C0B1B4F90A00002814DC002DDD
:1014B00009DD2946206802F0C3FD00BF002020613D
:1014C00000BF2846DBE700BF00BF00BF0B20206144
:1014D00000BF4FF0FF30D2E720680078102805D118
:1014E0000AA9206802F08AFD834604E00AA9206860
:1014F00002F014FC834600BF00BFBBF1000F23D0F5
:10150000002D09DD2946206802F09AFD00BF002069
:10151000206100BF2846B2E700BF00BF00BFCBF18B
:101520000000102805D26848CBF1000150F82100D6
:1015300000E00520206100BF0BF10C0008B900207D
:101540009DE74FF0FF309AE700BF0A9810B95FA0FF
:10155000F6F744FC00BF0A98606020680078102805
:1015600002D10A98099002E00A9800680990099847
:10157000B0F808A000BF00BF2089AAEB00001FFA46
:1015800080FA564501D9574600E0B7B223890C9836
:1015900041193A46099803F0F7FA3D44206800786B
:1015A000102817D100BFBE4202D24BA0F6F716FC9E
:1015B00000BFF61B5EB10998407B00F0010030B916
:1015C000B4F90A00002802DD08F0010020B1012072
:1015D000069001E0012006900698E8B31898E0B361
:1015E000B9F1000F3DD020680078102808D105A877
:1015F0000890002307AA2068089902F091FA05E0F4
:101600000A98083008900A98808907900020019075
:1016100002900390049010208DF8040002208DF8B1
:101620000500BDF81C00FFF7D2FEADF806000898D3
:1016300000680290D9F80000102802D91020C9F8DB
:10164000000001A9D9F800201898EEF740FE00BF6D
:1016500000BF00BF00BF01E004E002E000BF00BF28
:1016600000BF00BF08F00100F0B920680078102822
:101670000AD1AAEB0700002806DD0A9860602089DD
:101680003844208100BF0FE000206060208100BF4F
:1016900000BF20680078102803D10A9803F0E6FA0A
:1016A00002E00A9801F0BAFF069800283FF4EBAE7A
:1016B000002D03DD2946206802F0C2FC00BF002097
:1016C000206100BF2846DAE6A4550408627566204A
:1016D000213D204E554C4C00696E76616C6964204A
:1016E000636F70796C656E2C206C656E20776F75FA
:1016F0006C6420756E646572666C6F770000000024
:101700002DE9FE4F8046894692461E4600BF00BF27
:101710004046FDF775FA04461CB94FF0FF30BDE8AE
:10172000FE8F20680078102809D0002000903346F2
:10173000524649460190404600F032F8EFE706F085
:10174000100008B1022000E0002040F0010006F087
:10175000080109B1042100E0002140EA010700204E
:10176000029002A800903B4652464946206802F08B
:10177000CBFC054600BF00BF00BF6842102804D262
:101780000648694250F8210000E00520206100BFB2
:101790000DB90298C3E74FF0FF30C0E7A455040825
:1017A0002DE9FF4F85B09146DDE9125A0598FDF706
:1017B00027FA064626B94FF0FF3009B0BDE8F08F92
:1017C00030680078102806D14A46089BDDE90501FB
:1017D000FFF796FFF1E700BFB9F5803F02D32DA0D8
:1017E000F6F7FCFA00BF1FFA89FB00BF15B9BAF182
:1017F000000F13D0BAF1100F05D16878022802D17A
:1018000005F0030050B12CA0F6F7E8FA00BF32480B
:10181000806B306100BF4FF0FF30CEE700BF2F4636
:1018200000200290019045B1786803907888FFF716
:10183000EEFD8046ADF8108005E04FF00008002076
:101840000390ADF8100000BF00BF00BF00BF00BF95
:1018500000BF5A4601A8069901F012FF044624B9B8
:1018600001A9306802F006FC044601A801F0E6FE7A
:1018700000BF6042102804D21748614250F821008E
:1018800000E00520306100BF0CB9584695E74FF0E5
:10189000FF3092E76C7769705F73656E64746F3ABE
:1018A0002073697A65206D75737420666974206988
:1018B0006E207531365F74006C7769705F73656E8A
:1018C00064746F3A20696E76616C69642061646447
:1018D0007265737300000000A45504082DE9F043FD
:1018E00087B081460F46154698464846FDF788F969
:1018F000044600261CB9701E07B0BDE8F083B8F19D
:10190000000F06D100BF0E20206100BF4FF0FF3056
:10191000F2E79FB3062F42D0A7F6FF7000285BD1F5
:1019200041F20501681A8D420CD004DC082D08D064
:10193000202D1DD104E0012805D0052818D107E08D
:1019400000BF00BF00BF0E98042800D2162613E087
:101950000E98042800D2162620680078202805D189
:1019600020684068007C00F0020000B1612603E0BE
:1019700000BF00BF5C2600BF00BF31E0FFE7012DC4
:1019800002D0022D05D100BF0E98042800D21626E1
:1019900003E000BF00BF5C2600BF00BF20E00E9840
:1019A000042801D216261BE020680078102801D0F8
:1019B0000020A1E7062D09D2DFE805F008030405A1
:1019C000060700BF00BF00BF00BF03E000BF00BFAD
:1019D0005C2600BF00BF03E000BF00BF5C2600BF65
:1019E00000BF2EB100BF266100BF4FF0FF3083E77C
:1019F0000094CDF8049002970395CDF810800EA8BE
:101A000005908DF81860012269460A4808F0D2F85E
:101A1000216801F10C00002104F0A7F99DF918607C
:101A200000BF266100BF16B14FF0FF3064E7002011
:101A300062E70000391A01082DE9F047064600BFA9
:101A400016B96CA0F6F7CAF900BFB0464646D8F8FA
:101A50000040D8F804A0D8F80890D8F80C70D8F84E
:101A60001050B9F1000F51D0B9F1060F68D0A9F6A6
:101A7000FF70002876D141F20501781A8F421FD0FD
:101A800004DC082F08D0202F38D104E001281CD016
:101A9000052833D11EE000BF286838B120684068AF
:101AA000007A384321684968087206E02068406877
:101AB000007AB84321684968087200BF00BF23E07C
:101AC00028682168C1F81C011EE028682168C1F857
:101AD000200119E0286840B120684068007C40F08F
:101AE000010021684968087407E020684068007CAC
:101AF00020F0010021684968087405E000BF40A09B
:101B0000F6F76CF900BF00BF00BF6BE0012F08D0F3
:101B1000022F0DD1287821684968887200BF00BF64
:101B20000CE0287821684968487200BF00BF05E0D2
:101B300000BF33A0F6F752F900BF00BF00BF51E06D
:101B4000062F41D2DFE807F040031A222D3828681B
:101B500048B120684068807F40F0400021684968B3
:101B6000887708E038E020684068807F20F04000F7
:101B700021684968887700BF00BF2BE0286821688A
:101B80004968C1F88C0000BF00BF23E04FF47A71B0
:101B90002868484321684968C1F88C0000BF00BF2D
:101BA00018E04FF47A712868484321684968C1F801
:101BB000900000BF00BF0DE0286821684968C1F8A7
:101BC000940000BF00BF05E000BF0DA0F6F706F9C6
:101BD00000BF00BF00BF05E000BF0EA0F6F7FEF893
:101BE00000BF00BF00BF216801F10C0004F055F9EF
:101BF000BDE8F08761726720213D204E554C4C00B6
